:1000000000000120A1F50000C9F50000CBF50000BB
:10001000CDF50000CFF50000D1F500000000000094
:10002000000000000000000000000000D3F5000008
:10003000D5F5000000000000D7F50000D9F500005C
:10004000DBF50000DBF5000059FB0000DBF50000EC
:100050008DA00000DBF50000DBF50000DBF5000003
:10006000DBF50000DBF50000DBF50000DBF5000050
:10007000DBF50000DBF50000DBF50000DBF5000040
:10008000DBF500001DFF0000DBF50000DBF50000E4
:10009000DBF50000DBF50000DBF50000DBF5000020
:1000A000DBF50000DBF50000DBF50000DBF5000010
:1000B000DBF50000DBF500000000000000000000A0
:1000C000DBF50000DBF50000DBF50000DBF50000F0
:1000D000DBF50000DBF50000DBF5000000000000B0
:1000E0000000000000000000000000000000000010
:1000F0000000000000000000000000000000000000
:1001000000000000000000000000000000000000EF
:1001100000000000000000000000000000000000DF
:1001200000000000000000000000000000000000CF
:1001300000000000000000000000000000000000BF
:1001400000000000000000000000000000000000AF
:10015000000000000000000000000000000000009F
:10016000000000000000000000000000000000008F
:10017000000000000000000000000000000000007F
:10018000000000000000000000000000000000006F
:10019000000000000000000000000000000000005F
:1001A000000000000000000000000000000000004F
:1001B000000000000000000000000000000000003F
:1001C000000000000000000000000000000000002F
:1001D000000000000000000000000000000000001F
:1001E000000000000000000000000000000000000F
:1001F00000000000000000000000000000000000FF
:1002000010B5054C237833B9044B13B10448AFF350
:1002100000800123237010BDA40200200000000014
:10022000608E010008B5034B1BB103490348AFF3CF
:10023000008008BD00000000A8020020608E0100C0
:10024000154B002B08BF134B9D46A3F5803A0021A8
:100250008B460F461348144A121A12F092F90F4BAC
:10026000002B00D098470E4B002B00D09847002061
:10027000002104000D000D48002802D00C48AFF307
:10028000008012F0C7F8200029000FF087FE11F05F
:100290000FFF00BF00000800000001200000000068
:1002A00000000000A40200209409002000000000CB
:1002B00000000000002070470020704700207047B9
:1002C00000207047F0B5044685B00E4668461146DA
:1002D0001F4609F047FB23686A465D6A31463B4684
:1002E0002046A84705B0F0BDF0B5044685B00E46DF
:1002F000684611461F4609F045FA23686A465D6A5A
:1003000031463B462046A84705B0F0BD70B590B0D9
:100310000C4615461E4605F001FA48B364B3214663
:100320004022684613F001F92F21684613F094F833
:1003300028B9234603224021684609F095FA3F2256
:100340003146684613F0CBF80C480DF0FDFF78B14C
:100350000B4B93F90030062B0CD10A4B93F900306C
:1003600043B901232A46694604480EF04AFA01209F
:1003700010B070BD0020FBE72046F9E7E403002041
:10038000DC030020B403002007B5002300931A46C5
:10039000194603480EF03CFF03B05DF804FB00BFB4
:1003A000C002002007B5002300931A4619460348EF
:1003B0000EF02EFF03B05DF804FB00BFC802002062
:1003C0000020704700207047406808B508B101F070
:1003D0006DFF012008BD13B5002204461146684692
:1003E00003F02EFE606801F061FF052805D80123A7
:1003F00003FA00F010F0250F0BD161684FF4007282
:10040000684604F00FFA0021684604F0DBF802B0F9
:1004100010BD0020FBE713B50022044611466846D4
:1004200003F00EFE2046FF22694604F046F92046FE
:1004300002B010BD07B5002300931A4619460348C1
:100440000EF0E6FE03B05DF804FB00BFD002002012
:10045000704743683BB1B0F90A00012806D002DBBF
:100460000338022801D9002070470220704700009D
:100470002DE9FF4102AC84E80600064638493948B8
:100480009DF828501F460EF00BFF204604F034FB69
:10049000204603F053FF40BB204604F0B5F9052881
:1004A00004D8DFE800F015221603031605462E498E
:1004B0002C480EF0F5FE0A2229462A480EF059FF74
:1004C00028480EF0FDFE204604F016FB002009E04F
:1004D000012533680095DD6B94E806003B46304605
:1004E000A847012004B0BDE8F081204604F0D6F80A
:1004F000012812D0022830D01C491A480EF0D0FE34
:10050000204604F0CBF80A22014616480EF04AFFB6
:1005100014480EF0D5FE0125C9E70021204603F05E
:10052000A3FF13280EDC1E21204604F00DF871688D
:100530004FF40072204604F033FE4FF420617068DF
:1005400002F07EFB336801250095D3F83C8094E8E7
:1005500006003B463046C047C3E700230393F1E75C
:10056000C46F01006C030020DA6F0100CD6F010041
:1005700008B511B9B0F9080008BDB0F90A208A42DF
:1005800003DC0089084400B2F6E7406801F032FF5E
:10059000F9E7000007B5002300931A4619460348FF
:1005A0000EF036FE03B05DF804FB00BFD802002059
:1005B0000A460068022100F06FBD000070B50368B4
:1005C0000546F3B17221FFF7F3FF28680E4E03686A
:1005D0000021DB69984700242868042C03680CD0AC
:1005E000DB689847A35D984205D0286803685B6A7A
:1005F0009847002070BD0134EEE75B6A9847012000
:10060000F8E71846F6E700BF347001002DE9F04125
:10061000036804461BB900263046BDE8F081FFF7A9
:10062000CDFF07460028F6D0254672212046FFF769
:10063000BFFF55F8100B03680421DB69984704F1EC
:100640001608002620680368DB689847C0B205F8E2
:10065000010B0138C0B2FD2898BF3E46A845F1D134
:10066000206803685B6A9847D6E7F8B503680446D4
:100670000F4613B900252846F8BDFFF79FFF054632
:100680000028F7D061212046FFF792FF2068036819
:100690002646DB690421984756F8100B03680622AA
:1006A0005B68394698473B682361BB88B380206804
:1006B00003685B6A9847DEE770B5036804460D4639
:1006C000164613B90025284670BDFFF777FF0028AE
:1006D000F8D072212046FFF76BFF206803684021A5
:1006E000DB699847731E2A46002120680FF0BCF88A
:1006F00006B2206803685B6A9847002EE2D00023A8
:10070000AB55E0E738B5036804460D460BB9002049
:1007100038BDFFF753FF0028F9D0284612F0D7FE66
:100720000F28F4D872212046FFF742FF20680368A3
:100730004021DB699847294620680EF0BAFD206801
:10074000036800211B6898470546206803685B6AB8
:100750009847281C18BF0120DAE738B5036804461B
:100760000D460BB9002038BDFFF728FF0028F9D04F
:10077000284612F0ACFE0F28F4D872212046FFF76D
:1007800017FF206803685021DB69984729462068D5
:100790000EF08FFD2068036800211B68984705460E
:1007A000206803685B6A9847281C18BF0120DAE7B5
:1007B00070B5036804460D46164613B90025284651
:1007C00070BDFFF7FBFE0028F8D072212046FFF72E
:1007D000EFFE206803682021DB699847731E2A46D4
:1007E000002120680FF040F806B2206803685B6AB9
:1007F0009847002EE2D00023AB55E0E738B50368F8
:1008000004460D460BB9002038BDFFF7D7FE00287F
:10081000F9D0284612F05BFE1F28F4D8722120463A
:10082000FFF7C6FE206803682021DB699847294648
:1008300020680EF03EFD2068036800211B68984781
:100840000546206803685B6A9847281C18BF01208A
:10085000DAE773B5036805460E461BB90024204647
:1008600002B070BDFFF7AAFE04460028F6D0722140
:100870002846FFF79DFE286803681021DB6998472A
:1008800004220DEB020128680EF0D9FF01993046D1
:100890000EF0DBFC286803685B6A98473379002B0D
:1008A000DCD0FF2BDBD17379FF2BD8D1B379FF2BB1
:1008B000D5D1F479FF3C18BF0124D0E773B50368A4
:1008C00005460E461BB90024204602B070BDFFF756
:1008D00075FE04460028F6D072212846FFF768FE10
:1008E000286803681C21DB69984704220DEB02018C
:1008F00028680EF0A4FF019930460EF0A6FC286887
:1009000003685B6A98473379002BDCD0FF2BDBD17F
:100910007379FF2BD8D1B379FF2BD5D1F479FF3C74
:1009200018BF0124D0E773B5036805460E461BB90E
:100930000024204602B070BDFFF740FE04460028A8
:10094000F6D072212846FFF733FE28680368142189
:10095000DB69984704220DEB020128680EF06FFF57
:10096000019930460EF071FC286803685B6A98476D
:100970003379002BDCD0FF2BDBD17379FF2BD8D15F
:10098000B379FF2BD5D1F479FF3C18BF0124D0E710
:1009900073B5036805460E461BB90024204602B015
:1009A00070BDFFF70BFE04460028F6D072212846E2
:1009B000FFF7FEFD286803681821DB6998470422C9
:1009C0000DEB020128680EF03AFF019930460EF057
:1009D0003CFC286803685B6A98473379002BDCD0BD
:1009E000FF2BDBD17379FF2BD8D1B379FF2BD5D176
:1009F000F479FF3C18BF0124D0E737B54B68019369
:100A00000368044613B9002003B030BDFFF7D6FDDC
:100A10000028F8D072212046FFF7CAFD206803683D
:100A20001021DB6998472068036804225B680DEB9E
:100A3000020198470546206803685B6A9847281CAE
:100A400018BF0120E0E737B54B68019303680446FF
:100A500013B9002003B030BDFFF7B0FD0028F8D077
:100A600072212046FFF7A4FD206803681C21DB6982
:100A700098472068036804225B680DEB02019847E1
:100A80000546206803685B6A9847281C18BF012048
:100A9000E0E737B54B6801930368044613B90020BB
:100AA00003B030BDFFF78AFD0028F8D07221204640
:100AB000FFF77EFD206803681421DB6998472068F2
:100AC000036804225B680DEB020198470546206825
:100AD00003685B6A9847281C18BF0120E0E737B518
:100AE0004B6801930368044613B9002003B030BD7E
:100AF000FFF764FD0028F8D072212046FFF758FD6B
:100B0000206803681821DB6998472068036804227D
:100B10005B680DEB020198470546206803685B6A35
:100B20009847281C18BF0120E0E713B577230093EE
:100B300003680446A3B1FFF741FD88B17221204646
:100B4000FFF736FD206803680C21DB699847042213
:100B5000694620680EF073FE206803685B6A984758
:100B6000009B0020DAB262F30700C3F3072262F3AE
:100B70000F20C3F3074262F317401B0E63F31F609D
:100B800002B010BD37B501910368044613B90020C7
:100B900003B030BDFFF712FD0028F8D072212046C7
:100BA000FFF706FD206803680C21DB699847206881
:100BB000036804225B680DEB020198470546206834
:100BC00003685B6A9847281C18BF0120E0E707B557
:100BD000FFF7ABFFC043C0F3C01003B05DF804FBE8
:100BE00037B505460C46FFF7A0FF84F001040190DD
:100BF00064F3C7108DF804000199284603B0BDE8DE
:100C00003040FFF7BFBF07B5FFF78FFF80F0080048
:100C1000C0F3C00003B05DF804FB37B505460C46D1
:100C2000FFF783FF84F00104019064F3C3008DF8A3
:100C300004000199284603B0BDE83040FFF7A2BF89
:100C400037B50D460446FFF770FF019065F30200CB
:100C50008DF804000199204603B0BDE83040FFF74D
:100C600091BF37B50D460446FFF75FFF019065F36E
:100C700006108DF804000199204603B0BDE830400D
:100C8000FFF780BF07B5FFF750FF00F0070003B084
:100C90005DF804FB07B5FFF748FFC0F3021003B08F
:100CA0005DF804FB70B51E4D0C468AB00646043450
:100CB0001C4928460EF0F4FA214607A80FF011F857
:100CC00007A928460EF0F0FA2846174D0EF0F8FA5C
:100CD00007A80EF076FF294601A80EF0B7FF01A97C
:100CE00004A80EF0FEFF214604A80FF03AF82946AA
:100CF000044607A80EF0AAFF07A920460FF031F816
:100D0000014630460EF0EDFF07A80EF05AFF04A88A
:100D10000EF057FF01A80EF054FF30460AB070BD28
:100D20006C03002039700100447001007FB50D464E
:100D30000446222128460FF069F82221064628465B
:100D40000FF07EF8002E034604F1040422DB002895
:100D500020DD721C294601A80FF076F801A9204673
:100D60000EF0C9FF01A80EF02CFF0D490D480EF042
:100D700097FA214601A80EF0B4FF01A909480EF028
:100D800093FA08480EF09CFA01A80EF01AFF012011
:100D900004B070BD294620460EF094FFE5E700BF81
:100DA000467001006C0300207FB503680446002BE9
:100DB00039D07721FFF7FCFB206803680021DB694D
:100DC00098470025206802690368954204D21B6891
:100DD000002198470135F5E7DB69144E002198475B
:100DE00000252068715D036801351B689847042D54
:100DF000F7D1206803685B6A98470D4901A80EF097
:100E000025FF01A92046FFF791FF01A80EF0D9FEAA
:100E100007212046FFF714FF07212046FFF721FF97
:100E2000012004B070BD1846FBE700BF347001001C
:100E30001A8901007FB50368044613B9002004B085
:100E400070BDFFF7BBFB0028F8D0E3681F2BF5D877
:100E5000264672212046FFF7ABFB56F8040B0368C9
:100E60006021DB699847314620680EF01DFA206842
:100E7000036800211B6898470546206803685B6A81
:100E800098478DB10A490B480EF00AFA314601A87D
:100E90000EF027FF01A907480EF006FA05480EF0EC
:100EA0000FFA01A80EF08DFE281C18BF0120C6E71E
:100EB0005E7001006C03002030B5036885B0044605
:100EC00013B9002005B030BDFFF778FB0028F8D03B
:100ED000254672212046FFF76BFB55F8040B03688B
:100EE0006021DB6998470022216801A80EF0D6FC3A
:100EF00001A928460EF0FFFE01A80EF062FE206850
:100F000003685B6A98470B490B480EF0C9F92946FC
:100F100001A80EF0E6FE01A907480EF0C5F9064843
:100F20000EF0CEF901A80EF04CFEE068003018BFBC
:100F30000120C7E7517001006C03002007B50023B2
:100F400000931A46194603480EF062F903B05DF8A3
:100F500004FB00BFE002002007B5002300931A46FF
:100F6000194603480EF054F903B05DF804FB00BFC6
:100F7000E802002001207047C08A7047027D1AB144
:100F80000368FF211B68184770470369994228BF0F
:100F90001946816108467047037D10B5044633B990
:100FA000A069236998422CBF0020012010BD03686E
:100FB0001B699847FF28F3D10020F7E7036810B5B5
:100FC00004461B699847A3690133A36110BD7047AC
:100FD00008B502698369934205D2C169034819447F
:100FE0000CF071FA08BD4FF0FF30FBE7F002002073
:100FF00010B5D0E906345A1C82610A460248E1184D
:101000000CF063FA012010BDF002002090F82020BF
:10101000772A02D10368DB6A18477047F0B50D469E
:1010200085B004463F21284617460EF0EFFE031E0A
:101030000BDB0022294601A80EF006FF01A9284675
:101040000EF059FE01A80EF0BCFD114928460EF025
:1010500094FE064660B10023A3614FF4FA43236176
:1010600001208423E361207584F8207005B0F0BD71
:10107000084928460EF081FE0028F7D08423C4E9F1
:1010800006662361267584F820700120EEE700BF14
:101090006A7001007770010001294FF0000303D04E
:1010A00002290CD01846704783614FF4FA4303615C
:1010B0008423C361017580F82020012070478421BA
:1010C000C0E9063301610375F5E7000007B50023A9
:1010D00000931A46194604480EF09AF8034803B0E4
:1010E0005DF804EB0CF0ECB9F1020020F0020020F6
:1010F00038B5002383608380036804460D46002BC7
:1011000047D0274A1268002A43D0002908BF1D464D
:101110002B7C03F00F03062B10D1224A22482946CC
:101120000CF03DFE08B143692371204A1E48294650
:101130000CF035FE00282DD0436963711C4A2168EC
:1011400019480CF02CFE054608BB1A491A480EF047
:10115000A7F80A22617918480EF024F917491648B1
:101160000EF09EF80A22217913480EF01BF912485E
:101170000EF0A6F82B460E4A21680B480CF053FEE1
:101180000B4A216808480CF00AFE054608B11435E0
:10119000A56038BD286810F06EFF6071CEE700BF13
:1011A000340400205888010090070020C47001001A
:1011B0002A7101002D7101006C030020C47A010026
:1011C00010B5044601601146FFF792FF204610BD9E
:1011D00041790C4A002352F82300884203D10A4A7D
:1011E00052F82300704752F8230028B942F8231020
:1011F000054A42F8230070470133052BEBD100204C
:10120000704700BF080300201C03002010B50A4AE5
:101210004079002352F82340844203D1074A42F820
:10122000231010BD52F8234014B952F82320F5E7DB
:101230000133052BEED1F4E7080300201C03002046
:101240002DE9F0412DED028B9AB00546FFF7C0FF66
:1012500004460EF021FE0023014643F69822204664
:1012600008F096FB002800F0DB800623162269793F
:1012700005A80DF01FFC372105A80DF02BFC00225E
:10128000114605A80DF040FD002108EE900A05A8C2
:101290000DF0D2FD654908EE100A65480EF000F821
:1012A0000A22697962480EF07DF8624960480DF0C3
:1012B000F7FF18EE900A10F01DFB022402460B46C1
:1012C00000945B480EF02AF95B4959480DF0E8FF9D
:1012D00018EE100A10F00EFB00940B46024654481C
:1012E0000EF01CF9554952480DF0DAFF50480DF048
:1012F000E7FF534A296853480CF051FD524A2968C8
:10130000804650480CF04BFD0AAC074618EE901A88
:101310000026204602F0A1FECDE900664FF0FF3125
:1013200094E80C00404608F04DFB18EE101A2046D9
:1013300002F093FECDE900664FF0FF3194E80C0017
:10134000384608F03FFB414A29683E480CF027FD2B
:10135000074600285ED0037C03F00F03042B59D10D
:10136000F5EE408AF1EE10FA54D0B5EE408AF1EE77
:1013700010FA4FD0F4EE688AF1EE10FA4AD1B4EECA
:10138000488AF1EE10FA45D13C2231460BA80A9664
:1013900011F0F7F879694022204612F0C6F82F21A3
:1013A000204612F059F828B97B69032240212046D3
:1013B00008F05AFA2649204612F03FF802A818EE23
:1013C000901A08F0DFF923480CF0BEFF40B1224B21
:1013D00093F9003023B902AA21461E480DF0FCF90A
:1013E000204612F074F81AAB1844482300F8413C28
:1013F00018EE101A02A808F0C5F916480CF0A4FF60
:1014000040B1154B93F9003023B902AA2146114887
:101410000DF0E2F90EF040FD01462846FFF7F6FE1A
:101420001AB0BDEC028BBDE8F08100BF267101004F
:101430006C0300203271010042710100497101000A
:101440004B710100900700205071010054710100A0
:1014500058880100E4030020B40300202DE9F04F78
:101460000546006887B00F46904640B1A86830B185
:101470000378FF2903F0100335D11BB9012007B011
:10148000BDE8F08F032AF9D047789C499C480DF0BD
:1014900007FF0A2269799A480DF084FF9949984814
:1014A0000DF0FEFEAB68964859780A2201F00F0154
:1014B0000DF078FF3F09944991480DF0F1FE0A22A2
:1014C00039468F480DF06EFF8D480DF0F9FEAB6880
:1014D0005A7802F00F02BA4207D11A786FF3041259
:1014E0001A700020CBE7002BFBD100220DF1080978
:1014F0001146484602F0A4FDAB685B7803F00F0389
:10150000BB4223D0B8F1030F20D080497C480DF0B6
:10151000C7FE0A2269797A480DF044FF7949784874
:101520000DF0BEFEAB68764859780A2201F00F0133
:101530000DF038FF744972480DF0B2FE0A223946A8
:101540006F480DF02FFF6E480DF0BAFE29680C2F82
:1015500000F2AF80DFE807F0073A94A1A3947394F8
:10156000A5A784A9AB00AB685B7803F00F03023B2F
:10157000082B24D8DFE803F00523239D230F232322
:101580001900634A63480CF00AFCAB681C780646F5
:1015900004F001042DE0604A5E480CF000FCAB68EA
:1015A0001C780646C4F3400423E05C4A59480CF01A
:1015B000F6FBAB681C780646C4F3800419E0584A71
:1015C00054480CF0ECFB0646002412E0554A514802
:1015D0000CF0E5FBAA681378D94303F0010461F32A
:1015E00000031370064620B90122494604A803F0FF
:1015F00004F94D4A296847480CF0D1FB4B4A296849
:10160000824644480CF0CBFB834638B9BAF1000F50
:1016100004D15246494604A803F0EFF8002E4BD1FE
:10162000484602F08BFE002846D1AB685A7867F333
:1016300003025A701A7866F304121A701EE73C4AC5
:1016400034480CF0ACFBA9680B7883F00202C2F3BB
:101650004002C3F34004064662F341030B70C8E73F
:10166000344A2C480CF09BFBA9680B7883F00402E9
:10167000C2F38002C3F38004064662F38203EDE7FF
:10168000274A24480CF08BFB064600289CD10222F6
:10169000494604A803F0B1F896E7274A72E7274ABB
:1016A00070E7274A78E7274A76E7274A7EE7274AFE
:1016B0007CE7002426469CE7AB68B8F1030F5A7814
:1016C0000FD067F303025A701A786FF304121A707E
:1016D000CDE900AB214699E80C00304608F072F9DC
:1016E000CCE602F00F01B9423FF4C8AE67F307122F
:1016F0005A701A7842F010029FE700BFBC700100D8
:101700006C03002068710100C6700100C470010004
:10171000CA70010090070020C9700100D07001005C
:10172000D7700100DC7001001271010054710100DA
:10173000E1700100E7700100ED700100F27001003E
:10174000F8700100FE700100057101000B710100CD
:101750002DE9F0435C4A95B00746884601685B482E
:101760000CF01DFB5A4A3968814658480CF017FBAB
:101770000646B9F1000F01D1002879D0554A3968E1
:1017800052480CF00CFB544A396805464F480CF09F
:1017900006FB5249044652480DF082FD0A2279792F
:1017A0004F480DF0FFFD4F494D480DF079FD0A22DD
:1017B00041464B480DF0DDFD49480DF081FD5EB31B
:1017C000337C03F00F03042B26D14022716904A857
:1017D00011F0ABFE44480CF0B7FDE8B1434B93F970
:1017E0000030CBB92F2104A811F036FE28B9736957
:1017F0000322402104A808F037F8B8F1000F40D0C8
:1018000025B12B7C03F00F03042B34D0384A01237D
:1018100004A935480CF0F5FFB9F1000F28D099F86C
:10182000103003F00F03042B22D1D9F8141004A8B0
:1018300000F0CEFF04A800F009FFB0B1B8F1000F2E
:1018400033D025B12B7C03F00F03042B24D002AC42
:1018500001220021204602F0F3FB0123009394E8CB
:101860000600002304A801F04DFA04A800F014FDBE
:1018700015B0BDE8F0836A691378002BCCD0012342
:10188000C6E724B1237C03F00F03042B02D001230D
:10189000184ABDE76269EFE769690B78002BE4D06D
:1018A000002204A801F0E2FFDFE724B1237C03F06B
:1018B0000F03042B02D002AC0222CAE761690B7845
:1018C000002BD2D04246ECE71271010090070020B5
:1018D00054710100DC700100D77001001F7101001C
:1018E0006C03002047710100E4030020B4030020D2
:1018F0000E8301001983010070B598B0054602AC53
:1019000084E8060039483A490DF0CAFC0A22697990
:1019100036480DF047FD374934480DF0C1FC2046EC
:1019200003F0EAF82968344A34480CF038FA002306
:10193000CDE900334FF0FF3194E80C0008F042F895
:1019400029682F4A2D480CF02AFA29682D4A0646A4
:101950002A480CF024FA054660B3037C03F00F0319
:10196000042B27D14169402208A811F0DEFD2F2168
:1019700008A811F071FD28B96B690322402108A85D
:1019800007F072FF0023102200930DEB02014FF4C9
:101990000073204602F09CFF1B480CF0D5FC48B1B8
:1019A0001A4B93F900302BB9012304AA08A9164851
:1019B0000CF027FFBEB1337C03F00F03042B12D1D0
:1019C000716908A800F004FF08A800F03FFE38B1D4
:1019D0000123009394E80600002308A801F092F97F
:1019E00008A800F059FC18B070BD00BF6C030020BF
:1019F00026710100477101001B7101009007002052
:101A00001271010054710100E4030020B4030020AE
:101A100010B503788B42044604D14378402B01D1A2
:101A2000408810BD40232170637008460EF02EFBE5
:101A300080B26080F5E7000083682DE9F04104463C
:101A40000D46002B00F05A81AD4F3B780133DBB2DD
:101A50000A46FF213B70FFF701FD637926790E3BB3
:101A6000072BC6F3400830D8A64A2168A6480CF0D8
:101A700096F9064648B3037C03F00F03052B24D1E7
:101A80006179A248FFF7C4FF0022804631469E4894
:101A90000CF07DF9436998451FDA0026032D60D0CC
:101AA000A3685A7802F00F02013A0B2A59D8DFE8EE
:101AB00012F01F00ED0042006A00ED007200ED0020
:101AC0009100A200AA00D300E50060790EF00EFCA0
:101AD000A8EB00035E425E41E0E7314601228A48FE
:101AE0000CF055F94669B045CCBF00260126D5E774
:101AF000B3F802800EF0D0F94FF6FF7381B24FF4C5
:101B00007A72404607F044FF58B3814A21687E4804
:101B10000CF045F928B12A4603212046FFF79EFC28
:101B20001FE07C4A216878480CF039F90028F2D18E
:101B30002A460D21F1E7B3F802800EF0ADF94FF619
:101B4000FF734FF4967281B2404607F021FF40B117
:101B50002A4604212046FFF781FC0EF09DF9A36878
:101B60005880A2681378C3F3C001B14200F04681E7
:101B700013F0E00F00F09C80C3F34211013961F3D0
:101B800047131370B6E0B3F802800EF085F94FF6F4
:101B9000FF739622D7E7B3F802800EF07DF94FF677
:101BA000FF7381B24FF47A72404607F0F1FE0028CD
:101BB000D7D0594A216854480CF0F1F810B12A46A0
:101BC0000821AAE7554A21684F480CF0E8F8002898
:101BD000F5D1ADE7B3F802800EF05EF94FF6FF7372
:101BE0004FF4967281B2404607F0D2FE0028B8D07A
:101BF0002A460921AEE7B3F802800EF04DF94FF600
:101C0000FF739622EEE7B3F802800EF045F94FF627
:101C1000FF7381B24FF47A72404607F0B9FE002894
:101C20009FD03F4A216838480CF0B9F810B12A46D5
:101C30000B2172E73B4A216833480CF0B0F80028CA
:101C4000F5D1394A216830480CF0A9F800287FF412
:101C50006FAF2A46062160E7B3F802800EF01CF948
:101C60004FF6FF734FF4967281B2404607F090FE34
:101C700000283FF476AF2A460C216BE7B3F80280C8
:101C80000EF00AF94FF6FF739622EDE7B3F80280E3
:101C90000EF002F94FF6FF7381B24FF41672404610
:101CA00007F076FE00283FF45CAF2A46002134E7B7
:101CB0000EF0F2F8A36858805B7803F00F03002E53
:101CC00051D0072B11D8DFE803F04810041010049E
:101CD000104B164A21680C480CF061F840B32A46B4
:101CE00006212046FFF7BAFB20B1A3681A7866F3F5
:101CF000C3021A703B78013BDBB23B70BDE8F08158
:101D00000403002017710100900700203003002019
:101D1000ED700100F2700100F8700100FE7001002A
:101D2000057101000B710100E7700100E170010015
:101D3000334A216833480CF032F80028CFD1324AB8
:101D4000216830480CF02BF80028C8D12F4A2168B0
:101D50002C480CF024F80028C1D12A460121C0E704
:101D60002A460A21BDE7013B0C2BBED801A252F83E
:101D700023F000BFA91D0000EB1C0000AF1D0000F8
:101D8000AF1D0000EB1C0000B51D0000EB1C0000A7
:101D9000F71D0000F71D0000F71D0000F71D0000F3
:101DA000F71D0000AF1D00002A46022199E72A46D0
:101DB000052196E7164A216812480BF0F0FF10B192
:101DC0002A4607218DE70E4A21680E480BF0E7FFEF
:101DD0000028F5D10C4A21680A480BF0E0FF0028E2
:101DE000EED12168094A07480BF0D9FF01460028C7
:101DF000E6D12A4675E72A46002172E70221BEE6AF
:101E0000F870010090070020FE700100C970010009
:101E1000E17001002DE9F047032986B0804669D0C2
:101E20000168624A62480BF0BAFF98F8051006464E
:101E30006048FFF7EDFD05B2002E69D0337C03F05A
:101E40000F03052B64D1314659480BF098FF032846
:101E500053D90022314656480BF099FF01224469BC
:101E6000534831460BF093FF0222D0F814A050489B
:101E700031460BF08CFF43694D480A270322314657
:101E800007FB03F90BF083FF43695F43214600978B
:101E90004B46524628460DF08AFE044631464448D9
:101EA0000BF06DFF052830D10422314640480BF07D
:101EB0006EFFB0F914A03E48BC42C4BF3C4640F29D
:101EC000FF3531464C45BCBF4C4600250BF057FF53
:101ED000022826D10022314635480BF058FF4369CD
:101EE000AB4251DC0122314631480BF050FF4369CF
:101EF000AB4258DB06B0BDE8F08705EB8504640013
:101F00004FF000094FF42057C8E74FF0010AD2E71D
:101F100005EB850464004FF000094FF420574FF0A3
:101F2000010AD8F80830B3F902002A1A002AB8BF0B
:101F30005242524507DC1A785109052907D8013168
:101F400061F3471202E01A786FF347121A701B7898
:101F50009F2B03D94C4501D0BC42CBD1A842C9D05C
:101F60000022114604AE02A802F06AF8224602A935
:101F7000304602F0CEFB96E806004046FFF7BCFC78
:101F8000D8F808305D80B5E70024D8F80830B3F9F8
:101F90000230A342AED021464046FFF7D9FBD8F825
:101FA00008305C80A6E70124EFE700BF177101004D
:101FB000900700203003002008B583680246F3B183
:101FC000012916D00ADB032908DC0379402B0CD049
:101FD00006D8032B02D81046FFF72EFD002010E094
:101FE000422B02D0FAD3803BF3E71046FFF712FFF3
:101FF000F4E70379042BF1D1FFF722F9EEE74FF074
:10200000FF3008BD7FB5037C03F00F03062B0546A8
:1020100023D10146124A13480BF0C1FE90B1037C54
:1020200003F00F03052B0DD1C4680026ACB129467F
:1020300001A80194FFF75CF8039B1E600DF082FF7E
:102040006468F3E704AC002144F80C5D2046FFF718
:102050004FF802212046FFF7AFFF04B070BD00BF6C
:102060001B7101009007002038B583680446BBB19E
:10207000124B1B68A3B10068FFF7C4FFA3680025DB
:102080001D602379032B0CD8012B94BF0221294614
:1020900060790EF0F1F8A3685A7865F303025A707C
:1020A00038BD402B03D0422BFAD1294600E0022153
:1020B0006079BDE838400EF0DFB800BF340400207E
:1020C000002303807047000013B5002423460094CA
:1020D0002246214603480DF09BF8034B1C8002B0BA
:1020E00010BD00BFFC0200203003002010B50446E4
:1020F00070B3204911F0BDF958B31F49204611F0C3
:10210000B8F940B31D49204611F0B3F928B31C4972
:10211000204611F0AEF910B31A49204611F0A9F982
:10212000F8B11949204611F0A4F9E0B11749204649
:1021300011F09FF9C8B11649204611F09AF9B0B1D3
:102140001449204611F095F9002814BF00200E20F4
:1021500010BD0120FCE70220FAE70520F8E7062081
:10216000F6E70A20F4E70B20F2E70C20F0E70D2059
:10217000EEE700BF7871010093710100B5710100B5
:10218000A7710100BA710100B0710100AB710100CB
:102190006F7101008371010010B50446002843D01F
:1021A0000378002B41D02D4911F063F900283ED06F
:1021B0002B49204611F05DF900283AD029492046E4
:1021C00011F057F9002836D02749204611F051F96F
:1021D00098B32649204611F04CF980B32449204693
:1021E00011F047F968B32349204611F042F950B382
:1021F0002149204611F03DF938B32049204611F01D
:1022000038F920B31E49204611F033F908B31D49AF
:10221000204611F02EF9F0B11B49204611F029F9A2
:10222000002814BF00200C2010BD1846FCE7022037
:10223000FAE70120F8E70820F6E70520F4E7062092
:10224000F2E70720F0E70920EEE70A20ECE70B2091
:10225000EAE70320E8E70420E6E700BF9F710100FA
:102260007B710100BF7101008B710100977101004A
:10227000877101008F7101009B710100C471010021
:10228000A37101007F710100C9710100406910B1A3
:1022900003685B691847704710B50446406910B180
:1022A00003685B689847204610BD000008B503220C
:1022B000016804480BF06BFD08B1007D08BDFF20EC
:1022C000FCE700BF9007002010B503220C46016810
:1022D0000F480BF05CFDD0B1037C13F00D0F16D14D
:1022E000022262F30303037443690A4903F47F4340
:1022F0002343436108480CF0D3FF21460A220648D5
:102300000DF050F80448BDE810400CF0D9BF10BDE6
:1023100090070020527301006C03002010B50322C7
:102320000C46016808480BF032FD58B1037C03F0FD
:102330000F03022B01BF406924F0FF04204000B2CC
:1023400018BF002010BD00BF9007002010B5032269
:102350000C46016808480BF01AFD60B1037C13F0CD
:102360000D0F08D1022262F303030374436904F4DE
:102370007F442343436110BD9007002010B50446FD
:10238000406968B103689B69984718B16069036840
:102390005B69984760690368DB68984708B9012062
:1023A00010BD2046FFF782FF20B14FF48071204618
:1023B000FFF7CCFFA368002BF1D04FF4007120464B
:1023C000FFF7C4FFEBE7000010B503220C460168DD
:1023D00007480BF0DCFC48B1037C13F00D0F05D16E
:1023E0004369E44364F47F441C40446110BD00BF72
:1023F0009007002038B50C464168054609B9002011
:1024000038BD0B7C03F00F03022B03D1002CF6D157
:102410004869F5E7052BF2D105480BF0B0FC844282
:10242000EDDAE2B2696802480BF0B1FC4069E7E717
:102430009007002038B50D464168044621B9DFED0C
:102440001A7A17EE900A38BD0B7C03F00F03052BA8
:1024500015D116480BF093FC854210DAEAB2616898
:1024600012480BF094FC0028E9D0037C03F00F0322
:10247000022B0FD1D0ED057AF8EEE77AE1E7002DD7
:10248000DDD16268137C03F00F03022B07D1D2ED7C
:10249000057AF1E7032BD2D1D0ED057AD1E7032BF2
:1024A000CDD1D2ED057ACCE70000000090070020E6
:1024B00008B5416869B10B7C03F00F03022B06D00D
:1024C000052B06D104480BF05AFC00B208BD0120D0
:1024D000FCE70020FAE700BF9007002008B58168FC
:1024E00009B9002008BD087C00F00F039A1E012ADC
:1024F00000D90BB90009F5E7052BF2D100220348FA
:102500000BF045FC0028ECD0007CF3E7900700209E
:10251000826810B5BAB1137C03F00F039C1E012C26
:1025200000D983B9516183681A7C022161F30302E7
:102530001A748268137C03F0F001602902BF0A213B
:1025400061F30713137410BD826810B5BAB1137C20
:1025500003F00F039C1E012C00D983B951618368DD
:102560001A7C032161F303021A748268137C03F05E
:10257000F001602902BF072161F30713137410BD36
:10258000836853B11A7C02F00F02901E012800D913
:102590001AB91A7C61F307121A74704708B5C1683A
:1025A00009B9002008BD0B7C03F00F03022B01D1F9
:1025B0004869F7E7052BF4D1002203480BF0E7FB4D
:1025C0000028EED04069EDE7900700202DE9F041AA
:1025D000C36804460E46A3B901681948184F0BF0AA
:1025E000CEFB0546042D0CDC3846D4F800800BF0F9
:1025F00005FC41460246E06038460BF0DDFB013544
:10260000F0E7E268CAB1137C13F00F0113D1022185
:1026100061F303031374E3680A495E610A480CF02E
:102620003FFE31460A2208480CF081FE0648BDE80C
:10263000F0410CF045BE0229EDD0BDE8F08100BFAD
:10264000900700205A7301006C030020006828B135
:10265000007C00F00F00431F5842584170470000B3
:10266000F8B50446FFF7F2FF002831D0216837485B
:10267000364F0BF084FB0546032D266809DC3846EF
:102680000BF0BCFB3146024638460BF095FB01359A
:10269000F2E7002231462D480BF079FB43692374A1
:1026A0000122216829480BF072FB02226060216838
:1026B00026480BF06CFB0422A060216823480BF035
:1026C00066FBE060207C0C282CD002D803280ED0BA
:1026D000F8BD102830D01228FAD10C200DF072FC71
:1026E0001B4B44600360054606F08EF818E010208E
:1026F0000DF068FC174B036005464460002120463E
:10270000FFF778FE03B2002BB6BF40422B81288131
:102710006868FFF7CDFE104B2B6000236881AB810A
:102720006561D5E714200DF04DFC0C4B446003604F
:10273000054605F007FDF3E70DF044FC084B446047
:102740000360054606F040FAEAE700BF9007002064
:10275000A4830100F46F0100F8830100C48201002A
:102760009884010010B5002304460160436103769C
:102770008362FFF775FF204610BD000070B5056845
:1027800006462F21284610F0F1FE044698B100239A
:1027900000F8013BFFF700FD0B4905460B480CF024
:1027A0007FFD0A22294609480CF0E3FD07480CF09A
:1027B00087FD284670BD2846FFF7EEFC0546002839
:1027C000F7D03460F5E700BF597101006C030020B9
:1027D0002DE9F04389B0002400F118080546CDF832
:1027E00004804461047684620E4600293BD01F4B6E
:1027F0001F68002F37D02F21304610F02DFE814664
:1028000050B3234602AAF05C19B238B12F2805D084
:10281000142B02D0D0540133F5E7194608AB194404
:10282000002301F8183C124839460BF0B8FA0F2281
:10283000286009F10101404610F077FE01A8FFF77A
:102840009DFF019BA86203B92B762846FFF708FF7E
:10285000284609B0BDE8F0833246394604480BF0FB
:102860009EFA2860F1E700232B60EEE7D8030020F2
:102870009007002008B543693BB9007C052809D0C2
:1028800014280CBF0020FF2008BD1A681846526BA0
:102890009047F3E75020F7E718B1034903480CF0DD
:1028A000FFBC0349FAE700BF657101006C0300201B
:1028B0006A7101002DE9F0439FB04FF0000802ACAF
:1028C00084E806000646102241460AA81D46269FB7
:1028D000CDF824800FF055FE2046CDE906888DF80E
:1028E000208002F009F9EB051BD5204601F0D6FE49
:1028F000172800F2CE80012303FA00F047F6424386
:1029000018420AD18B4B0340002B40F0C68010F0D8
:10291000240F00F0BE80884900E0884906A810F026
:10292000B2FD87480BF010FD002800F0AA80854B0F
:1029300093F900209846002A40F0A380002F44D14C
:102940003B46032240210EA806F08EFF33683F224B
:1029500019680EA810F0C3FDA80540F1AD8020460F
:1029600001F09CFE022800F0A780204601F096FEB0
:10297000052800F0A180204601F092FE012840F0D9
:102980008F804FF001094FF40073142209A9CDF88C
:102990000090204601F09CFF4B4609AA0EA968480A
:1029A0000BF02FFF684969480CF07AFC0EA96748C4
:1029B0000CF07FFC664965480CF072FC09A963487D
:1029C0000CF077FC61480CF07BFC204601F0C7FC62
:1029D00005F4805908B1AA0503D4B9F1000F00F03D
:1029E00098800023032240210EA806F03DFF3368A3
:1029F0003F2219680EA810F072FD47B155490EA884
:102A000010F01BFD3F2239460EA810F068FD514919
:102A10000EA810F012FDB9F1000F63D04E490EA8B8
:102A200010F00BFD204601F03BFE043801285BD876
:102A30001722214604A801F0E0FE002300934FF482
:102A40004073142209A9204601F042FF3E493F4845
:102A50000CF026FC0EA93D480CF02BFC3C493B48F1
:102A60000CF01EFC09A939480CF023FC37480CF087
:102A700027FC33480BF068FC18B198F90030002BA4
:102A80003CD0304629B2FFF761FC00201FB0BDE802
:102A9000F08332492D480CF003FC25F4807540E7A3
:102AA000204601F0FDFD02283FF46BAF204601F007
:102AB000F7FD08283FF465AFE90586D5012306AA8E
:102AC0000EA91F480BF09DFE1F4920480CF0E8FBA3
:102AD0000EA91E480CF0EDFB1D491C480CF0E0FB54
:102AE00006A96CE71E499AE70023B9F1000F00938D
:102AF00014BF4FF440734FF40073A2E70EA90123F3
:102B000009AA0F480BF07DFE4FF400713046FFF725
:102B10005BFCEB0571D5204601F0C0FD01380D28A6
:102B200024D8DFE800F07223232323722323231FFA
:102B30006C75706E01008000937101007871010066
:102B4000E4030020B4030020057201006C030020A0
:102B5000C6700100C47A01007F710100F7710100A5
:102B60009F7101002B4906A810F08DFC0023032261
:102B700040210EA806F078FE33683F2219680EA89F
:102B800010F0ADFC47B124490EA810F056FC3F22CE
:102B900039460EA810F0A3FC1F490EA810F04DFCFA
:102BA0001E490EA810F049FC1D491E480CF078FB88
:102BB0000EA91C480CF07DFB1B491A480CF070FB59
:102BC00006A918480CF075FB16480CF079FB17485D
:102BD0000BF0BAFB00283FF454AF98F90030002BFB
:102BE0007FF44FAF0EA9012306AA10480BF009FE8F
:102BF0004FF480713046FFF7E7FB012046E70C49B0
:102C0000B1E70C49AFE70C49ADE7337C052BADD1FB
:102C10000A49A8E7BA710100C47A01007B7101007A
:102C2000057201006C030020C6700100E40300205F
:102C3000B0710100837101006F710100AB7101007F
:102C4000F0B5CB070C4644BF21F4006424F0010426
:102C500014F4006785B005460CD004F44071284692
:102C6000FFF774FB144915480CF01AFB4FF0FF30C6
:102C700005B0F0BD06F07FFD9528EED902F04EFDBF
:102C80000028EAD002AE3A463946304601F0D8F97B
:102C90004FF440722946304601F0C4FD4FF44071B4
:102CA0002846FFF73BFB009740EA040396E806003E
:102CB0002846FFF7FFFDDBE7CD7101006C03002024
:102CC00010B54FF440710446FFF728FB014670B180
:102CD000074B93F90030062B09D12046FFF7B0FFD0
:102CE00020464FF44071BDE81040FFF76DBB10BDAA
:102CF000DC03002043691BB11A681846526B104769
:102D0000007C70472DE9F04F8FB008AD07939DF818
:102D10006030069385E8060006460DF0BDF8059084
:102D2000284601F071FD8146044602F0F7FC079B3E
:102D300004901BB11A78002A40F02C85337E13B121
:102D400006F118030793002C40F03D85079B002BEC
:102D500040F02385D6F82890B9F1000F00F03385B4
:102D6000284601F051FD002840F02D855FFA89F2D8
:102D700029460CA801F04CFD00F025BD284601F0C5
:102D8000BBFE079B63B11B78242B09D1BF49C04808
:102D90000CF086FABE480CF093FA6FF0030B22E0B9
:102DA0003168002900F03B85B9F1040F65D1B948BD
:102DB000DFF8E0820AF0E3FF0446052C376809DCFF
:102DC00040460BF01BF83946024640460AF0F4FF35
:102DD0000134F2E705223946AE480AF0D8FF04462E
:102DE00028B94FF0000B58460FB0BDE8F08F2846C9
:102DF00001F054FC0F28F4D8284601F0EBFA002823
:102E000003DD237C13F00D0F0DD0237CA249A048D5
:102E10006FF3071323740CF043FA9D480CF050FA3B
:102E20004FF0010BDFE70DF037F80646284601F0BA
:102E3000D1FA237C022262F30303304460612374DD
:102E4000284601F02BFC237C944960F3071323747C
:102E50008F480CF025FA284601F0BCFA0A220146F8
:102E60008B480CF064FA8E4989480CF019FA0A2252
:102E7000616987480CF05BFACFE7284601F00EFC49
:102E8000092800F2A781DFE810F00A00A501A501DA
:102E9000A5012A01A501A501A501470147010022BD
:102EA0000DF1280A1146504601F0CAF8284601F0F3
:102EB00056FA0746002800F01081B9F10B0F00F216
:102EC0008981DFE819F00C0087015A00870187012A
:102ED0008701870187018701C500B100F3003046F3
:102EE00000F082FE0028D4BF002101210A220446FE
:102EF00067480CF03EFA6B4965480CF0DAF9284651
:102F000001F068FA0A22014661480CF010FA6048A4
:102F10000CF0D6F9002C284640F3348401F05AFA1C
:102F200080BB022229460CA801F067FC40F2011484
:102F30004FF0010808E0012229460CA801F05DFCD1
:102F400040F201144FF000084FF400723146504631
:102F500002F062F9504601F0A3FB042814D1284680
:102F600001F09EFB022814D1284601F099FB0AA922
:102F700002460CA801F097FB0BE0002427464FF017
:102F8000FF38E1E70024D3E7504601F089FB05282C
:102F9000E5D0337C072B08D1284601F0E7F920B1B2
:102FA00002220AA90CA801F07EFB3046FFF7A2FE20
:102FB00000B200900DF1280B0DF1200A0CA89AE840
:102FC0000C00594601F012FE584601F095FD3FB144
:102FD000504601F065FB022816D1584602F048F928
:102FE0009BE8030044F420648AE803004FF0000AE1
:102FF000337C072B40F0A081039BB3F5AF7F80F2B9
:10300000EC80294900F005BC504601F049FB01283D
:10301000E3D0504601F044FB0A28DED0504601F0D0
:103020003FFB0B28DCD1D8E731464FF40072504605
:1030300002F0F2F8284601F0EBF8C1B2504601F078
:103040008FF898B9BA4600273C464FF0FF38CFE7D3
:1030500031464FF40072504602F0DEF8284601F087
:10306000D0F80146504601F061F8EAE79AE803001B
:10307000022285E8030029460CA801F0C9FB4FF4A1
:10308000206400274FF0000ADFE700BF2B72010029
:103090006C030020900700203F720100497201007C
:1030A00054720100687101005A7201004FF40072FD
:1030B0003146504602F0B0F8284601F088F8014643
:1030C000504601F05EF89AE8030085E803004FF0EF
:1030D000000A4FF420645746B7E78246B4E730460B
:1030E00000F082FD00280BDD022229460CA80127F2
:1030F00001F083FB40F201144FF0000AB84677E775
:10310000012229460CA84FF0000A01F076FB40F29C
:1031100001140127D0466BE795E803000DF128085C
:1031200088E80300284601F01AF9E0B9052428468A
:1031300001F0B4FA4FF4007209283146284608BF5E
:10314000644202F069F8002229460CA801F055FB00
:10315000B9F10A0F3ED8DFE809F01F3D0D3D3D3DB6
:103160003D3D3D213500284601F00CF9044600287C
:10317000DCD0DCE700273046FFF77CFB2146024627
:10318000284601F047F8044608BB98E803004FF0D2
:10319000010A85E8030058E70127ECE721462846A5
:1031A00001F094F828B1022229460CA801F030FB66
:1031B0008DE798E8030085E8030000244FF0010A3A
:1031C000274642E72146284601F0A5F8EAE74FF4F2
:1031D000206457E70024A246F2E7069B5BB17068C3
:1031E000037C03F00F03052B05D1049B1BB1079A49
:1031F00008A900F081FC08A801F050FA033804285F
:1032000028D8DFE800F003277A4C2A003046FFF781
:103210004DF80528804602D04FF0030BE3E5B34993
:10322000B3480CF03DF80A224146B1480CF0A1F831
:10323000AF480CF045F84FF400723146284601F0D3
:10324000EBFF012229460CA801F0D7FA44F4807460
:1032500044F001044FF0000837E03046FFF726F84D
:10326000062880460ED1A349A1480CF019F80A227D
:1032700041469F480CF07DF89D480CF021F8022251
:1032800008A9E0E79C499A480CF00AF80A2241464E
:1032900097480CF06EF896480CF012F8BCE73046F0
:1032A00000F0A2FC002823DC4FF4007231462846CF
:1032B00001F0B2FF012229460CA801F09EFA44F465
:1032C000807444F001044FF0060808A801F03BF8B0
:1032D00030BB08A844F0010401F041F818B344F4ED
:1032E00000744FF0010BBAF1000F7FF456AD63E1AB
:1032F00082497F480BF0D4FF8EE7304600F074FC23
:1033000000280BDD022208A90CA844F4807401F007
:1033100074FA44F001044FF00508D6E77849E8E76D
:1033200044F48074D5E74FF40072314608A801F0E8
:1033300079FA0028D3D1D4E7B8F1FF3F08D130465D
:1033400000F052FC0028D4BF4FF000084FF00108F5
:10335000B8F1000F6B49664818BF01270BF0A0FFBA
:103360000A22414662480CF004F8674960480BF0B5
:1033700097FF0A2239465E480BF0FBFF5C480BF0D2
:103380009FFF079808B3FEF7B1FE03903046FEF7A3
:103390008DFF0FFA80FB039BBBF1000F01D10FFAE9
:1033A00088FB4BB39B450ED0584951480BF078FF32
:1033B00059460A224E480BF0DCFF4D480BF080FFC7
:1033C0006FF0020B0FE50023079308A801F066F9E0
:1033D0000E2800F2D980DFE810F0E600B0009B0074
:1033E0001C00E600790063004800E600E600C50026
:1033F000C500C500C500C500706900283FF4F1ACE8
:103400000368009708AA9C6A079B06CAA0478346E0
:10341000E9E43046FEF74AFF052807467FF4FCAE94
:10342000324933480BF03CFF0A22394630480BF052
:10343000A0FF2F480BF044FF4FF40072314608A85C
:1034400001F0EAFE337C052B0CBF0C22012208A9F7
:103450000CA801F0D2F944F4807444F001044FF058
:1034600000084FF0FF3B01273DE73046FEF71EFF07
:10347000062807460DD11F491D480BF011FF0A22EF
:1034800039461B480BF075FF19480BF019FF022253
:10349000DDE7194916480BF003FF0A223946F7E623
:1034A000B8F1000F7FF424AF4FF400723146284684
:1034B00001F0B2FE44F48074012229460CA801F008
:1034C0009CF944F001044FF00608CAE7B8F1000F78
:1034D0003FF424AF022208A90CA844F4807401F040
:1034E0008CF944F001044FF00508BAE7807201003E
:1034F0006C0300208F720100A0720100B8720100FD
:10350000CC720100E3720100EB720100F272010063
:1035100008A800F018FF0746002843D03046FEF701
:10352000C5FE05283FF478AE44F4807444F00104ED
:103530004FF000084FF0FF3BD5E608A800F003FF6E
:1035400080B3B8F1000F0DD0B749B8480BF0A8FE12
:1035500030460121FEF7B8FE4FF410613046FFF708
:103560006FFB59E608A800F0EEFE0746D0B108A8A8
:1035700000F0F5FE28B94FF40072314608A801F0BA
:103580004BFE44F44074D1E708A800F0D7FE08B120
:1035900044F4807408A800F0E2FE074610B144F439
:1035A0000074C5E70127BAF1000F7FF4F6AB002CD9
:1035B00045D0D0464FF0FF3B2246314608A801F0E7
:1035C000EFFDD6F814A0BAF1000F3CD0DAF80030C5
:1035D00000979F6A079B95E806005046B8478346C8
:1035E000706903685B6B9847052801D144F00104BA
:1035F000B8F1000F03D041463046FEF765FE049B4C
:103600001BB121463046FFF71BFB894987480BF069
:1036100047FE0A22594685480BF0ABFE8549834890
:103620000BF03EFE0CF038FC059B0A22C11A7F48C5
:103630000BF0ABFE7D480BF043FEFFF7D4BBA0467A
:103640004FF0FF3BBDE7337C052B4BD0062BCFD192
:1036500051463046FEF7CEFE05B2074608A801F0F7
:103660001DF8002DC4D0BCBF7D422DB205F1FF3343
:103670009BB2B8BF4FF0010A192BB9D807B201218C
:1036800028460CF0F9FDBAF1000F24D0012F20D00C
:103690000C3F18BF0127394628460CF015FE664935
:1036A00062480BF0FDFD0A22294660480BF061FEDE
:1036B00062495E480BF0F4FD0A2239465B480BF084
:1036C00058FE5A480BF0FCFD44F4807444F00104A9
:1036D00052E00027DFE7012FDDD0A7F10C035F42A6
:1036E0005F41D8E7B9F1020F49D0B9F1030F09D012
:1036F000B9F1010F7FF47CAF44F4807444F001040D
:10370000CB4675E73046FEF749FF030C074605D167
:1037100033684B491A684B480BF05EF8284600F0B6
:1037200079FE0EF0E7F8484B00220EF03BF90EF060
:10373000E9FB0FFA80F9082006F0A8FA69F30F07F1
:10374000054660F31F47414938480BF0A9FD0A229E
:10375000494636480BF00DFE3D4934480BF0A0FDBC
:10376000A9B20A2231480BF004FE30480BF0A8FD44
:1037700039463046FEF72AFF4FF0010B38E744F494
:103780000074A3E700F026FE00287FF4D4AB0446C3
:10379000FFF7D8BBB9F1000F15D11B78002B3FF410
:1037A000D9AA07A8FEF7EAFF8146284601F02CF8BF
:1037B00028B95FFA89F229460CA801F029F8B9F175
:1037C000000F3FF4C7AA05F0D6FF2249039017481F
:1037D0000BF066FD0A22039914480BF0CAFD1E493E
:1037E00012480BF05DFD3368104819680BF061FD5D
:1037F0001A490E480BF054FD07990C480BF059FD7F
:1038000017490A480BF04CFD039BC72B3FF7B6AA9C
:10381000144915480BF044FD13480BF051FD4FF0CF
:10382000FF3BFFF7E0BA00BFB97201006C03002054
:10383000257301002F730100087301004771010017
:103840000D730100E4030020000059401C730100C7
:10385000207301000B720100107201001772010049
:10386000687101001D720100880300202DE9F047F6
:103870008EB08046CDE90221002900F036810AB1E0
:1038800013782BB998F8183013B108F11803029384
:10389000029B63B9D8F8286096B90024039D2F5D78
:1038A0000FB3384610F035FE28550134F6E71B7883
:1038B000002BEFD002A8FEF761FF06460028E9D0F2
:1038C0000C2EEAD108AC00221146204600F0B8FBCD
:1038D000039A21460AA800F084FF324621460AA82E
:1038E00000F096FF69E0284600F078FB04ACC2B215
:1038F00005463946204600F0A3FB052E20D0062EB3
:1039000008BF17255FFA86F90AAF4A4621463846AE
:1039100000F07EFF092D15DC082D80F2D880AA1C4E
:1039200003DB6B1C40F3E180B5B103A805F07AFE20
:103930000246002841D02146384600F0D2FE3CE045
:103940001825DFE7172D00F09180182DEDD100220A
:103950002146384600F051FF06AD03A9284605F080
:1039600082FE4A462946384600F052FF284600F0BB
:1039700097FE10F1000918BF4FF001094FF0000A3F
:10398000039A0FFA8AF35AB1BAF1030F07D003A8CA
:1039900005F048FE47F82A000AF1010AF0E753460D
:1039A0000A2E15D00B2E1BD0092E21D1284600F04F
:1039B00011FD81B2204600F0B9FB0123009394E889
:1039C0000600029B4046FFF79DF90EB0BDE8F08768
:1039D000284600F0FFFCC1B2204600F0C1FBECE736
:1039E000284600F0F7FC0146204600F0CAFBE4E759
:1039F0004B449BB2013B032B30D8DFE803F00207B6
:103A0000122095E8030084E80300D6E7284600F07A
:103A1000E1FC9DF8283082B2214608A800F0AAFEF9
:103A2000CBE7284600F0D6FC9DF82C2000929DF8AC
:103A3000283082B2214608A800F085FEBDE728465E
:103A400000F0C8FC9DF82C200092214682B29DF81F
:103A5000283008A800F077FE0C99C5E724492548CE
:103A60000BF01EFC23480BF02BFCA6E7002221469E
:103A7000384600F0C2FE0025039A2BB242B1042D55
:103A80000AD003A805F0CEFD47F825000135F3E77D
:103A9000032B10D0042B90D19DF8341001919DF888
:103AA000301000919DF82C309DF82820214608A860
:103AB00000F084FE81E79DF8301000919DF82C30D5
:103AC0009DF82820214608A800F068FE75E708AC9C
:103AD00003A9204605F0C7FDEAB22146384600F0AA
:103AE0008CFE4A4621463846FAE600206DE700BFC4
:103AF00036730100880300202DE9F0470E468EB092
:103B00009146002853D0037C03F00F03052B62D1AC
:103B1000324DC4682B78DFF8C8A0DFF8C8800133C5
:103B20002B70002C54D0237C03F00F03042B4DD1B9
:103B30006269DAF8001040460AF031F907460028B9
:103B400044D0037C03F00F03052B3FD1014603A8AB
:103B5000FEF708FE5EB103A8FEF778FD38B100233A
:103B60000093316872684B4603A8FFF7CBF8002238
:103B7000394640460AF00BF9E0B1037C03F00F032D
:103B8000022B17D14369072B14D101223946404635
:103B90000AF0FDF84A463146FFF7AEFF9EB990B1F4
:103BA0002B7803A8013B2B70FEF776FB01200EB0AB
:103BB000BDE8F0873EB903A8FEF748FD18B103A899
:103BC00000F012F8EBE703A8FEF766FB6468A8E7CD
:103BD0002B78013B2B700020E9E700BF6903002030
:103BE000D80300209007002073B500220546114637
:103BF000684600F025FA2B68464819680BF059FB17
:103C0000454944480BF04CFB2846FEF71FFD58B9C8
:103C1000424940480BF044FB3E480BF051FB4FF04B
:103C2000FF34204602B070BD2846FEF73FFB064633
:103C3000686958B10368DB6A984704B2002C05DB59
:103C400014BF01200020FEF727FEEAE72B7C072B9C
:103C500014D0701C0D2811D8012606FA00F043F686
:103C60008404044004D110F0490F07D02046EAE74D
:103C70002B4928480BF014FB3446D2E74FF400726E
:103C80002946684600F0CEFD2B7C033B062B39D835
:103C9000DFE803F0341F383804341F006B681B7CE6
:103CA00003F00F03052B33D11E491A480BF0F8FA25
:103CB000002211466868FFF71FFF1B49044615489C
:103CC0000BF0EEFA2046FEF7E7FD12480BF0F8FA8B
:103CD000A7E70021684600F075FC044613490D482B
:103CE0000BF0DEFA21460A220A480BF042FB094893
:103CF0000BF0E6FA003418BF012492E7684600F0A2
:103D000069FBEAE70A4903480BF0CAFA002488E78E
:103D10000024E3E76C030020687101006673010072
:103D2000657101004A7601006F7301007C73010028
:103D3000727301002DE9FF412C4BB3F90060054679
:103D4000002E4DD14FF48061FEF7E8FA00284AD0EA
:103D500002AC32463146204600F072F94FF4407210
:103D60002946204600F05EFD214922480BF098FAD2
:103D700028464FF48061FEF727FB6869002832D09F
:103D8000036801270097D3F8288094E8060033469B
:103D9000C047431C044626D02B681648196884B9CE
:103DA0000BF087FA144913480BF07AFA13491148BB
:103DB0000BF076FA0F480BF083FA204604B0BDE80A
:103DC000F0810BF076FA0C490A480BF069FA0C49BD
:103DD00008480BF065FA07480BF072FA3C46ECE72E
:103DE0004FF0FF34E9E70224E7E700BF3E0300207D
:103DF000DE7101006C03002058720100017C01009B
:103E0000F37101002DE9F041244BB3F900308CB07F
:103E1000002B3FD1224E234F3278013232703A6864
:103E2000002A35D0D568DFF8888001243A680AB3C3
:103E300005B32B7C03F00F03052BF8D12946404630
:103E400009F09DFF0128F1D9294601A8FEF78AFC57
:103E500001A8FEF7FBFB30B101A8FFF76BFF00B232
:103E60000028D8BF00240CF06DF801A86D68FEF79B
:103E700013FADBE70C480BF023FA3378013B33707D
:103E800054B10A4B00221A7020460CB0BDE8F081F4
:103E90000124F2E70024F7E70124F5E73E030020C0
:103EA00069030020D80300206C0300203C0300209D
:103EB000900700202DE9F0473C4B1B7886B0044664
:103EC0008A460BB1FFF79EFF05222168384809F0AA
:103ED0005EFF0746002851D090F8108046694FEAEF
:103EE00018180BF0D9FFB8F1000F47D002AD361A01
:103EF00042460B2128460DF1100900F0A1F8324688
:103F00002946484600F0EDFBBAF1040F17D1002313
:103F1000009395E806004FF480532046FEF7CAFC54
:103F20000A224FF47A71234896FBF1F10BF0FFF966
:103F3000214920480BF0B4F91E480BF0C1F9002EBE
:103F40001CDA1E4B9E4219DB002600964FF480536C
:103F500095E806002046FEF7ADFC4246314648464D
:103F600000F06EF80123009399E8060033462046DE
:103F7000FEF7C8FE3B7C66F307133B74BAF1010FF2
:103F800002D12046FEF79CFE606918B9002006B0F9
:103F9000BDE8F08703689B6998470028F6D0606900
:103FA00003680FFA8AF19B689847F0E73C0300200A
:103FB000900700206C030020437301000200008082
:103FC00007B5002300931A46194603480BF020F961
:103FD00003B05DF804FB00BF34030020F8B50646CB
:103FE000F0B10378E3B12D2B1ED0A3F13002092AE2
:103FF0001AD9252B1AD07B2B1AD0232B1BD00F4F6D
:10400000012404EBC4053D4428460FF060FA29461C
:10401000024630460FF077FA20B10134192CF0D166
:104020004FF0FF342046F8BD0024FBE70824F9E7F1
:104030006FF00104F6E71724F4E700BF997301005D
:1040400010B500238370C370037143718371C37112
:1040500061F307134370027010BD10B500230724ED
:1040600003708370C37064F307134370416010BD25
:1040700093B2112B70B516469CBF134AD25C4B7895
:1040800088BF002262F307134B7005460C460F48A9
:104090000F490BF005F90A2231460C480BF069F97B
:1040A0000C490A480BF0FCF8617808480A22090913
:1040B0000BF078F905480BF003F923682B6063686F
:1040C0006B60284670BD00BF877301006C03002041
:1040D000F0740100FB7401004B781B09013B082BB5
:1040E0001AD8DFE803F0160E0E19191919050C007D
:1040F0000C4B4B600B6803604B68436070470A4B86
:10410000F7E764238B71CB7923F00103CB71002394
:104110004B71FF230B71EDE700230B714B718B711A
:10412000CB71E7E70000A0410000964243781A09EE
:1041300003D0022A05D000207047022262F3071341
:10414000437040F26D139942A8BF1946C37981713B
:1041500023F00103C1F300211943C171012070470D
:1041600043781A0903D0022A05D0002070470222A2
:1041700062F3071343706429A8BF642141710120D1
:10418000704713B50446084631B9E37960F3470335
:10419000E371012002B010BD642300934FF4FA7262
:1041A000002399210BF003FD63781A0908D0032A34
:1041B0000BD820EAE0706428A8BF64200130E4E74F
:1041C000022262F307136370F3E70020E2E707B50A
:1041D000C27912F0FE0F11D043781B09013B022B6C
:1041E0000CD850084FF4FA730093642299230021ED
:1041F00001380BF0DCFC03B05DF804FB4FF0FF303E
:10420000F9E7C379827903F0010342EA032070479A
:104210004079704743781B09013B10B50A2B53D8EE
:10422000DFE803F00606525252482F2F2F101000DD
:104230000279642391FBF3F1114481F308010171C8
:10424000012010BD632944684FF064030FDC03FBB9
:1042500004112AB153439942A8BF194621EAE171DA
:1042600043784160062262F307134370E8E791FB4D
:10427000F3F12144E2B19142A8BF114621EAE17174
:1042800016E0436807EE903AFDEEE77A642417EEF5
:10429000903A91FBF4F1194422B19142A8BF114622
:1042A00021EAE17107EE901AF8EEE77A17EE901A1C
:1042B0004160C5E743681944002AF9D06423534399
:1042C0009942A8BF1946D9E70020BAE743781B09ED
:1042D000022B1ED1C279837902F0010243EA022344
:1042E000642291FBF2F11944B1F5B77F0FDA40F285
:1042F0006D1331EA210128BF1946C379817123F07A
:104300000103C1F300211943C1710120704700214D
:10431000F3E70020704743781B09022B0CD1437947
:10432000642291FBF2F1194421EAE1719142A8BFA4
:10433000114641710120704700207047007800301D
:1043400018BF01207047437803F00F03012B04D8F6
:104350000078003018BF0120704700207047437874
:1043600013F0F00F14BF012000207047407800F0D8
:10437000E000202804D0A0F1400358425841704783
:104380000120704743781B09013B0A2B1ED8DFE848
:1043900003F00A0A1D06061B0F0F0F0606004368EE
:1043A0006420584370470079642310FB03F0704782
:1043B00043689FED077A07EE903A67EE877AFDEE45
:1043C000E77A17EE900A7047406870470020704700
:1043D0000000C84243781B09013B0A2B18D8DFE8CC
:1043E00003F00808170606120A0A0A0606004068C3
:1043F000704700797047406807EE900AFDEEE77A53
:1044000017EE900A70474068642390FBF3F0704702
:104410000020704743781B09013B0A2B1ED8DFE8B8
:1044200003F013131D06060E19191906060043683A
:1044300007EE903AF8EEE77A17EE900A7047436875
:10444000642293FBF2F3F3E7037907EE903AF8EE78
:10445000677AF1E7436807EE903AEDE7DFED017A1E
:10446000EAE700BF0000000043781B0907B50B2BEB
:1044700060D8DFE803F06216165F5F5F44245F5F79
:104480000606406849B1D0F1640056D46428A8BF3C
:10449000642000B203B05DF804FB0028F6DA084699
:1044A000F8E7007931B1002100916423FF220BF07D
:1044B0007EFBEEE764230093FF220B46F7E7436899
:1044C00007EE903A99B19FED1F7A77EE677AF5EE95
:1044D000C07AF1EE10FA30D4F4EEC77AF1EE10FAA9
:1044E0002DDCFDEEE77A17EE903A18B2D2E7F5EE42
:1044F000C07AF1EE10FAD2D49FED127AECE743685D
:1045000061B142F27372934217DC13F1630F16DB51
:104510006FF0630093FBF0F06430BAE713F1630FC0
:10452000BDDB42F2737293424FF06400B2DC93FB46
:10453000F0F0AEE74FF0FF30ACE70020AAE76420D0
:10454000A8E700BF0000C84213B5044608466378D8
:104550001B09013B0A2B32D8DFE803F00F0F313182
:1045600031281A3131060600FF230093002364220C
:1045700019460BF01CFB606007E0FF23009300234B
:10458000642219460BF013FB2071012002B010BD0C
:10459000FF2300930023642219460BF008FB07EE6B
:1045A000900AF8EEE77A17EE900AE4E746F29C33B9
:1045B00000930023642219460BF0F9FA6060002092
:1045C000E4E7000043781B090B2B5FD8DFE803F01A
:1045D0006117175E5E5E461E5E5E0606406841B16C
:1045E000002839DBFF28A8BFFF20C0F1FF0001B27F
:1045F0000AE0002808DBFF28A8BFFF20F7E70079C2
:104600000029F4D0C0F1FF01084670474368A9B102
:1046100007EE103AB5EEC07AF1EE10FA1CD4DFEDD9
:104620001E7AB4EEE77AF1EE10FA32DC77EEC77A52
:10463000FDEEE77A17EE903A19B2E5E707EE903A09
:10464000F5EEC07AF1EE10FADED49FED137AF4EEB7
:10465000C77AF1EE10FAEBDDFF21D5E7406859B1DA
:1046600010F1630FF8DBB0F5C84F12DA6FF0630199
:1046700090FBF1F0FF30BAE710F1630FC4DBB0F547
:10468000C84FE9DA642190FBF1F0B0E74FF0FF3159
:10469000BAE70021B8E700BF00007F430078704709
:1046A0004078000970474B7810B562F307134B70E0
:1046B0000B6803604B68436010BD4B7810B51C0954
:1046C000013C012C84BF012464F3071382F3080228
:1046D000D2B288BF4B700B680A7103604B684360AD
:1046E00010BD4B784A6030B50A2565F307134B704F
:1046F0000B6803604B68436030BD4B784A6030B54F
:10470000072565F307134B700B6803604B68436024
:1047100030BD4B7830B5062565F307134B700A237F
:104720005A434A600B6803604B68436030BD4B7866
:104730004A6030B5062565F307134B700B680360BC
:104740004B68436030BD70B54C788A71022666F3C1
:1047500007144C70C2F30024CA794B7122F0010295
:104760009DF810300B7122430B68CA7103604B68CF
:10477000436070BD70B54C788A71032666F30714E8
:104780004C70C2F30024CA794B7122F0010222431B
:104790000B68CA7103604B68436070BD70B54D789B
:1047A0004B71042666F307159DF810304D700B71A0
:1047B0008A710B6803604B68436070BD70B54D78BB
:1047C0004B7105269DF810300B7166F307159DF8A7
:1047D00014304D70CB718A710B6803604B68436075
:1047E00070BD4B784A6030B50C2565F307134B70EC
:1047F0000B6803604B68436030BD10B50A700B68EE
:1048000003604B68436010BD407800F00F007047B4
:104810004B7810B562F303034B700B6803604B6871
:10482000436010BD2DE9F041044616460D4619B906
:1048300000273846BDE8F0810846FDF707FF074628
:104840000028F5D02846FDF749FEF305804603D53C
:104850002846FDF72BFD207006F40076B8F1000F16
:1048600009D0637868F307136370002EE1D0AB685A
:104870005B696360DDE7002EDAD0AA68137C03F081
:104880000F03022B03D0032B09D04746D1E76378EF
:10489000526962600A2161F307136370C9E75369C3
:1048A0006278072161F307126270E2E710B5002316
:1048B0000446037043708370C37003714371837146
:1048C000C3714FF40072FFF7ADFF204610BD00002A
:1048D0002DE9F0432DED028B85B00446154699462F
:1048E0009DF838800F46002948D0002A00F0E78064
:1048F00000230B70017871B319F4807F2BD0714BBA
:1049000001EBC101194438460EF00FFE637813F035
:10491000F00F07D019F4007F04D02A466A493846C0
:104920000EF0DDFD38460EF0D2FD2D1A3E18013D89
:10493000637813F0F00F21D019F4007F1ED01B090B
:10494000013B0B2B1AD8DFE803F0084071A6AC2519
:104950007B7B7B221FB43E46EAE72079B8F1000F4B
:1049600006D0642300930023FF2219460BF01FF9A1
:10497000564A0346294630460EF09EFC384605B09E
:10498000BDEC028BBDE8F0836368514AF2E76368CF
:10499000504AEFE7616800294FF064020EDA91FB9C
:1049A000F2F04B4202FB1011494293FBF2F34A4AE8
:1049B0000091294630460EF07FFCDFE791FBF2F3D1
:1049C00002FB13120092454AF3E72046FFF7FFFB74
:1049D000E279A37994F8059001B20029207902F0D8
:1049E000010202DBB8F1000F14D043EA0224B8F14F
:1049F000000F06D0642300930023FF2219460BF01A
:104A0000D6F8CDE900902346354A294630460EF0C7
:104A100053FCB3E7CDE90101CDF8009043EA02234E
:104A2000304A294630460EF047FCA7E7E379A279E1
:104A30006179009103F0010342EA03232A4AB8E7AF
:104A4000636808EE103AB5EEC08AF1EE10FA4CBF7A
:104A5000F1EE487AF0EE487AFDEEE78AB8EEE87AB1
:104A600077EEC77A9FED217A67EE877A17EE900A84
:104A70000BF0F0FC07EE900AB5EEC08AFDEEE77A87
:104A8000F1EE10FACDED007A18EE903A01D5184A01
:104A90008FE7184A8DE72279A37901926279009213
:104AA000B2E7E279A37902922279019262790092C7
:104AB000B6E72A46616830460EF037FD5EE71746D6
:104AC0005CE700BF99730100687101001175010076
:104AD00014750100187501001C7501001D75010099
:104AE00029750100267501002C75010000007A442B
:104AF000327501003375010030B58BB0134C0023C3
:104B00002022009302A94FF440730546FFF7E0FE10
:104B100002A920460AF0CDFB0D4920460AF0C0FB51
:104B200069780A22090920460AF03CFC0949204616
:104B30000AF0B6FB69780A2201F00F0120460AF05C
:104B400031FC20460AF0BCFB0BB030BD6C030020EA
:104B5000FE7401000375010070B54B78B2EB131FB2
:104B600086B005460C46164606D123682B6063685E
:104B70006B60284606B070BD184919480AF090FBD2
:104B8000617817480A2209090AF00CFC15491448F3
:104B90000AF086FB0A22314611480AF003FC12494A
:104BA0000F480AF07DFB0023CDE9043366F30713B9
:104BB00022788DF811304FF0FF338DF810200093DC
:104BC00002A86368226804A900F010F8029B236021
:104BD000039B63602046FFF78FFFC6E73B7501002C
:104BE0006C030020C6700100687101002DE9F04FD0
:104BF0008DB004AD85E80C00BDF85830112B98BF7E
:104C0000B64A804628460C4694BF12F803904FF0EF
:104C10000009FFF7DCFA011E02DB2046FFF7B1FABC
:104C20009DF811306278C3F3030161F303026270EF
:104C30009DF810102170C2F303120B2A38D8DFE858
:104C400012F0A0000C000C00C9002F010D01A800FB
:104C5000CF00CF00CF00A800A8001B090C2B77D8ED
:104C6000DFE803F0265244180A07395576763030CB
:104C70006E009DF81720E2719DF81620A2719DF834
:104C8000152062719DF814202271627863F3071277
:104C900062700DE0BDF81630C3F30802E379A2712B
:104CA00023F0010343EA1223E3719DF81530637189
:104CB000B9F1000F00F0FC804A46214606A8FFF734
:104CC0004BFFF5E0059B002B36DBFF2BA8BFFF2336
:104CD000DBB22371ECE7059B13F1630F2CDBB3F51B
:104CE000C84F2BDA642293FBF2F3F1E7BDF81630DC
:104CF000C3F30802E379A27123F0010343EA12230C
:104D0000E3719DF8153063719DF81430E1E7DDED36
:104D1000057AF5EEC07AF1EE10FA0DD49FED707AB7
:104D2000F4EEC77AF1EE10FA08DCFCEEE77ACDED8E
:104D3000027A9DF80830CCE70023CAE7FF23C8E7D2
:104D400063780C2262F307136370059B6360AFE71F
:104D5000644965480AF0A4FA9DF8111062480A22D5
:104D600009090AF01FFB61495F480AF099FA617866
:104D70005D480A2209090AF015FB5B480AF0A0FA0F
:104D800096E762781B0963F307120598627060600A
:104D90008EE71B09032B04D00C2BD1D0059A62603F
:104DA00073E700212046FFF70DFCBDF81630207197
:104DB000C3F30802E379A27123F0010343EA12234B
:104DC000E3719DF8153063716378022262F3071373
:104DD00063706DE700212846FFF7F4FB2071F3E7CD
:104DE0001B090C2BB4D801A252F823F0B14C0000DF
:104DF0002B4E0000594E0000A34D0000594E0000FC
:104E0000594E0000214E00004D4E00004D4E000056
:104E10004D4E0000394E0000474E0000414D00004D
:104E2000059B636006226378D0E79DF8143007EE97
:104E3000903AF8EE677A03E0DDED057AF8EEE77A6E
:104E400017EE903A82E7DDED057AF2E7627863F3D8
:104E500007126270059B79E7627894E701271B09C6
:104E60000C2B3FF675AF01A252F823F0B14C0000B5
:104E7000C54E0000194F0000C54E0000A54E0000B1
:104E8000A54E0000C54E0000C54E0000514D00006B
:104E9000514D0000C54E0000C54E0000414D0000C0
:104EA0000027DCE7059A6260627863F3071262709C
:104EB0002368C8F800306368C8F8043040460DB075
:104EC000BDE8F08F013B0A2B00F2CD80DFE803F054
:104ED000BACB10CBCBBFC4CBCBBDBD008773010019
:104EE00000007F437A7401006C030020C67001004B
:104EF000FF23BDF816208DF81430642161F30802F9
:104F0000ADF8162000228DF815209DF81120022101
:104F100061F307128DF811200023FF259DF815007D
:104F20000095642219460AF042FE0028C0F29D80D6
:104F300000239DF815000095642219460AF037FEFB
:104F4000A84208DC002300959DF81500642219464C
:104F50000AF02DFE05469DF81400FBF779FA064687
:104F6000002F47D09DF817707F08013F3FB27B1C90
:104F700040F088807F2D4FF0FF0778DC0023C5F1DB
:104F80007F00194647F68162704300970AF00FFED2
:104F90004FF4FF73009300231946E0717F222846E7
:104FA0000AF005FE0023194600903A4630460AF002
:104FB000FEFD00970646642328467F2200210AF062
:104FC000F6FDBE420546A8BF3E466B496B480AF057
:104FD00067F90A22294669480AF0CBF96849674807
:104FE0000AF05EF90A22314664480AF0C2F96348C1
:104FF0000AF066F900231A46194606A809F0C9FF07
:10500000BDF816004FF6FF7300930023194640F2D7
:105010006D12C0F308000AF0CAFDF2B2E9B280B224
:1050200009F0CDFF030CA371030A63712071554988
:1050300052480AF035F92046FFF75EFD06A809F050
:105040003DFF35E69DF8143053E7059B51E7059B7E
:10505000642293FBF2F34CE7DDED057AFDEEE77A8F
:1050600017EE903A45E7002343E7002573E76423F2
:10507000284600973A4680210AF099FD002305460C
:10508000E371A2E74FF01E0B64231A46CDF800B07F
:10509000002138460AF08BFD4FF0640A03905B460E
:1050A0003846CDF800A0524600210AF080FD7F2D41
:1050B00083464FF0FF0754DCC5F17F0000237043A7
:1050C0001946314A00970BFB00F00AF070FD4FF4CF
:1050D000FF73E0710398009300231946E322281818
:1050E0000AF065FD00231946029000903A463046CA
:1050F0000AF05DFD00230646009728467F221946E8
:105100000AF055FDBE420546A8BF3E461F491B4852
:105110000AF0C6F80A22039918480AF008F91C494F
:1051200016480AF0BDF80A22594614480AF0FFF85A
:10513000184912480AF0B4F80A2229460F480AF022
:1051400018F915490D480AF0ABF80A2231460B4808
:105150000AF00FF9114909480AF0A2F80A22029947
:1051600042E75346284600973A4680210AF01FFD41
:1051700000230546E371C9E78C7401006C0300202D
:1051800099740100CC740100646A3100A7740100B5
:10519000AD740100B3740100BB740100C37401005D
:1051A000F8B5054617460C4611B900263046F8BD3D
:1051B0000846FDF74BFA06460028F6D0FA0503D557
:1051C00029782046FDF780F8BB050DD56B78696816
:1051D0001B09073B2046042B11D8DFE803F003032B
:1051E000100D0D00FDF7B0F909490A480AF058F80A
:1051F0002846FFF781FCD9E7FDF78AF9F4E7FDF7C8
:1052000087F9697820460909FDF7BAF9ECE700BF8C
:105210000A7501006C03002073B504460D46FFF7C4
:1052200001FB0646E8B9104910480AF039F828464B
:10523000FDF760FD214602B26846FEF719FF2146E0
:105240006846FEF749FF29464FF400722046FFF7F3
:10525000A7FF2046FFF750FC4FF420612846FDF7DA
:10526000EFFC304602B070BDD37401006C03002027
:1052700043781B09013B012B37B5054620D8002395
:10528000FF2400790094642219460AF090FC00285B
:1052900014DB002328790094642219460AF087FC65
:1052A000A04207DC002300942879642219460AF002
:1052B0007EFCC4B22C71012003B030BD0024F9E79C
:1052C0000020F9E707B5002300931A461946034862
:1052D00009F09EFF03B05DF804FB00BF400300200F
:1052E00002F000BD02F0C4BC07B5002300931A46CB
:1052F0001946034809F08CFF03B05DF804FB00BFBA
:105300004803002038B5094D01244FF47A700AF0A3
:10531000F7FD214601340A222846E4B20AF042F899
:10532000142CF2D14FF4FA7038BD00BFB80300203E
:1053300008B50449044809F0B3FF04F019FB4FF421
:10534000FA7008BD247A0100B803002010B50446A5
:1053500004300AF036FC204610BD00000128F8B5E4
:1053600007460C46174E184D13DD48680CF083FEB7
:10537000C1B216483170FBF763FC022F07D0A0685A
:105380000CF079FEC1B211482970FBF76AFCC82401
:1053900001E04FF4C8740E490E4809F081FF0A225B
:1053A00031780C4809F0FEFF0B490A4809F078FFF4
:1053B0000A222978074809F0F5FF064809F080FF1E
:1053C0002046F8BD05000020060000204004002013
:1053D000B97B0100B8030020CD7B010030B587B058
:1053E0000023044600931A460D4602A8194609F008
:1053F0000FFF04A809F004FF042C12DD04A928699A
:1054000004F0C1F968B104A92348FBF71CFB04A907
:10541000E86804F0B8F950B104A91F48FBF75FFB36
:105420000BE002A91C48FBF70EFB032CEFDC02A9E2
:105430001948FBF754FB022C18DD04A9A86804F0F6
:10544000A2F998B104A91448FBF723FB04A96868E2
:1054500004F099F980B104A90F48FBF7CEFA0F497F
:105460000F4809F01DFFC82007B030BD02A90A4847
:10547000FBF70FFB012CE9DC02A90748FBF7BDFA9B
:10548000012CECD102A90448FBF7B7FA05490448FE
:1054900009F006FFE3E700BF40040020AA76010000
:1054A000B80300209A76010008B548B1496805485C
:1054B000FBF728F90449054809F0F2FEC82008BDA9
:1054C0000146F4E7400400200C770100B8030020F7
:1054D00008B548B149680548FBF73FF90449054854
:1054E00009F0DEFEC82008BD0146F4E740040020B4
:1054F0000E7A0100B803002030B5144D144C85B06D
:10550000772201212846FBF7C7FD00230193114BA9
:105510000093114902954FF0FF332046039309F0A1
:10552000BFFE0E4B0E4819686A4608F001FC28467B
:10553000FBF76CFD0B49204609F0B2FE204609F04E
:10554000BFFE0948FBF776FC05B030BD58040020CB
:10555000B8030020F88801007479010034040020A9
:10556000900700208E79010040040020012810B52A
:105570000C4622DD124960680DF041FF18B9012187
:105580001048FBF72DFB104960680DF038FF01460D
:1055900010B90C48FBF724FB0C490D4809F080FEBC
:1055A0000848FBF714FB0A220146094809F0E1FE0E
:1055B000074809F085FEC82010BDFFF79DFFFAE7F8
:1055C000DC81010040040020DF8101009E790100A0
:1055D000B803002070B52DED028B08EE102A8EB0B6
:1055E0001C22334B06930C460DEB020000210CF0FD
:1055F000C8FF06AA0821204603F0CCFF2D4B1B68EC
:1056000000258DF82950002B4ED02B4809F058FE6C
:105610002A49294809F044FE18EE100A0CF06AF9EC
:1056200002230246009324480B4609F077FF2449E1
:10563000214809F035FE06A91F4809F03AFE214924
:105640001D4809F02DFE1C4809F03AFE1E4B1F486C
:10565000196806AA08F0A3FBDFED1D7AB4EE678A8D
:10566000F1EE10FA06461FD0DFED1A7AB4EE678A23
:10567000F1EE10FA18D0B5EE408AF1EE10FA13D020
:1056800018EE101A04AC02A8FEF7E7FC032202A9E8
:105690002046FFF7BDF8CDE900554FF0FF3194E803
:1056A0000C00304604F08EF90EB0BDEC028B70BDDC
:1056B0004E494C00340400206C0300201D7301008F
:1056C000B47F0100C770010028040020900700206B
:1056D0000000FEC20000AA4210B50C48FBF764FBB4
:1056E00018B10B490B4809F0DBFD0B4C722201216C
:1056F0002046FBF7D1FC237D1BB1FF212046FBF7A1
:1057000077FC0548FBF782FCC82010BD4004002050
:10571000157D0100B803002058040020034B93F9C5
:105720000000053818BF0120704700BFDC030020CF
:1057300030B593B000230A460546402101A804F085
:1057400093F801A80DF0C3FE01A9044602462846BD
:105750000DF0D9FE00280CBF2046002013B030BD4C
:10576000F0B504469DB00E4601B18AB96E496F4846
:1057700009F096FD6E496D4809F092FD21466B488F
:1057800009F097FD6B49694809F08AFD674821E0F7
:1057900000258D5403F0EFFF63490746634809F085
:1057A0007FFD0A223946614809F0E3FD62495F48FE
:1057B00009F076FD21465D4809F07BFD5F495B48B5
:1057C00009F06EFDB7F59D7F08DA5D495D4809F087
:1057D00067FD5C4809F074FD1DB0F0BD04215A4816
:1057E0005A4F03F04FFE5A49504809F059FD3146CF
:1057F0004E4809F05EFD56494C4809F051FD4B48B2
:1058000009F05EFD3C2229460DA80C950CF0B9FE6E
:1058100097F90020052A2FD103212046FFF788FFA2
:1058200005B2002D34D14B4BDB681B78DB07D3D599
:1058300002212046FFF77CFF00B2A8B124212046B8
:105840000DF094FE0028C7D14349384809F028FDDF
:105850002146364809F02DFD344809F031FD214636
:105860003C4808F05AFFB7E701212046FFF760FFE8
:1058700000B20028B0D0E1E701212046FFF758FF31
:1058800005B2C5B902212046FFF752FF05B2C5B1E6
:105890002544324928460DF0ECFDA0B930460DF004
:1058A00016FE01280FD921462A4808F036FF304657
:1058B00008F028FB90E73F2221460CA80DF035FEAA
:1058C000E6E727495FE7204624210DF04FFE044616
:1058D000002881D1294601A8FCF77AFF01A8FCF72E
:1058E000B5FEE0B12246314601A8FDF7BFFF002812
:1058F00015DD9DF8303093B197F90030052B0ED0AF
:1059000018490A4809F0CCFC0CA9084809F0D1FC58
:10591000064809F0D5FC0CA90E4808F0FEFE01A8C7
:10592000FCF7BAFC58E700BF198901006C0300209E
:1059300043760100588E01004C7601004F7601003D
:10594000527601008803002038040020DC03002088
:1059500044700100E40300205F7601006A810100C9
:1059600077760100827601002DE9F041164917484B
:10597000174E184F154D09F093FC0024A6F10F089F
:1059800016F8013F0F2B03D83946284609F091FC41
:10599000052C4FF010020DD03178284609F0C7FCD5
:1059A0000D49284609F07CFC0134E4B2062CE7D10D
:1059B000BDE8F08198F81510284609F0B8FC284693
:1059C00009F07EFCF0E700BFAF790100B8030020CA
:1059D0004F040020DC8801005872010010B58AB025
:1059E0000DF11F0304930DF12503039309AB0C463E
:1059F00002930DF1230301930DF12203009308AAF2
:105A00000DF121030E4960680DF08AFC05280BDCBE
:105A10000C490D4809F044FC61680B4809F049FC49
:105A20004FF4C8700AB010BD08A90848FAF71DFE67
:105A3000FFF79AFF0649074809F032FCC820F1E752
:105A4000367A01004A7A01008803002040040020D1
:105A50005C7A0100B803002008B508B9002008BD31
:105A6000037C03F00F03052BF8D1CAB201460648A8
:105A700008F08DF90028F1D0037C03F00F03042B0C
:105A8000ECD14069EBE700BF90070020F7B53C4C34
:105A90002678002E6CD13B4B93F90030012B67DD4B
:105AA000394B1968002963D0384A394808F077F92A
:105AB000054600285CD00146354808F060F907B279
:105AC000002F55D031462846FFF7C6FF012F064666
:105AD00050D0294601222E4808F059F945696846F8
:105AE00005F06EF810222B49684603F071FE2A4932
:105AF0002A4809F0D5FB3146284809F0DAFB284945
:105B0000264809F0D6FB0A222946244809F031FC30
:105B10002349224809F0CDFB1E49204809F0C9FB62
:105B20001E4809F0CDFB40F202211E4805F0E0FAC4
:105B3000AAB231461C481D4D09F0B0FA15491A4861
:105B400009F0B0FA1A4B186818B10021FFF784FF6A
:105B50002860296889B1144809F0ACFA002112487C
:105B600009F0B0FA012313490C48237009F098FB9F
:105B700003B0F0BD40F20225B1E70F49EBE700BFEB
:105B80007C040020DC030020340400200C7601009B
:105B9000900700205803002013760100B80300206E
:105BA00058720100BC0400209804002084030020E7
:105BB000E003002022760100308201002DE9F04F41
:105BC000A7B0002396488DF81330CDE90533CDE911
:105BD000073308F0B9FB934F054610B105233B701E
:105BE000F8E0914C216841B99049914809F058FB7F
:105BF0008F4809F065FB0F23F1E78E4808F0BFF8E6
:105C00000FFA80F8B8F1010FEEDD294620688A4EC0
:105C1000FFF722FF002800F0E080306087498848C5
:105C200009F03EFB3168864809F043FB844809F0DF
:105C300047FB01212068FFF70FFFB8F1020F8246F2
:105C400000F0CE80022221687A4808F0A0F8B8F16E
:105C5000030FD0F8149000F0C58003212068FFF7EF
:105C6000FBFE0546102205A97648FAF725FD002817
:105C700040F0BB80B8F1040F40F3B78004212068E6
:105C8000FFF7EAFE704904466D4809F009FB6C48CD
:105C900009F016FB1FFA89F25146614808F0C0FE70
:105CA0000DF1240869495E4808F0BDFE0DF1340B82
:105CB0001022674940460DF038FC002301222021C4
:105CC000584603F0D1FD634958460DF0B6FB6249D2
:105CD0005B4809F0E5FA5146594809F0EAFA5F498C
:105CE000574809F0DDFA0A224946554809F041FBB8
:105CF0005B49534809F0D4FA2946514809F0D9FACA
:105D000058494F4809F0CCFA2B780BB91C461D4670
:105D1000CDF80C804FF002094FF001082A46CDE97A
:105D20000198CDF800B0234631683D484E4D08F04B
:105D300021FC00285BD04D4B4D49414800241C708C
:105D400009F0AEFA31683E4809F0B3FA3C4809F070
:105D5000B7FA484B032283F800804121234615A857
:105D600003F082FD444915A80DF067FB15A92C48E6
:105D700008F024FE23464A46412115A803F074FD8D
:105D80003E4915A80DF059FB15A93D4809F0A8FAA0
:105D900015A9234808F012FE42462346412115A8C2
:105DA00003F062FD354915A80DF047FB15A93548EC
:105DB00009F096FA15A91A4808F000FE05233B7071
:105DC0000AF06AF8304928601D4809F069FA1C4851
:105DD00009F076FA27B0BDE8F08F2C4B33601DE751
:105DE00040F25B790DF113053CE705AC52E7284919
:105DF0000F4809F055FA0A4808F017FE0A22014632
:105E00000B4809F0B6FA2349094809F049FA08484D
:105E100009F056FA0AF040F80C232860DFE600BFCC
:105E2000E4030020DC030020E0030020D57E010015
:105E30008803002090070020840300200B7F0100CE
:105E4000B803002040040020187F010061570000C3
:105E5000CF8101001A820100387F010058720100D1
:105E6000587F01000A8101008404002024040020DE
:105E70005F7F01006A0300206D7F0100C470010094
:105E80006C030020EC070020737F010030820100CA
:105E9000907F01009C7F010010B5114C11492046F4
:105EA00009F0FEF91049204609F003FA4FF4FA70A0
:105EB0000AF026F8012115200AF0DEF9002115204C
:105EC0000AF002FA4FF4FA700AF01AF815200121CC
:105ED0000AF0FAF94FF4FA70BDE810400AF010B871
:105EE000B8030020478101006781010070B592B0BE
:105EF00002A809F085F904A809F082F906A809F0BA
:105F00007FF908A809F07CF955495648564E09F022
:105F1000C7F9544809F0D4F902A95448FAF799FC92
:105F2000002877D052494F48524C10AD09F0B8F9CB
:105F3000039B10942846119303F070FC04A94B486E
:105F4000FAF7F1FC00285DD04B49464809F0A8F962
:105F5000059B10942846119303F060FC06A9434862
:105F6000FAF716FD002841D044493E4809F098F957
:105F7000079B10942846119303F050FC08A93B4856
:105F8000FAF79CFC10B33E49364809F089F9099BA1
:105F900011932846109403F041FC039B0095CDE932
:105FA0000B34059B37480A94CDE90D34079BCDE9A6
:105FB0000F34099B11930CAA0EAB0AA904F02AFD19
:105FC000284809F07DF9022333703BE0039B2D48FC
:105FD0000C94CDE90D34059BCDE90F34079B11934B
:105FE0000EAA2B460CA904F045FDE9E7039B2548C2
:105FF0000E94CDE90F342A46059B11930EA904F0A7
:1060000061FDDDE7039B1F4810942946119304F0BE
:1060100073FDD5E71C49134809F042F94FF47A6241
:1060200042F6E061174804F06BFC68B9174918485C
:1060300009F036F91749164809F032F9F62333709A
:10604000FFF72AFF12B070BD1349064809F028F97E
:1060500010A804F0B5FD10A803F0E0FBB0E700BF06
:10606000537C0100B8030020DC0300204004002022
:10607000607C0100C4890100767C01007C7C010009
:10608000817C010050040020887C0100947C010088
:1060900088030020D67C0100057D010007B510496A
:1060A000104809F0FDF8684604F08AFD684603F0E0
:1060B000B5FB0D4B00930D4B68465B68019303F0F5
:1060C000ADFB684604F0C0FD684603F0A7FB6846D8
:1060D00004F098FD684603F0A1FB03B05DF804FBF3
:1060E0002D7C0100B8030020C48901007C0600203B
:1060F00018B10349034809F0D3B80349FAE700BFD0
:1061000045810100B80300205B8E010010B5264CCC
:106110002649204609F0C4F82549204609F0C0F870
:10612000244B1868003018BF0120FFF7E1FF224917
:10613000204609F0B5F8214B1868003018BF01203F
:10614000FFF7D6FF1E49204609F0AAF81D4B186834
:10615000003018BF0120FFF7CBFF1B49204609F094
:106160009FF81A4B1868003018BF0120FFF7C0FFD6
:106170001749204609F094F8164B1878FFF7B8FF36
:10618000204609F09DF81449204609F089F803F0EB
:10619000F2FA0A220146204609F0F7F82046BDE847
:1061A000104009F08DB800BFB8030020827B0100C9
:1061B0008F7B0100D8030020977B0100D4030020CF
:1061C000A07B0100E0030020A77B01002804002041
:1061D000B07B01007C0400200B72010010B5424C22
:1061E0004249204609F05CF84149204609F058F838
:1061F0004049204609F054F83F49204609F050F83C
:10620000204609F05DF83D49204609F049F83C492F
:10621000204609F045F83B49204609F041F83A4943
:10622000204609F03DF83949204609F039F8384947
:10623000204609F035F83749204609F031F836494B
:10624000204609F02DF83549204609F029F834494F
:10625000204609F025F83349204609F021F8324953
:10626000204609F01DF83149204609F022F830494E
:10627000204609F015F82F49204609F011F82E495B
:10628000204609F00DF82D49204609F009F82C495F
:10629000204609F005F82B49204609F001F82A4963
:1062A000204608F0FDFF2949204608F0F9FF28495B
:1062B000204608F0F5FF2749204608F0F1FF26495F
:1062C000204608F0EDFF2549204608F0E9FF244963
:1062D000204608F0E5FF2046224908F0E1FF20466D
:1062E000BDE8104008F0ECBFB8030020257D010098
:1062F000477D01005A7D0100687D0100707D01002D
:10630000807D01008C7D0100997D0100AE7D010042
:10631000BD7D0100C57D0100D07D0100DA7D010059
:10632000E97D0100F17D0100FD7D01006781010033
:10633000137E0100327E0100477E0100547E010081
:10634000627E01006E7E0100767E0100817E01008A
:106350008E7E0100967E0100A17E0100B07E0100CC
:10636000B97E0100C77E010008B5FFF737FFFFF7D0
:1063700095FE0349034808F093FFC82008BD00BFFD
:1063800023770100B803002070B594B003F0F3F94F
:10639000064609F081FD0546234807F0D5FF002891
:1063A0003FD0224B1C7864B2002C3AD12346012204
:1063B000402104A803F058FA1D4904A80DF03DF847
:1063C0001C4904A80DF039F81B4904A80DF035F854
:1063D0003146684603F0C6FA01236A4604A912480A
:1063E00008F00FFA23460122402104A803F03CFAEA
:1063F0000F4904A80DF021F80E4904A80DF01DF86E
:106400000E4904A80DF019F868464FF47A71B5FBEF
:10641000F1F103F0A7FA01236A4604A9024808F043
:10642000F0F914B070BD00BFE4030020B4030020F5
:1064300021820100C47A01007D81010039820100BE
:1064400010B50C4C2046FAF7E1F878B90A490B4828
:1064500008F026FFDE232374AD236374BE23A374E8
:10646000EF23E374FE232375FF236375BDE810401B
:10647000FFF77ABA40040020E7790100B803002052
:1064800008B5002007F0E8FD1A491B4808F008FF8E
:106490001A491B4807F07AFD1A491B4807F076FD98
:1064A0001A491B4807F072FD1A491B4807F06EFD98
:1064B0001A491B4807F06AFD1A491B4807F066FD98
:1064C0001A491B4807F062FD1A491B4807F05EFD98
:1064D0001A491B4807F05AFD1A491B4807F056FD98
:1064E0001A491B4807F052FD1A491B48BDE80840ED
:1064F00007F04CBDB47901006C0300206963000013
:10650000B87901006D550000BD7901009D70000053
:10651000C2790100A97300009D820100DD590000CD
:10652000C779010005530000CB790100DD5300005D
:10653000D0790100A9540000D6790100D15400009F
:10654000D3790100D9560000DA79010031530000F7
:10655000E07901005D5300000F7601002DE9F04F56
:10656000494F3B6887B08046002B00F08A80474C3B
:1065700025786DB2002D40F084802278444EDFF8FB
:106580001C91013252B222703278013252B2327012
:10659000D9F800A009F080FC2B4601460B2250469A
:1065A00003F0F6F900283AD03B68DFF8F4A0DD6884
:1065B000DFF8F0B04DB32B7C03F00F03062B22D194
:1065C00052462946584607F0EAFB98B1037C03F08F
:1065D0000F03052B0ED1C368ABB119462A4603A899
:1065E0000193FAF7EDFD414603A8FBF7E5FC019B9B
:1065F0005B68F1E72946002203A8FAF7E1FD41466E
:1066000003A8FBF7D9FC6D68D4E7B8F1030F03D0FA
:1066100009F042FCC9F800001E48FBF751FDB8F133
:10662000030F26D01C4DD5F8008009F035FC00235F
:10663000014641F28832404603F0AAF9A846C0B1AB
:106640003B68DD688DB12B7C03F00F03062B08D16E
:106650002946002203A8FAF7B3FD012103A8FBF79E
:10666000ABFC09F06FFC6D68ECE709F015FCC8F8AD
:1066700000003378013B5BB233702378013B5BB29F
:10668000237007B0BDE8F08FD4030020D1030020B1
:1066900069030020300300208C04002080040020C7
:1066A0001B710100900700200320FFF757BF000077
:1066B00010B5094C237801335BB2237009F042FC1A
:1066C0000320FFF74BFF09F03DFC07F0B9FC2378EE
:1066D000013B5BB2237010BDB403002030B5114BF9
:1066E000196885B0D9B1104CCD682278013252B208
:1066F000227085B12B7C03F00F03062B07D10022FB
:10670000294601A8FAF75CFD01A8FBF7ADFC09F0EA
:1067100019FC6D68EDE72378013B5BB2237005B08F
:1067200030BD00BFD4030020690300202DE9F04FE5
:10673000914C23688FB0002B00F019818F4F3B786C
:10674000002B40F014813B788D498E488E4D0133EB
:106750005BB23B7008F0A4FD8A4808F0B1FD8B4A9B
:1067600021688B4807F01BFB8A4A2860216888480B
:1067700007F015FB884B894A18602168844807F0A8
:106780000EFB874B874A18602168814807F007FB9A
:10679000854B1860FFF77AF9844A21687C4807F036
:1067A000FEFA834BA946186030B3824D2B781BBB91
:1067B000C468814802F0C0FC002814BF01230023F4
:1067C0002B7003D07D496F4808F06AFD7C4B002296
:1067D0001A608CB12B787BB1237C03F00F03062B5E
:1067E00006D1206803A902F006FF03A802F0E0FD2D
:1067F00009F0A8FB6468ECE7724A00231360D9F83B
:1068000000309246002B00F09480D3F80C80DFF823
:10681000D8B16D4CD9F80030002B00F0AB80B8F146
:10682000000F00F0838098F8102002F00F02052A74
:10683000F2D14146564807F0A2FA0128EAD941466A
:1068400003A8FBF78FFF03A8FBF700FFA8B103A87D
:10685000FBF794FD064680B9014603A8FBF7CAFD85
:10686000051E03A8BCBF6D420126FBF71FFD9DF866
:106870001C20052A09D0062A32D009F063FB03A8A0
:10688000D8F80480FBF708FDC4E718B9022103A873
:10689000FBF71AFD4FF4807103A8FBF757FD059B2A
:1068A00023B14FF4007103A8FBF750FD01212846E6
:1068B00009F0E2FC0021284609F006FD5946204671
:1068C00008F0EEFC29460A22204608F052FD3F4916
:1068D000204608F0E5FC3E49204608F0E1FCCCE704
:1068E00001900121284609F0C7FC019BD6B113F1A4
:1068F000FF3618BF01263146284609F0E5FC354928
:10690000204608F0CDFC0A222946204608F031FD39
:106910003149204608F0C4FC0A223146204608F0DE
:1069200028FDD8E7013B5E425E41E4E7DB68CAF838
:1069300000302548294C08F0C3FCFFF7CFFEFFF7D5
:10694000E5FB274B274801221A7004F0DDF920B13E
:10695000244804F09BFA0423237094F90030072B99
:1069600004BF042323703B78013B5BB23B700FB044
:10697000BDE8F08FDB68FFDE3404002069030020EF
:10698000CF750100B8030020D8030020DF75010097
:1069900090070020897F010094040020807001008E
:1069A000D4030020E5750100E0030020EA75010032
:1069B000280400202C040020D5550000ED750100AE
:1069C0003C050020300400206C0300200576010007
:1069D0000A7601000873010047710100DC03002002
:1069E00068030020A0030020FD7501002DE9F0439D
:1069F0003B4C23688DB0002B6ED03A4D2E6809F0C9
:106A00004BFA002301464FF47A72304602F0C0FF81
:106A1000074610B109F040FA2860334DDFF8D490F2
:106A20002B7801335BB22B702368DE687BB2002BBE
:106A300014BF4FF004084FF002082268F2B1EEB123
:106A4000337C03F00F03052BF8D13146484607F09D
:106A500096F90128F1D9314601A8FBF783FE01A878
:106A6000FBF7F4FD18B1414601A8FDF723FA09F040
:106A700069FA01A87668FBF70FFCDEE72B78013B8B
:106A80005BB22B70194B93F90030052B24D01FB348
:106A9000174F00263D463968F1B1EEB90B7C03F083
:106AA0000F03052B0CD101A8FBF75CFE012101A807
:106AB000FDF700FA061C01A818BF0126FBF7ECFB46
:106AC0002B684BB109F03EFA2B685B682B60002BFA
:106AD000E1D12368DB682B600DB0BDE8F08300BF17
:106AE000D80300208804002069030020DC03002074
:106AF000300400209007002070B580EAE074A4EB19
:106B0000E0740E4605460121204609F0B5FB022E31
:106B10000CD10021204609F0D7FB0B490B4808F0A7
:106B2000BFFB0A48BDE8704008F0CABB36B9E9436C
:106B3000C90F204609F0C8FB0549EFE7E90F2046D9
:106B400009F0C2FB0349E9E73B7601006C03002032
:106B50000D830100188301002DE9F0472DED048B12
:106B6000754B94B01C6809F097F90023014647F271
:106B70003052204602F00CFF002800F0D7806F4B07
:106B80001A68002A00F0D2806D49D4680B78DFF8CB
:106B9000EC819FED6C9A01335BB20B70002C00F01E
:106BA000BA80237C03F00F03052B12D1002221466B
:106BB000404607F0ECF84369052B0AD1214609A8A5
:106BC000FBF7D0FD09A8FBF741FD20B909A8FBF7A9
:106BD00063FB6468E2E709A907A8FDF767FE09A857
:106BE000FBF7DCFC0021064609A8FBF703FC054681
:106BF00007A8FDF70FFC08EE900A09A8FBF756FB63
:106C000033B207EE903AF8EEE77A824687EE898A49
:106C100009A8FCF7E9FF4C4981464C4808F040FBC5
:106C2000022718EE900A0AF065FE009702460B460E
:106C3000CDE90401454808F071FC4549434808F096
:106C40002FFB18EE100A0AF055FE009702460B467D
:106C5000CDE902013D4808F061FC3E493B4808F09F
:106C60001FFB51460A22394808F083FB5FEA164AA7
:106C70004CD0082003F00AF84FF6FF7381B240F6BB
:106C80002712504602F084FEA8B12168324808F06D
:106C900010FB3249304808F003FB22683049314884
:106CA00007F09AFDB1B209A8FBF790FC39462846D7
:106CB000FFF722FF8AE7DFED2C7AB4EEE78AF1EEE8
:106CC00010FA04DD22682949264807F085FDB9F14C
:106CD000000F01D10121EAE70022254BDDE9040183
:106CE0000AF0A8FCDDE902230BF0ECF808B1002162
:106CF000DDE7F4EEC88AF1EE10FAEBD91D4913482E
:106D000008F0CEFA114808F0DBFA5FE71A490F489D
:106D100008F0C6FA5AE70A4A1378013B5BB21370CF
:106D200009F0BAF8044B1860FFF72EFB14B0BDEC65
:106D3000048BBDE8F08700BF90040020D80300203A
:106D4000690300200000C8428B7501006C0300201D
:106D500091750100B272010088030020977501004F
:106D6000A7750100E403002000001842B37501007C
:106D70000000F03FC07501009D75010090070020E4
:106D80002DE9F043664E33688DB0002B00F0C580CE
:106D900064496548654CDFF8E48108F081FA62488F
:106DA00008F08EFA09F078F8274605462378F3B103
:106DB00009F072F80023014642F21072284602F0F0
:106DC000E7FDA0B907F03CF998F80030002B4FD14F
:106DD000574B93F90030052B01D0FFF707FEFFF763
:106DE000BBFE0220FFF7BAFB09F0ACF8DEE73B7808
:106DF000002B44D101274F494F4D4B4808F050FA22
:106E0000494808F05DFA2B784C4A01335BB22B708D
:106E100013689046002B3BD0DC68DFF84491002CCF
:106E200036D0237C03F00F03052BF8D121464846CA
:106E300006F0A5FF0028F2D0237C03F00F03052BFA
:106E400014D12146484606F09AFF78B1216801A87E
:106E5000FBF7BEFC01A8FBF7F9FB10B101A8FBF79B
:106E600015FA09F06FF801A8FBF716FA6468D6E77F
:106E7000334B1B68002BABD002F084FAA8E73149F2
:106E8000314808F00DFA304808F01AFA0027B2E746
:106E90002E4B2F49244800241C6008F001FA224898
:106EA00008F00EFA642009F02BF82A4B2A491C70CE
:106EB0002A4B1D481C7008F0F3F902F05CFC0A2212
:106EC0000146194808F061FA3168254806F072FB5E
:106ED000244B25491C60254B13481C60244B34600F
:106EE0001C60244BC8F800401C60154B1C6008F067
:106EF000D7F902F040FC0A2201460B4808F045FA97
:106F0000094808F0DDF91C4B1C702B78013B5BB283
:106F10002B7038460DB0BDE8F0830127F9E700BFBC
:106F200034040020D78001006C0300206903002096
:106F3000DC0300200F8101007D040020D803002025
:106F400028040020EC800100880300203004002089
:106F5000258101007C0400202D81010068030020B0
:106F600090070020D40300208273010094040020C5
:106F7000E0030020840300206A0300202C0400208A
:106F800030B5394B1D786DB289B0002D37D13749F6
:106F9000374C384808F084F9364808F091F97222E5
:106FA00001212046FAF778F82046FAF711F87B28F5
:106FB00036D1314B04934FF0FF3307930595069478
:106FC000FFF7DEFE04A92D482D4D06F00BFE2860CC
:106FD0002046FAF71BF82C689CB92A492A4808F081
:106FE0005FF9294808F06CF9284901A808F02EFE3D
:106FF00001A92748F9F79AFE01A808F0E2FD002050
:107000000CE024491B4808F04BF91A4808F058F9DD
:10701000FFF78CFB1E48F9F74FFF012009B030BD88
:107020002046F9F7B9FF98B1237D1BB1FF21204617
:10703000F9F7DEFF154904A808F008FE04A9144872
:10704000F9F774FE04A808F0BCFD1148F9F7F2FE48
:107050000748F9F7DBFF1049064808F021F9054811
:1070600008F02EF9CBE700BF69030020E27B0100A6
:1070700058040020B8030020F88801009007002081
:1070800034040020FD7B0100880300201A890100E0
:1070900040040020097C01001C7C010008B5FFF7BA
:1070A0006FFF28B9034BF6221A704FF4FA7008BD2F
:1070B000C820FCE7DC0300202DE9F041C0B000212E
:1070C0001C2214A813910BF05CFA202213A99B48F0
:1070D000F9F76EFB78B92022994913A80CF025FA2C
:1070E0009849994808F0DCF813A9974808F0E1F8A6
:1070F000954808F0E5F8914D6A7D2B7C04922A7D35
:107100000392EA7C0292AA7C01926A7C009240215E
:107110008E4A1BA80CF0D0F88D498B4808F0C0F8B7
:1071200013A9894808F0C5F81BA9874808F0C1F8D9
:10713000854808F0C5F84FF47A730022CDE90F2393
:10714000844A0E922BAC08228DF84820ADF84A30C4
:1071500013AA50230EA9204605F0AAFE4FF47A6325
:107160007D497E483B9308F09BF802F004FB0A221D
:1071700001467A4808F009F9784808F0A1F8204655
:1071800005F0C5FE1BA9204605F0E8FF7449064638
:107190000AA808F05BFD294607A8F9F783FD079ABE
:1071A0000A99204605F0B8FE07A808F00AFD0AA8CB
:1071B00008F007FD204605F0CEFF002E40F0B68017
:1071C000204605F0D9FFDFF8DC810646204606F0B0
:1071D00045F9074600B3214607A806F043F84146A3
:1071E0000AA808F033FD0AA907A808F0D8FD074649
:1071F0000AA808F0E6FC07A808F0E3FC002FE5D099
:1072000021460AA806F048F80AA92846F9F78EFD93
:107210000AA808F0D6FCD9E752494B4808F040F8D4
:107220000A223146484808F0A4F8474808F048F8D0
:10723000C82E6FD14C4B4D490A9348480C944FF0DF
:10724000FF330D930B9708F02BF802F094FA0A2203
:1072500001464248464D08F098F8404808F030F89A
:10726000FFF78EFD43493D4808F01AF83B4808F007
:1072700027F83E49394808F013F802F07CFA0A2250
:107280000146364808F081F8344808F019F80AA990
:10729000394806F0A7FC2860204605F02DFE2C6832
:1072A000C4B93649364807F0FBFF364907A808F04D
:1072B000CDFC07A92148F9F739FD07A808F081FCA2
:1072C0002646314B2B933DA808F07BFC304640B05E
:1072D000BDE8F0812D49214807F0E2FF02F04BFAAA
:1072E0000A2201461D4808F050F81C4807F0E8FF44
:1072F000FFF71CFA2649144807F0D2FF254B1B78EC
:10730000002BDED00D48F9F762FC0028D9D0FEF73B
:10731000F3F8D6E7B6F5987F0CBF1F491F49184808
:1073200007F0BEFF204605F0E7FDCAE71C491448F8
:1073300007F0B6FF4FF0FF36C3E700BF4004002060
:10734000A2810100657A0100B8030020837A010060
:10735000B27A010058870100C67A01006C03002050
:10736000DC7A0100EF7A0100F8880100377B010028
:1073700034040020027B010090070020187B0100EC
:10738000880300201A890100648801002F7B010016
:107390003D7B010068030020447B0100587B010015
:1073A000727B0100EA7A0100012838B50C4630DD15
:1073B0004D682F4928460CF022F828B901212D48A4
:1073C000F9F72BFCC82038BD2B4928460CF017F8DC
:1073D00001460028F3D02949294807F061FF2548D4
:1073E000F9F711FC0A220146254807F0C2FF24489C
:1073F00007F066FF61681F48F9F700FA61682048E6
:1074000007F057FF1F491E4807F04AFF1C4807F0C6
:1074100057FF1D4C94F90030012B1FDDFFF74CFE88
:10742000C82802D104232370CDE7431C10D117498B
:10743000174807F035FF164807F042FF154B16486E
:1074400000221A700323237003F020FDC920BAE73D
:10745000124B1B78002BE5D10F23E4E710491148AC
:1074600007F01EFF0F4807F02BFF4FF4FA70AAE752
:10747000DC81010040040020DF810100BD760100B5
:10748000B8030020DD760100DC030020E476010073
:107490006C0300206A030020A00300206803002082
:1074A000FF760100880300202DE9F3470024324DC8
:1074B00000942246214623463048314FDFF800A190
:1074C00007F0A6FE28464FF47A762E4B6C60AE602D
:1074D00040F8143B4FF0080807F092FE85F8208032
:1074E0002946294D0122384607F0C0FD4FF0010919
:1074F00000943B4629460722244802F00FF83B46F9
:107500002946CDF800900322214802F007F80094A4
:107510003B4606221F4F20482946204D01F0FEFF22
:107520004FF48053C5E901462B611D491D4B2B606B
:10753000381D85F8204008F089FB3D601A4D1B4935
:107540005246384608F080FFC5E90146184C194BF1
:1075500019482B60494685F810806E8201F090FF33
:107560002946204607F07CFA14495246204602B0CC
:10757000BDE8F04708F068BFBC04002050030020BD
:1075800098040020B4870100EC0700206C03002061
:107590008803002040040020B80300205804002085
:1075A0001A8901008C700100A00300204D530000D7
:1075B000E40300205887010038040020B5E00000F3
:1075C000000000202DE9F0470024C8B03C222146ED
:1075D00009A808940AF0D5FF7C22214629A82894FE
:1075E0000AF0CFFF23460122402108A802F03CF90F
:1075F000AF49B04EB04F08A80BF01FFF7F22AF4934
:1076000028A80BF092FF012328AA08A9AC4807F08C
:10761000F8F823460122402108A802F025F9A949DB
:1076200008A80BF00AFF7F22A74928A80BF07DFFCE
:10763000A64928A80BF001FF012328AA08A9A04801
:1076400007F0DFF823460122402108A802F00CF9D8
:107650009F4908A80BF0F1FE7F229E4928A80BF055
:1076600064FF012328AA08A9954807F0CAF8234611
:107670000122402108A802F0F7F8974908A80BF06A
:10768000DCFE7F22954928A80BF04FFF012328AA92
:1076900008A98B4807F0B5F833783D6801335BB231
:1076A0003370002D00F03B818D4BDFF86092B3F812
:1076B0000080ADF800801E2221460DF102000AF084
:1076C00060FF3E2221460DF16200ADF86080DFF8D8
:1076D00040A2DFF840820AF054FFED683B68002BBF
:1076E00000F0AE80002D00F0AB802B7C03F00F0388
:1076F000052B40F08E802946404606F040FB0028CE
:1077000000F0878028680BF0E2FE01340444002278
:107710002946404606F03BFB4369112B12D8DFE8AF
:1077200003F07C87877C7C097C7C7C7C11111111A7
:10773000111111871F226B4968460BF0F6FE0023DA
:107740008DF8603000230122402108A802F08CF857
:107750003F22296808A80BF0C2FE494608A80BF092
:107760006CFE514608A80BF068FE01235E4A54489F
:1077700008A907F0ABF800230122402108A802F075
:1077800073F83F22296808A80BF0A9FE494608A80B
:107790000BF053FE554908A80BF04FFE0123544A45
:1077A000474808A907F092F800230122402108A8C1
:1077B00002F05AF83F22296808A80BF090FE4D49C4
:1077C00008A80BF03AFE514608A80BF036FE01233C
:1077D0006A4608A93A4807F014F89DF86030C3B12A
:1077E00000230122402108A802F03EF83F22296828
:1077F00008A80BF074FE3F4908A80BF01EFE3B4999
:1078000008A80BF01AFE012318AA08A92C4806F0B4
:10781000F8FF08F097FB6D6860E71F22364968465D
:107820000BF083FE35493F2218A80BF07EFE89E756
:107830001F22334968460BF078FE3F223149F3E7B7
:1078400000230122402108A802F00EF82E49DFF89B
:10785000C4901B4D08A80BF0F0FD0123621E08A97F
:10786000174807F048F83B68DC683B68002B53D0AA
:10787000002C51D0237C03F00F03052B14D121469B
:10788000484606F07CFA78B1D4F8008040460BF008
:107890001EFE41460246284606F0FDFB63681BB10A
:1078A0002C21284606F0EAFB08F04CFB6468DCE774
:1078B0001A82010069030020D8030020148201000D
:1078C000E4030020F48101005382010040820100A2
:1078D000218201008C810100068201008681010065
:1078E0004775010000820100EF810100288201003C
:1078F000AE810100B7760100E78101009C810100A3
:10790000FA810100E38101000D820100B1760100DE
:107910007381010090070020044806F0A4FC33782E
:10792000013B5BB2337048B0BDE8F087E403002050
:1079300030B5A24C94F900300B3393B01A2B2BD8EE
:10794000DFE813F0EE00DE002A002A002A002A00F9
:107950002A002A002A002A002A001B0042004500B3
:107960004E008C00A900CE002A002A002A002A001E
:107970002A00FE000B0120011A01914B91481B784F
:10798000002B14BF0921012101F07BFD03F0CAF88F
:10799000022801D0FEF7AAFA94F90030012B40F337
:1079A0003E8103F0C9F8054603F0BCF8022800F058
:1079B0002D81681E042800F23281DFE810F03401C6
:1079C000360144014601270102232370E4E77E4D7E
:1079D0002B781BB9FEF75AF801232B700323F4E729
:1079E000774D78482B78002B14BF0B21032101F031
:1079F00048FD764B1B78002B40F029817448F9F73D
:107A000002F9E8B1734B1B78C3B9FFF755FBC828DF
:107A100001D10423D9E72B783BB16F496F4807F0B8
:107A20003FFC6E4807F04CFCF3E701A803F0C8F8F0
:107A3000029B002B00F0C0800F23C6E76849EDE7EA
:107A40002B784BB1042367496448237007F028FC66
:107A5000624807F035FC9FE70F23F4E7584B59487D
:107A60001B78002B14BF0B21032101F00AFD5E4B94
:107A7000196841B95D49594807F012FC574807F0A9
:107A80001FFC0723A1E75A4806F079F90128F1D92C
:107A9000FEF794F880E7574B1D6808F0FDF90023C6
:107AA00001464FF4FA52284601F072FF00283FF4D5
:107AB00073AF00230322412101A801F0D5FE4E49F6
:107AC00001A80BF0BAFC01A94C4806F07AFFFFF7B9
:107AD00079FD06234A494148237007F0E1FB5BE743
:107AE000374B38481B78002B14BF0A21022101F0C4
:107AF000C8FC424806F028FC00287FF44DAF88E718
:107B000008F0CAF93B4B1860F52323702C4B2D4825
:107B10001B78002B14BF0921012101F0B2FC3BE7C7
:107B2000344B1D6808F0B8F90023014641F2883251
:107B3000284601F02DFF00283FF42EAF002344E734
:107B40002E4806F001FC10B12C4806F0CAFB08F0E4
:107B5000A3F9284B18600D2337E7264B1D6808F062
:107B60009BF90023014642F21072284601F010FFF3
:107B700000287FF44EAF0FE708F08EF91D4B186018
:107B80000E2322E71B4B1D6808F086F900230146EF
:107B900041F28832284601F0FBFE00283FF4FCAE9B
:107BA0001849194807F07CFB174807F089FBFFF7D5
:107BB000E7F900287FF42DAFF62306E7DC03002069
:107BC0006803002038040020D0030020690300204F
:107BD000400400206A030020B67F0100B8030020A3
:107BE000DD7F0100ED7F0100E00300202780010020
:107BF00090070020840400206D7F0100E403002032
:107C00003A800100518001006C03002011491248A4
:107C100007F046FB104807F053FBF623237094F956
:107C2000000013B030BD0D49F1E70D490D4807F0D4
:107C300037FB01A802F0C4FF01A801F0EFFD0948DD
:107C400007F03EFBEBE70849E1E70849EEE70320D0
:107C5000E7E700BF6E800100880300207780010005
:107C60008B800100B8030020A8800100BB800100C8
:107C700008B5164801F007FC08F064F906F0E0F9D1
:107C8000FFF756FE022802DD114806F085FC08F0D9
:107C900059F9104B1B7823B10F4B1B680BB101F046
:107CA00071FB0E4B1B6853B10D4B93F90030052B44
:107CB00001D0FEF79BFE08F045F9FEF74DFF08F0F6
:107CC00041F90220BDE80840FEF748BC3804002016
:107CD000E40300202C04002028040020D803002006
:107CE000DC03002008B519484FF4E13107F0F0FD3E
:107CF0001748F8F763FC30B91649144807F0E6FA5C
:107D00001348F9F751F81248F8F7BCFF124B1870F6
:107D10000F48F8F7BFFF114B1870FEF7B1FBFEF7E5
:107D20005DFAFEF78DFB142008F0EAF80C4801F02C
:107D30008FFB0C490C4806F076FE4FF4FA7008F001
:107D4000DFF8BDE80840FFF71BB900BFEC070020D3
:107D50004004002067750100050000200600002097
:107D6000A966000061570000E403002007B5002366
:107D700000931A461946034807F04AFA03B05DF823
:107D800004FB00BFE004002007B5002300931A465F
:107D90001946034807F03CFA03B05DF804FB00BF46
:107DA000E804002001207047014B1868704700BFAD
:107DB000F8040020032070477047000010B5044607
:107DC0000B490C4807F08CFAA17C94F9080008F0E4
:107DD0007BFAA17C94F9090008F076FA606800212A
:107DE000FAF7F4FB044B00221A60012010BD00BF1B
:107DF000A18201006C030020F804002073B56E46D8
:107E00000546304686E80600FCF7FEFC0446304690
:107E1000FCF794FA10B1002C08BF01244FF4005174
:107E20006868FAF793FA012C1BD0022C04D0FCB935
:107E30001C491D4807F034FA3046FCF790FA70B33D
:107E40006868FAF7ABFB18B90124204602B070BD90
:107E500000206C6801F01AFF01462046FAF7B6FBD5
:107E6000F2E73046FCF71AFC01280AD0022808D0B5
:107E70000E490D4807F014FA0B4807F021FA0024C8
:107E8000E3E76868FAF78AFB0028DDD000206D6818
:107E900001F0FCFE01462846FAF798FBD5E70446B8
:107EA000D3E700BF5D8201006C0300206E820100F9
:107EB00010B5044608F08AF8204610BD2DE9F043BD
:107EC000012985B0044600F0B8804FF400514068A5
:107ED000FAF724FA002800F0B0804FF4804160687F
:107EE000FAF71CFA68B98E4D95F90030002B00F0B6
:107EF000A4804FF480416068FAF728FA2B78013BA0
:107F00002B706068FAF74AFB00221146814602A8EE
:107F1000FCF796F84FF40072616802A8FCF782FC47
:107F2000002102A8FCF74EFB80466068FAF7BEF914
:107F3000022801D0052801D14FF0000894F90A0069
:107F4000A0F10E03DBB2072B00F2CF8008F09EF801
:107F5000FF25E289218A00950023074607F027FEC6
:107F6000061EC0F2BE80AE4200F3BD80B9F1000F24
:107F700040F0C180A8EB060507E06A496A4807F0AF
:107F80008FF9694807F09CF900256849664807F0B1
:107F900087F90A2294F90A10634807F0EAF964495C
:107FA000614807F07DF90A2239465F4807F0E1F998
:107FB00060495D4807F074F90A2231465A4807F0D3
:107FC000D8F95D49584807F06BF90A2241465648EE
:107FD00007F0CFF95949544807F062F90A222946B7
:107FE000514807F0C6F9504807F06AF915F10A0F31
:107FF0002CDA94F90900A17C08F066F96068FAF7B8
:10800000CDFA30B9666801F041FE01463046FAF714
:10801000DDFAA37C6842A3B100210091FF2319225D
:1080200007F0C5FDFF280146A8BFFF21462994F9A6
:108030000800B8BF462108F0CDF8002005B0BDE823
:10804000F083FF22009219461922E9E70A2D27DD65
:1080500094F90800A17C08F037F96068FAF79EFAF5
:1080600030B9666801F012FE01463046FAF7AEFA02
:10807000A37C83B100210091FF233322284607F01F
:1080800096FDFF280146A8BFFF214629B8BF46211B
:1080900094F90900CFE7FF22009219463322EDE759
:1080A0002749214807F01CF9A17C94F9080008F041
:1080B0000BF9A17C94F9090008F006F90021606829
:1080C000FAF784FA4FF400516068FAF77DF94FF43B
:1080D00080416068FAF778F9114A13780133137018
:1080E000ABE7002642E72E4640E74FF0FF37B9F1F5
:1080F000000F0FD03E4607F0CFFE00230146B4F933
:108100000C20484601F044FC00287FF436AF731C75
:108110007FF430AFA8F17F054FF0FF3635E700BFA1
:10812000040000207A8201006C0300208882010094
:108130008C820100C47A0100C670010092820100A5
:108140009A820100002110B5044681744068FAF754
:1081500051F943B2002BBBBF40422072237201236E
:10816000B8BFA374237A6068013B182B84BF202317
:1081700023720121FAF73EF943B2002BBBBF404204
:10818000607263720123B8BFA374637A6068013BB5
:10819000182B84BF212363720221FAF72BF9C3B293
:1081A000192B8ABF0023A072A37203216068FAF71B
:1081B00021F980B2431EB3F5806F26BF0023E3810F
:1081C000E08104216068FAF715F980B2B0F5806F9C
:1081D0008ABF4FF480632082238205216068FAF70A
:1081E00009F900B20028D6BF42F21073A081A38122
:1081F00010BD000010B50446F8F7E6F82046FFF77A
:10820000A1FF1849184807F06BF894F908000121FC
:1082100008F032F894F90900012108F02DF8A17C4A
:1082200094F9080008F050F8A17C94F9090008F0CE
:108230004BF894F90A00002108F01EF8606800214C
:10824000FAF7C4F960684FF40051FAF7BDF86068B6
:108250004FF48041FAF7B8F8044B01201860044B42
:10826000187010BDAF8201006C030020F8040020DC
:108270000400002007B5002300931A46194603485E
:1082800006F0C6FF03B05DF804FB00BFF004002059
:1082900001207047014B1868704700BF040500209B
:1082A000002070470320704770470000F8B504466F
:1082B000F8F78AF8A468002C3CD0E468224E234DDD
:1082C000234F64B3236843B31B7833B3324621464C
:1082D000284605F064FD30B94FF0FF3332462146A1
:1082E000284605F0A0FD3A462146284605F057FDF0
:1082F00030B94FF0FF333A462146284605F093FD4A
:10830000144A2146284605F04AFD30B94FF0FF33A4
:10831000104A2146284605F086FD6468D1E70E49DB
:108320000E4806F0BDFF0D4806F0CAFF0C4B0120B9
:108330001860F8BD0B49094806F0B2FF074806F07F
:10834000BFFF2046F5E700BF6F83010090070020C4
:108350007682010084820100738301006C03002097
:10836000040500208283010010B5064C0649204612
:1083700006F096FF204606F0A3FF044B00221A6089
:10838000012010BD6C0300205D8301000405002066
:108390002DE9F04F91B008AC8046204684E80600F5
:1083A0000693FCF731FA83462046FBF7C7FF20B15E
:1083B000BBF1000F08BF4FF0010B2046FBF7BEFFDB
:1083C00090B12046FCF720FA07280DD12046FCF793
:1083D00065F9112869D0122869D0102804D1FF222C
:1083E00021460EA8FCF769F9D8F80850002D00F0D6
:1083F0004B814FF00009EC68CDF80C90CA464D4611
:10840000CDF80890002C00F0DA80A14AA14821465E
:1084100005F0C5FCA04A214606469E4805F0BFFC73
:108420009E4A074621469B4805F0B9FC0590002E60
:1084300000F08780002F00F08480337C03F00F036E
:10844000022B7ED13B7C03F00F03022B79D1944A9F
:108450009048214605F0A3FC43690493069B002B3A
:108460005AD0194620680BF004F8002854D108A807
:10847000FBF764FF00BBBBF1070F6CD008AA1046E6
:108480000792FBF76CFF079A002839D010460021AD
:108490000792FCF797F87061FDF740F9079A78B3F7
:1084A000236800934FF4007325E0802298E70A21A7
:1084B0002046FCF749F897E708A8FCF7EFF8786141
:1084C00008A8FCF7EBF801283DD0022841D07B69D1
:1084D000012B08D17369132B05DC1E22726108A9D8
:1084E0000EA8FCF7EAF8FDF719F948B123680093E4
:1084F00008AA4FF4407306CAD8F80400FAF7DAF96C
:10850000059B4BB10023CDE9003308AB0CCB4FF0FA
:10851000FF31059801F056FA7B69022B0FD0013329
:108520000DD07369049A02994B4502FB03F2114482
:10853000C4BF9946049B0291C4BF92460393049B17
:108540001D4464685EE7726908A90EA8FCF7B5F8D7
:10855000BDE70022F8E708A8FBF701FF00288DD04F
:1085600008A8FBF737FF7B69A8B1022B01D00133C4
:108570000CD14C494C4806F09CFE4B4806F0A0FE3E
:1085800001227A6108A90EA8FCF737F908A8FBF7C1
:1085900021FF7061A7E7022B0ED001330CD04349B5
:1085A000414806F086FE404806F08AFE02227A61C3
:1085B00008A90EA8FCF721F90023736193E7002DA9
:1085C00062D03B493848029B93FBF5F706F068FE02
:1085D0000A222946344806F0CCFE3649324806F0D5
:1085E0005FFEFF25029B304893FBF5F10A2206F05F
:1085F000C0FE31492C4806F053FE0A2239462A486B
:1086000006F0B7FE2D49284806F04AFE9AFBF5F120
:108610000A22254806F0ADFE2949234806F040FE0F
:108620000A220399204806F0A4FE26491E4806F0B7
:1086300037FE1D4806F044FE234AD8F808101548B6
:1086400005F0ADFB0EAE8146224621460AA8FBF797
:10865000F7FC3A460AA93046FCF72FF80CAD002F7C
:1086600014BF0122022231462846FCF7C6F8CDE9A4
:1086700000444FF0FF3195E80C00484601F0A2F9A4
:10868000D8F8083013BB0125284611B0BDE8F08F9B
:108690006F830100900700207682010000830100B3
:1086A00004830100068301006C0300201183010094
:1086B0001D830100268301003183010038830100FE
:1086C000468301004D8301001A890100DD68434F94
:1086D000DFF824B1002DD6D0414A2946384605F0AE
:1086E0005EFB5A4644692946384605F058FB3D4A28
:1086F00080462946384605F052FB3B4A81462946CA
:10870000384605F04CFBB8F1000F60D0B9F1000F0E
:108710005DD000285BD098F8102002F00F02022AEA
:1087200055D199F8102002F00F02022A4FD1027C95
:1087300002F00F02022A4AD1002C48D04269022AD4
:1087400047D0013245D0BAF1000F44D0D9F81430E7
:108750002968264803FB04F9039BC9EB092292FB15
:10876000F4F45C4306F0A5FD94FBFAF420491F489D
:1087700006F09FFD0A22FF211C4899FBF1F106F04B
:10878000F8FD1C49194806F08BFD0A2221461748BE
:1087900006F0CDFD154806F093FDD8F81430A3423D
:1087A00015D0002211460AA8FBF74AFC22460AA966
:1087B0003046FBF782FF0023CDE900334FF0FF3155
:1087C00096E80C00284601F0FDF8C8F814406D68E2
:1087D00080E70024E1E75446DFE700BF9007002070
:1087E000048301006F830100768201006C03002086
:1087F00051830100578301008482010010B50446B3
:1088000007F0E4FB204610BD0023836043683BB1C2
:108810005B682BB11A7C02F00F02062A08BF836046
:108820007047000007B5002300931A461946034815
:1088300006F0EEFC03B05DF804FB00BFFC04002072
:10884000014B1868704700BF1005002043687BB1DA
:10885000B0F90A20042A05D0052A05D0032A05D13B
:10886000022070470120704711207047187C704724
:10887000184670477047000010B504461E491F484F
:1088800006F00EFD0A22B4F908101C4806F071FD2E
:108890001B491A4806F004FD184806F011FD23682C
:1088A00020465B6B9847012805D002280AD000219A
:1088B000B4F9080019E003212046F7F759FE00211A
:1088C00007F0DAFC00212046F7F752FE002107F0FE
:1088D000D3FC01212046F7F74BFE002107F0CCFC2A
:1088E00002212046F7F744FE002107F0C5FC054BA6
:1088F00000221A60012010BDE08301006C030020FB
:10890000EA830100100500202DE9F041044688B0FB
:1089100040689DF8383002AE86E8060000286ED028
:10892000B4F90820002A69D0002B6BD00021F9F798
:1089300061FD236880465B6B2046984705B2022D97
:1089400051D0032D2BD0012D0CBF05210121002278
:1089500004A8FBF775FB4FF0FF33009396E80C007B
:1089600004A906A8FCF742F9012D3ED0022D38D10A
:108970009DF81610B4F9080007F02CFC01212046E0
:10898000F7F7F6FD9DF8151007F024FC02212046AC
:10899000F7F7EEFD9DF8141007F01CFC21E04FEAFC
:1089A000D8713046B4F90870FBF70CFE0146054655
:1089B000384607F00FFC1449144806F071FC0A22EF
:1089C000B4F90810114806F0D4FC11490F4806F01C
:1089D00067FC0A2229460D4806F0CBFC0B4806F03E
:1089E0006FFC01200BE00421B1E703212046F7F7DB
:1089F000BFFD9DF8171007F0EDFBB9E7104608B072
:108A0000BDE8F0811846FAE7087301006C03002006
:108A10004771010010B5044607F0D8FA204610BD92
:108A200038B50446F7F7D0FC2249234806F038FC55
:108A30000A22B4F90810204806F09BFC1F491E4882
:108A400006F02EFC1C4806F03BFC606870B3B4F9DD
:108A5000083063BB236820465B6B984701280546B6
:108A600005D002280AD00121B4F9080019E0032139
:108A70002046F7F77DFD294607F0FEFB0021204642
:108A8000F7F776FD012107F0F7FB01212046F7F704
:108A90006FFD012107F0F0FB02212046F7F768FD8A
:108AA000012107F0E9FB064B0120186038BD0020CA
:108AB000FCE700BFE08301006C030020FE8401009E
:108AC0001005002007B5002300931A4619460348F5
:108AD00006F09EFB03B05DF804FB00BF0805002014
:108AE000014B1868704700BF1C0500200320704729
:108AF0007047000010B50446F7F766FC184919489E
:108B000006F0CEFB0A22B4F90810164806F031FC34
:108B10001549144806F0C4FB124806F0D1FB0121A8
:108B2000B4F9080007F0A8FBB4F90800A17A07F02F
:108B3000CBFB606810B10021F9F748FD0B4B606872
:108B400001221A60FBF750F8002807DD0020646856
:108B500001F09CF801462046F9F738FD012010BDD0
:108B60006E8401006C030020FE8401001C050020BF
:108B700038B50E4C0E490546204606F091FB0A22F8
:108B8000B5F90810204606F0F4FB0A49204606F025
:108B900087FB204606F094FBB5F90800002107F09A
:108BA0006BFB054B00221A60012038BD6C030020CE
:108BB0006E840100EA8301001C05002010B5044604
:108BC00007F004FA204610BD002110B5044681725A
:108BD0004068F0B1F9F70EFC03B2002BBBBF404276
:108BE000208123810123B8BFA37223896068013BE0
:108BF000182B84BF202323810121F9F71BFC08F0E7
:108C000079FE0022054B08F0CDFE09F0A3F908B16A
:108C1000E06010BD41F28833E360FAE700408F4026
:108C200030B5044687B000232F22CDE90023ADF8EC
:108C30000830B0F90800A37A0D4600295DD083F012
:108C4000010107F041FBE368B3F57A7F53D3314963
:108C5000314806F025FB0A22B4F908102E4806F028
:108C600088FB2E492C4806F01BFB0A2229462A487D
:108C700006F07FFB284806F023FB294968460AF0E6
:108C8000DCFB6068F9F712FB002D3ED00D2838D0D0
:108C90000E2834D00B2836D1224903A80AF0F3FB62
:108CA00021491D4806F0FCFA6368196823680968C1
:108CB0005D6A03AA6B462046A8470A220146164869
:108CC00006F057FB1949144806F0EAFA636812489F
:108CD0001B68196806F0EDFA69460F4806F0E9FAD4
:108CE00013490D4806F0DCFA03A90B4806F0E1FA37
:108CF000094806F0E5FA07B030BD1946A1E70D496D
:108D0000CBE70D49C9E70D49C7E702280CBF0C495D
:108D10000C49C2E77A8401006C03002082730100D1
:108D200045840100538401007F84010058720100D2
:108D30008B8401004C840100388401005B840100B5
:108D40003C840100408401000129F7B5044644D069
:108D50004368002B41D0002211466846FBF770F9AA
:108D60004FF4007261686846FBF75CFD00216846BD
:108D7000FBF728FC05466846FBF790FC6068F9F7AE
:108D80000DFC064607F088F8E268FF216A430023DD
:108D9000B2FBF1F20146304600F0FAFD0746E6B1BB
:108DA00007F07AF800230146E268304600F0F0FD53
:108DB000064620B30020666800F068FF0146304692
:108DC000F9F704FC4DB1207A00F06AFFA37A8342E0
:108DD00003D101212046FFF723FF002003B0F0BD9F
:108DE0009FB131462046FFF71BFF6068FAF7FCFE93
:108DF00001460028F1D16068F9F7E8FBEDE7207A39
:108E000000F04EFFA37A8342EAD1002DE5D0207A0C
:108E100000F046FFA37A8342DFD1002FDDD1D8E7EF
:108E2000F7B56D4685E8060004463F493F489DF882
:108E300020601F4606F034FA2846FBF75DFE2FB18E
:108E40003B4938460AF015FB002844D060680028EA
:108E500041D02846FBF772FA00283ED12846FBF79E
:108E6000D3FC012839D011D302280ED00446314951
:108E70002E4806F015FA0A2221462C4806F079FA07
:108E80002A4806F01DFA002025E08EB10021284670
:108E9000FBF798FB00283DD06068F9F77FFBC8B965
:108EA000646800F0F3FE01462046F9F78FFB11E0FD
:108EB0006068F9F7FBF90E280CD8012303FA00F0DB
:108EC00045F60243184205D031462846FBF77AFBA7
:108ED0000028E1D1012003B0F0BD2846FBF7DEFBFE
:108EE000022817D012D80128D6D013490F4806F00F
:108EF000D7F92846FBF7D2FB0A2201460B4806F0B9
:108F000051FA0A4806F0DCF90124B0E70A380428CF
:108F1000EBD8C1E760680021F9F758FB0021204633
:108F2000FFF77EFED6E700BF638401006C030020DC
:108F300045840100DA6F0100CD6F010007B5002301
:108F400000931A461946034806F062F903B05DF82B
:108F500004FB00BF140500200139C9B2FF2906D067
:108F6000435C0139C9B2002BF8D0002070470120C2
:108F7000704700002DE9F04F85B006F08DFF634B80
:108F8000029018689A4608B101F0E4F8604C614F0D
:108F90002568386800210BB2AB4201F10101C0F233
:108FA0009D805D4DDFF88C91DAF80000002800F01C
:108FB0009C8021682B6803EBC10101F053FA002863
:108FC00040F393802368132B00F38F8006F064FF37
:108FD0000023014641F28832029800F0D9FC06468F
:108FE000002840F082802B682068072103EBC00036
:108FF00001F0A0F82B680193019A236802EBC30BE0
:109000009BF807208242CFD10FFA86F8434503939D
:1090100025DD019B082203EBC800594609F07EFAC2
:109020000136039B0028EFD13968019031F81830E0
:109030003A4843F0010321F81830394906F030F975
:109040002B682068019A03EBC000082100F082FA27
:109050003449324806F03AF9B8F1000FA4DAD9F8E9
:109060000030002BA0D022682868082100EBC20045
:10907000FFF772FF0646002896D13B68274801217A
:1090800023F81210284906F00BF90A222168234818
:1090900006F06FF92549214806F002F92B6820688F
:1090A000324603EBC000082100F054FA1B4806F0DA
:1090B00007F922682B6803EBC20113F83230282B22
:1090C00008D10C22D9F8000001F0EDFADAF800001E
:1090D00001F012F923680133236065E730F81320AB
:1090E00022F0010220F8132055E711490B4806F041
:1090F000D7F80A222168094806F03BF9074806F02C
:10910000DFF8012005B0BDE8F08F00BF2805002082
:109110003C05002044050020400500206C03002091
:1091200091850100988501009F850100A4850100BB
:109130008285010034050020F8B5424D2B680746B2
:109140000BB1012054E040494048414E06F0A8F8D8
:109150003E4806F0B5F83F493C4806F0A1F800F05B
:109160000AFB0A220146394806F00FF9374806F093
:10917000A7F8142006F026FF044600F0A5FFA02063
:109180002C6006F021FF344930603048334C06F043
:1091900087F800F0F0FA0A2201462C4806F0F5F8AC
:1091A0002A4806F08DF8282006F00EFF2C49206092
:1091B000264806F075F800F0DEFA0A220146234838
:1091C00006F0E3F8214806F07BF833680BB123681A
:1091D0007BB92449244806F063F800F0CCFA0A224F
:1091E0000146214806F0D1F81F4806F069F8002032
:1091F000F8BD1E4B1E481F6000F0CCFD286800F033
:109200007DFF0446B8B11B49104806F05FF8286896
:1092100001F0B0F8286800F07DFF17490B4806F010
:1092200055F8286801F0EAF800288AD01349074861
:1092300006F04CF885E71249044806F047F8204646
:10924000D6E700BF28050020E38401006C0300205E
:1092500040050020377B0100048501004405002003
:10926000108501001D850100880300202C050020C9
:10927000B40500203585010048850100688501009E
:10928000748501002DE9F041364E306800F02EFF64
:1092900002280DD13449354806F002F8334806F06B
:1092A0000FF8306801F0AAF842F21070BDE8F081C2
:1092B0002F4C304F2568EDB91C2006F083FE316835
:1092C0002D4E804601F052F94046C4F8008001F06E
:1092D0002DFA3A6820682BB2934205F1010506DAAF
:1092E00031680C2201EBC30101F0DDF9F1E7002147
:1092F00001F05AFA214E3A68B6F9003093423746E7
:1093000006DBFFF737FE002333804FF4FA50CDE73A
:10931000194D286800EBC30110F8330028281AD132
:10932000206801F0D1FA164B1B6802462BB1B6F942
:109330000000296801EBC00198472B68B7F90010BD
:10934000206803EBC10101F065FA3B8801333B80E3
:1093500040F6C410AAE701334FF4FA60338090FB63
:10936000F2F0A3E728050020D48401006C0300205C
:10937000340500203C050020400500203805002071
:109380002C05002038B5094C256806F085FD002322
:10939000014641F28832284600F0FAFA20B1FFF780
:1093A00071FF06F079FD206038BD00BF3005002058
:1093B0002DE9F0411F4C2049204D0746204805F07B
:1093C0006FFF0A2221681E4805F0D3FF1D491C4883
:1093D00005F066FF2B682068002203EBC00008211F
:1093E00000F0B8F8164805F06BFF2268132A1FDC5E
:1093F000D5F8008008EBC20608213046FFF7ACFD27
:10940000B0B9114B1B68012123F812103B6848F8D2
:1094100032307B68736022682B6813F83230282B57
:1094200003D10A4B186800F067FF236801332360FB
:10943000BDE8F0813C0500209F850100400500202B
:10944000B8030020A4850100440500202805002061
:10945000034B0146186808B100F046BE704700BFD4
:109460002805002007B5002300931A461946034833
:1094700005F0CEFE03B05DF804FB00BF2005002020
:10948000704770477047704707B5002300931A462E
:109490001946034805F0BCFE03B05DF804FB00BFAD
:1094A00048050020184B1B7870B504460D469BB14B
:1094B000164B027A1B789A420ED8154A0A2913686D
:1094C000164616D1134A0021D154406910B1217AB1
:1094D00005F064FE00233360E06898B10E4B227AF9
:1094E0001B789A420ED8036829461B68BDE8704075
:1094F00018474E2BF0DC0D291FBF591C1160054A7F
:10950000D554E9E7012070BD7C040020060000204E
:10951000A8050020580500200500002030B50025D2
:1095200045604361034D9DF80C300560C1600272D7
:10953000037430BDB485010007B5002300931A46BB
:109540001946034805F064FE03B05DF804FB00BF54
:1095500050050020F8B5441E0D4D16466718BC4254
:109560000ED014F8011F10220909284605F0DFFE6D
:109570002178102201F00F01284605F0D8FEEEE711
:1095800026B10348BDE8F84005F09ABEF8BD00BF1B
:10959000B803002070B501380C4D13464618B04290
:1095A00003F102030CD010F8014F24112C5D03F8D5
:1095B000024C047804F00F042C5D03F8014CEEE734
:1095C00009B2002302F8113070BD00BF0786010008
:1095D000A0F16103052B02D85738C0B27047A0F143
:1095E0004103052B01D83738F7E73038C0B20A28D5
:1095F00028BF0020704738B50139841C00F11205DE
:1096000014F8020CFFF7E4FF0001C2B201F8012FC9
:1096100014F8010CFFF7DCFF02341043AC42087071
:10962000EED138BD38B50546D8B10468ACB1247860
:109630009CB1286803783BB12D2B05D0303B092B1A
:1096400002D901302860F4E708F015FD2C2104460A
:10965000286809F001FF10B92860204638BD0130A4
:10966000FAE70446F9E72DE9F7430E460022062102
:109670000746FAF7E5FC002E55D03368002B52D090
:109680001B78002B4FD0D6F8008098F800404CB3E0
:109690002D2C6CD0303C092C03D908F10103336028
:1096A000F1E74146002400220FFA82F9013211F855
:1096B0000930303B092BF7D92E21404609F0CCFE6A
:1096C00018B3002211B2431801325B78303B092BEA
:1096D000F8D94378A3F13002092A01D82F2B03D8F7
:1096E000002204E0A146E7E7392B88BF09220A25BA
:1096F00055438278A2F13003092B05D82F2A16D9B9
:10970000392A88BF09231D4499B9404608F0B7FC9F
:10971000394602466846FAF7E4FF2C21306809F022
:109720009BFE10BB3060384603B0BDE8F0830023D9
:10973000E9E7022940460EDCB9F1070F0BDC08F01F
:109740009EFC6422424304B16D422A443946684675
:10975000FAF7EDFFE1E708F08BFC08F01BFC394657
:1097600002466846FAF7C9FFD7E70130DAE708F1A1
:109770000101012497E708B500200AF0B5FEADEB22
:10978000000008BD704730B5441E224612F8013F64
:10979000002BFBD11A460A2514F8010F70B1032AD9
:1097A00014DC2E2806D1FF2B10DC8818013203713F
:1097B0000023F1E7303805FB0303EDE7FF2B04DC62
:1097C000032A02DC114401200B7130BD0020FCE7AC
:1097D0002DE9F3410024DFF840800C700D46174658
:1097E000061D0A2201A916F8010B08F061FE3A468F
:1097F00001A9284609F073FE032C04D03A464146DD
:10980000284609F06CFE0134A3B2042B1CB2E8D147
:10981000284602B0BDE8F0810D8101002DE9F0413C
:109820000E4D0F4FDFF83C8006460024032C0ED06F
:1098300033190A221979284605F079FD4146284650
:10984000013405F02DFD042CF0D1BDE8F081F17953
:109850000A22284605F06BFD3946F0E7B8030020E0
:10986000687101000D8101002DE9F047DFF8F0A0DB
:10987000DAF8005004460E4617469946002D49D0A6
:109880002B7C03F00F03062B43D12C4A2C4829468E
:1098900004F085FA022F804637D0032F37D1294AAA
:1098A000DAF80010264804F07AFA0546B8F1000FFD
:1098B00030D098F8103003F00F03042B2AD1D8F8D9
:1098C00014103246204609F030FE32461E4920462A
:1098D00009F005FE0DB32B7C03F00F03042B1CD104
:1098E00069693246204609F0FAFD3246164920469B
:1098F00009F0F5FDB9F1000F04D032464946204683
:1099000009F0EDFD2046BDE8F087104AC8E70025C4
:10991000CCE7002532460E49D4E7022F0AD0032FA8
:1099200005D0012FE1D10B4B32461968DAE73246F8
:109930000949D7E732460949D4E700BFFD85010050
:109940009007002084820100C47A01000286010091
:1099500021860100840300201B8601001886010077
:10996000940400200B460A220146184606F0EBBA82
:1099700010B5054C0549204605F09BFC2046BDE886
:10998000104005F09DBC00BF6C030020ED85010078
:1099900010B54AB102441BB1B2FBF3F403FB14222D
:1099A0008A4208D288420AD9012010BD884294BF59
:1099B00000200120F9E78242F8D80020F5E7824232
:1099C000F5E700002DE9F04F99B00DF108090C46BC
:1099D00089E80C00DDE922AB0646002800F0C880CB
:1099E000037C03F00F03062B19D8DFE803F0BC1843
:1099F0001818B8041A00954BC5681A7801321A7005
:109A00001E464DB1CDE900AB284699E80C00214631
:109A1000FFF7D8FF6D68F4E73378013B337000201F
:109A20000EE001468A4A8B4804F0B9F9054650B168
:109A30000023CDE90033214699E80C00FFF7C2FF6F
:109A400019B0BDE8F08F844A8248314604F0A7F986
:109A5000824A804631467F4804F0A1F907461CB18E
:109A6000012C62D02C460CE07D4A7A48314604F045
:109A700096F905467B4A7748314604F090F904464A
:109A800005B93546002C08BF3446B8F1000F6DD03B
:109A9000002F08BF5F4635B12B7C03F00F03042B6A
:109AA0000CBF6D690025002C65D0237C03F00F03EB
:109AB000042B60D16469B8F1000F7FD0002D66D00F
:109AC00069496A4805F0ECFBD8F81410674805F0BE
:109AD000F0FB6749654805F0E3FB2946634805F05C
:109AE000E8FB624805F0ECFB4846FBF705F8002F61
:109AF00040F0A48098F8103003F00F03042B40F0DE
:109B00009B80D8F8141008A8F8F762FE08A8F8F7A8
:109B10009DFD30B1002D48D00022294608A8F9F754
:109B2000A5FE08A8F8F7B8FB86E0524A4948314636
:109B300004F035F9504A05463146464804F02FF9FD
:109B40000446002D7DD1464A4248314604F027F9AB
:109B50000546002C8ED0002808BF354695E7002426
:109B60002746A0468DE7002425462746D0468FE7A6
:109B70005F46D04605460023102200930DEB0201FC
:109B80004FF440734846FAF7A3FE044693E73B4977
:109B9000364805F085FBD8F81410344805F089FBE9
:109BA0003349324805F07CFB9EE70123009399E896
:109BB00006002B4608A8F9F7A5F8B2E7002F3BD01E
:109BC000002C39D03B7C03F00F03042B30D12C49FF
:109BD000264805F065FB7969244805F06AFB2449AD
:109BE000224805F05DFB2146204805F062FB1F4836
:109BF00005F066FB4022796908A809F096FC214827
:109C000004F0A2FBA0B1204B93F9003083B92F21BF
:109C100008A809F021FC28B97B690322402108A883
:109C2000FFF722FE0123224608A9164804F0E9FDA9
:109C3000B8F1000F7FF45EAF012001E7002CC1D125
:109C400058E700287FF421AF14E700BF6903002024
:109C50001B71010090070020127101005471010076
:109C6000BC850100C1850100D08501006C03002086
:109C7000D7850100C6850100CB850100DC85010088
:109C8000E6850100E4030020B403002010B504467B
:109C900006F002F9E040431E033388BF012010BDE7
:109CA000054B1A68054B53F8201001238B401342D3
:109CB00014BF01200020704708050050548901009E
:109CC00007B5002300931A461946034805F0A0FA89
:109CD00003B05DF804FB00BFAC0500202DE9F8439C
:109CE00080460D46174601EB02090C464C45A4EB95
:109CF00005060BD0D8F8003014F8011B1B6840464D
:109D000098470028F2D13046BDE8F8833E46FAE78E
:109D10007047203005F02DBC203005F01CBC2030F1
:109D200005F02DBC38B5437F0D460BB9002038BD7A
:109D300000F16804204605F02AFC0028F6D12046F0
:109D4000294605F0F9FB0120F1E700002DE9F0417B
:109D50001E4600254FF47A73C0E901530C4B0446AC
:109D600040F8203B8846174605F0DDFB04F168000B
:109D700005F0D9FB9DF8183063769DF81C302676E7
:109D8000C4E90487A37665772046BDE8F08100BF6B
:109D900030860100817E284A0123C37670B552F8CF
:109DA0002140417E52F821104FF0A04504F5E074A7
:109DB00001F5E07140F20C6645F8246045F8216039
:109DC00001694FF0CC74C1F8244501690624C1F83B
:109DD0000045847E016952F82440C1F80845447E5C
:109DE000016952F82420C1F80C2590F91820510976
:109DF00002F01F0293406031104A42F8213090F97E
:109E00001830002BBDBF03F00F0302F6FC32D2184E
:109E10009B18B5BF40234022137683F8002390F9A6
:109E200018300122590903F01F0302FA03F3034A11
:109E300042F8213070BD00BF5489010000E100E00C
:109E40002DE9F041044688461F461546002A50D0A9
:109E500000F12006304605F07AFB2369C3F88885B7
:109E6000236901221A622369C3F834652369C3F8A0
:109E7000385523691A602269D2F84C311BB9D2F8DF
:109E80002431002BF8D00023C2F84C312269D2F8DB
:109E90005C311BB9D2F82431002BF8D00023C2F872
:109EA0005C3122696FB9D2F8243153B90123D361EF
:109EB0002369D3F84821002AFBD00022C3F84821A7
:109EC00009E0012353612369D3F80421002AFBD060
:109ED0000022C3F804212369D3F8242112B10022FF
:109EE000C3F824212369D3F83C052066C0B2BDE83D
:109EF000F0811046FBE70123FFF7A2BF10B504462F
:109F000080F8B010683005F022FB0123637710BDA4
:109F1000F8B500234377036990F8B020C3F888258B
:109F2000036901261E62036900F168050446C3F84F
:109F3000445528460F4605F01CFB2369C3F8480525
:109F400023699E602369D3F850211AB9D3F82421DC
:109F5000002AF8D00022C3F85021284605F009FB5A
:109F6000236930B1D3F860211AB9D3F82421002A2B
:109F7000F8D00022C3F8602123696FB9D3F82421F7
:109F800052B90122DA612369D3F84821002AFBD0B3
:109F90000022C3F8482109E001225A612369D3F85D
:109FA0000421002AFBD00022C3F804212369D3F83E
:109FB000240168B10022C3F824212369D3F8C40422
:109FC000C3F8C404022803D004280CBF03200420D3
:109FD000F8BD0121FFF79CBF70B54369D3F8642138
:109FE000044692B10022012500F12006C3F8642145
:109FF0000577304605F0ABFA6369C3F834656369E9
:10A000004022C3F8382563691D636369D3F868216A
:10A01000DAB10025C3F8685104F1680601236377BB
:10A020002577304605F093FAD4F8B43003B1984759
:10A03000636965773046C3F8446505F09AFA636949
:10A04000C3F84805636901225A636369D3F80421A0
:10A0500062B10022C3F80421237F3BB16369D3F8C6
:10A060003C05D4F8B830206603B198476369D3F84B
:10A07000242152B10022C3F824216369D3F8D024EB
:10A08000C3F8D024636901225A6170BD0148FFF70B
:10A09000A3BF00BFB405002007B516231722CDE9E2
:10A0A00000324FF04022042311460348FFF74EFED2
:10A0B00003B05DF804FB00BFB40500200148FFF7C2
:10A0C00088BF00BFB405002010B54FF4C053038013
:10A0D00000230446837003610248FFF75BFE2046BD
:10A0E00010BD00BFB4050020016170478078704743
:10A0F00041780148FFF702BFB405002008B5FFF71B
:10A10000F7FF0348FFF765FFB0FA80F0400908BD8C
:10A11000B4050020012303707047FF23C37200239E
:10A120000373C370037143718371C371037243720C
:10A130008372704710B5064A01440023884204D058
:10A1400010F8014B6340D35CF8E7184610BD00BF20
:10A1500048860100FFF7E1BF38B5084C0D46FFF710
:10A16000C7FFE1212046FFF7DDFD29462046FFF726
:10A17000D9FDBDE83840FFF7A1BF00BFB4050020FE
:10A1800010B5054C417801222046FFF7B4FE204669
:10A19000FFF7C2FDC0B210BDB405002010B5F0211C
:10A1A0000446FFF7D9FF2046BDE81040FFF7E8BF9F
:10A1B00070B5054605F070FE002400F57A7605F0CE
:10A1C0006BFEB04246D22846FFF7E8FFC3070446BD
:10A1D00042D52B6903B198471420013800BF00BF56
:10A1E00000BF00BF00BF00BF00BF00BF00BF00BF77
:10A1F00000BF00BF00BF00BF00BF00BF00BF00BF67
:10A2000000BF00BF00BF00BF00BF00BF00BF00BF56
:10A2100000BF00BF00BF00BF00BF00BF00BF00BF46
:10A2200000BF00BF00BF00BF00BF00BF00BF00BF36
:10A2300000BF00BF00BF00BF00BF00BF00BF00BF26
:10A2400000BF00BF00BF00BF00BF00BF00BF00BF16
:10A25000C3D1B4E70123AB70204670BD10B5E12136
:10A260000446FFF779FF2046BDE81040FFF788BF9E
:10A2700010B50446FFF79CFF2046FFF739FF9621F3
:10A280000648FFF74FFDFFF719FF2046FFF790FF45
:10A290002046BDE81040FFF7E1BF00BFB405002035
:10A2A000FFF7E6BF10B5C3210446FFF755FF204670
:10A2B000BDE81040FFF764BF38B504460D46FFF710
:10A2C00077FF2046FFF714FFD2210A48FFF72AFD47
:10A2D000E94345EA0111C9B20648FFF723FDFFF73C
:10A2E000EDFE2046FFF74CFFA8421CBF0423A370DD
:10A2F00038BD00BFB405002010B50446FFF7D2FFFB
:10A3000040F00401C9B22046BDE81040FFF7D4BFB9
:10A3100070B5164604460D46FFF74AFF16B12046B3
:10A32000FFF7EAFF2046FFF7E3FEA5210548FFF708
:10A33000F9FC29460348FFF7F5FCBDE87040FFF73C
:10A34000BDBE00BFB405002070B500220C465521EB
:10A350000646FFF7DDFF651E073415F8011F0022D2
:10A360003046FFF7D5FFA542F7D170BDFFF7ECBF30
:10A37000FFF7CEBF10B50446FFF7BAFE2046002215
:10A38000F021FFF7C5FFBDE81040FFF797BE0000C2
:10A3900070B5164605460C46FFF70AFF16B128466B
:10A3A000FFF7AAFF2846FFF7A3FE87210648FFF71D
:10A3B000B9FC002C0CBF214680210348FFF7B2FCFA
:10A3C000BDE87040FFF77ABEB405002010B500224A
:10A3D00004460121FFF7DCFF2046FFF7E9FEC0F34A
:10A3E000401010BDFFF7F2BF10B50446FFF75AFF4B
:10A3F00020460021BDE81040FFF75EBF38B5044697
:10A40000FFF7D6FEC30729D42046FFF7EDFF20460D
:10A41000FFF7CEFE2046FFF76BFEB4211048FFF792
:10A4200081FCFFF74BFE2046FFF7C2FE10F004034D
:10A43000054602D00223A37002E0A278022AFAD0D5
:10A44000237843B12046FFF72DFF40F00101C9B248
:10A450002046FFF731FFC5F3400038BD0020FCE780
:10A46000B40500202DE9F74F057B04460F46002D6B
:10A470006BD1FFF7C3FF002869D02046FFF798FE95
:10A480002A46F0212046FFF743FFDFF8C8804FF04F
:10A49000FF394FF0010A94F90B30EEB24FEAD60BB8
:10A4A0009D4206F007060AFA06F623DA04EB0B03D0
:10A4B000DB78334020460193FFF77AFE2046FFF712
:10A4C00017FE78214046FFF72DFC019B002B0CBFA7
:10A4D000194680214046FFF725FCFFF7EFFD204697
:10A4E000FFF766FE820600F0400307D55BB16FF010
:10A4F000010027E00CBF01230023DBE71BB90306A3
:10A5000058BF4FFA85F904EB0B03010693F90320BA
:10A5100076B205F101054CBF3243B243402DDA70EB
:10A52000B9D1B9F1FF3F04BF0123237384F80B9025
:10A53000E31C013F0B3413F8012B07F8012FA34252
:10A54000F9D1012003B0BDE8F08F0020FAE74FF009
:10A55000FF30F7E7B405002008B5FFF783FF20EAD6
:10A56000E070C0B208BDFFF749BF7047054A82617D
:10A570000022027102700922427001228160827001
:10A58000C27070476BA5000010B50C46204607212D
:10A59000FFF7D0FDE3791B1A5842584110BD70B542
:10A5A000044680680E461546FFF7DDFFB8B1314618
:10A5B000A068FFF7DBFE0022BE21A068FFF7D8FEEF
:10A5C0006E1E0835A068FFF76BFE06F8010FAE425D
:10A5D000F8D1A068FFF7C7FF431E5842584170BD2D
:10A5E00010B51446FFF7DBFF38B108212046FFF70E
:10A5F000A1FD237A1B1A5842584110BD70B504467C
:10A600000D4680681646FFF7AEFF2946A068FFF7A3
:10A61000ADFE00224E21A068FFF7AAFE0022B1780D
:10A62000A068FFF7A5FE0022F178A068FFF7A0FE62
:10A630002B78102B04D000223179A068FFF798FE08
:10A64000A068FFF790FF2946A068FFF78FFE2278E9
:10A65000A0684821FFF78CFE142005F051FC2378F8
:10A6600013B10A2005F04CFCA068BDE87040FFF76C
:10A670007ABF38B504460D468068FFF774FF294657
:10A68000A068FFF773FE0022B421A068FFF770FEF8
:10A69000A068FFF7A7FE0546A068FFF764FFB5FABC
:10A6A00085F0400938BDF0B585B0144601AA0746CB
:10A6B0000E46FFF795FF054690B13378102B0FD06B
:10A6C0000B2C10D00C2C03D00A2C0ED13F2300E011
:10A6D0007F2301AA314638468DF80830FFF78EFFF8
:10A6E000284605B0F0BD5F23F3E71F23F1E71FB550
:10A6F0000B78102B10D001AAFFF772FF78B19DF8EC
:10A7000008303F2B0ED003D81F2B0DD0002006E0C1
:10A710005F2B03D07F2BF9D10C2000E00B2005B07C
:10A720005DF804FB0A20FAE70920F8E7F0B587B0E6
:10A73000044605F0B1FB00F51C55A068FFF70AFDC3
:10A74000002310352371012601A9A068FFF704FF3B
:10A7500040B305F0A1FBA84224D201A92046FFF78F
:10A7600013FF0028F0D023782BB901A92046FFF76A
:10A7700080FF00B1267003AA01A92046FFF70FFF52
:10A7800001A920466778FFF7B2FF874205D96078B4
:10A790002379607001332371D6E701A92046FFF7C2
:10A7A000A6FFF5E707B0F0BD817070471FB501AA9D
:10A7B000FFF7F5FE9DF80400003018BF012005B03A
:10A7C0005DF804FB0939C9B20229F8B598BF104BEE
:10A7D0000546164694BF33F9114040F2EE248AB183
:10A7E000C3787BB103786BB905F056FB0746314659
:10A7F0002846FFF7DBFF20B905F04EFB001BB842EF
:10A80000F5D3F8BD2046BDE8F84005F079BB00BFA0
:10A8100048870100F8B504460F46FFF768FF064673
:10A8200010B900252846F8BDA068FFF79CFE002857
:10A83000F7D03946A068FFF799FD2278A068442137
:10A84000FFF796FDA5782DB13A4631462046FFF731
:10A85000B9FFE7E70125E5E710785378C00040EA43
:10A86000C3200B78102B00B20BD1D1799379C000A3
:10A87000CB1ADB0120F07F0093FBF1F3103B18446F
:10A8800000B2704730B585B001AA04460D46FFF707
:10A89000A7FE30B101AA29462046FFF7DDFF05B02B
:10A8A00030BD0148FBE700BF80E4FFFF10F5DC5F2F
:10A8B000CABF07EE900ADFED037AFAEEEC7A17EEE4
:10A8C000900A70470000FEC208B5FFF7DBFFBDE845
:10A8D0000840FFF7EBBF01460422012001F0AABAAD
:10A8E00001460422052001F0A5BA014606220920EE
:10A8F00001F0A0BA014604220F2001F09BBA00002B
:10A900002DE9F04F3D4E3E4C336813F0010387B004
:10A9100082468B4615460ED1E3644FF47A73236565
:10A92000384BA36404F15C0004F06AFC082384F84B
:10A93000683001233360344E346001F04DFC002751
:10A94000002859D04FF000494FF00208CDF80C9084
:10A9500005978DF8108003AC94E80E002B4805F0A5
:10A960003DFD5046FFF7C1FF3B463A46394600974A
:10A97000204604F04DFC04A8FFF7BCFF234805F077
:10A9800039FD2B465A465146306801F08FFF0128A9
:10A9900005462DD1CDF80C9005978DF8108094E8E0
:10A9A0000E001A4805F01AFD3168204601F0E5FC5A
:10A9B00004A8FFF79FFF3168204601F0ECFC04A8D3
:10A9C000FFF789FF3168204601F0DEFC04A8FFF79D
:10A9D00087FF0E4805F00EFD3168204601F0E2FCCD
:10A9E0000B4B049A5A6005F071FA80B200F08EFDAC
:10A9F000284607B0BDE8F08F0546F9E7700600204D
:10AA000088060020B4870100840600206408002026
:10AA10007C060020F0B585B007460E4614461D465C
:10AA200001F0DAFB00B34FF00043019300230393DE
:10AA300002238DF8083004AB13E90E000B4805F033
:10AA4000CDFC3846FFF751FF301DFFF753FF281D9F
:10AA5000FFF741FF0A980430FFF742FF034805F073
:10AA6000C9FC034B62685A6005B0F0BD6408002061
:10AA70007C060020F0B58DB01D4600230F460093E4
:10AA8000FF230446164619461A4602A804F0C0FBE6
:10AA90000B4B7A680493CDE905237268CDE907234F
:10AAA0006A68CDE90923039B0B930AAB009306AABE
:10AAB00008AB04A92046FFF7ADFF0DB0F0BD00BF05
:10AAC000C489010000B50B4B4968526889B0CDE9D3
:10AAD0000231CDE905230493012301918DF807305C
:10AAE000019B079304AA06AB02A9FFF7C3FF09B0B5
:10AAF0005DF804FBC48901007FB5094B4A680493E3
:10AB0000CDE90232012301928DF80730019B0593B4
:10AB100004AA02A9FFF7D6FF07B05DF804FB00BF47
:10AB2000C489010008B501F0BDFB012803D002284B
:10AB30000CBF0220002008BD7FB51E4E30680028E3
:10AB400036D001F0CBFE0228044601D004282CD1D7
:10AB50004FF00043019300230393022301AD8DF8CE
:10AB6000083095E80E00144805F038FC3168284696
:10AB700001F003FC02A8FFF7BDFE3168284601F092
:10AB80000AFC02A8FFF7A7FE3168284601F0FCFB8B
:10AB900002A8FFF7A5FE084805F02CFC31682846FE
:10ABA00001F000FC054B029A5A60204604B070BDCB
:10ABB0000446FAE784060020640800207C06002092
:10ABC00030B585B0044604F01BFB4FF00043019301
:10ABD000002303930A4D02238DF8083004AB13E9D8
:10ABE0000E00284605F0FAFB0422A1180F2001F000
:10ABF000D9F9284605F0FEFB204605B030BD00BF60
:10AC00006408002030B585B0044604F0F9FA4FF02E
:10AC100000430193002303930A4D02238DF808306B
:10AC200004AB13E90E00284605F0D8FB0422A11856
:10AC3000052001F0B7F9284605F0DCFB204605B0F9
:10AC400030BD00BF6408002030B585B0044604F074
:10AC5000D7FA4FF000430193002303930A4D0223D8
:10AC60008DF8083004AB13E90E00284605F0B6FB5A
:10AC70000422A118012001F095F9284605F0BAFB3D
:10AC8000204605B030BD00BF6408002007B5002392
:10AC900000931A461946044804F0BAFA034803B070
:10ACA0005DF804EB04F0ACBA740600207C060020CA
:10ACB000007C07288CBF00200120704781F0010034
:10ACC00070470846704708B50368DB6B984780F00B
:10ACD0000100C0B208BD4182704713B502AB0268E3
:10ACE00003F8011D546819460122A04702B010BDA7
:10ACF000037C087C984204D107288CBF00200120E7
:10AD0000704700207047000010B50446007C0728FB
:10AD100016D800F0A1FD182806D80A4B23FA00F037
:10AD2000C04300F0010010BD1C2807D12368204655
:10AD30009B689847003018BF0120F4E70120F2E734
:10AD40000020F0E701001001F0B591B0044604A81E
:10AD50000F46164604F054FA00224FF47A73CDE9F8
:10AD600008230CA8184B079304F04AFA08236846F6
:10AD70008DF83C3004F044FA207C072807D800F016
:10AD80006BFD10B1207C00F0CBFD082323740F4B2A
:10AD90000F4D5B68039302A904A8029501F0DDFD45
:10ADA00041F288336A46394604A801F05FFF40B19A
:10ADB0002368019A9B6903920295324602A92046B4
:10ADC000984711B0F0BD00BFB48701007C06002099
:10ADD000C489010008B5007C072802D800F02EFFC6
:10ADE00008BD0020FCE710B50446207C07280BD8DE
:10ADF00000F032FD172801D01C2805D1207C00F07E
:10AE00001DFFB0F5006FF0D310BD38B50546007CCE
:10AE10000728144605D892B200F092FE10B901231B
:10AE20006B600024204638BD08B5007C072802D896
:10AE300000F02EFE08BD0020FCE7007C072802D8A9
:10AE400012B200F08BBD0020704707B501220DF152
:10AE50000701007C00F082FD0028CCBF9DF80700B0
:10AE60004FF0FF3003B05DF804FB10B5037C072BF7
:10AE7000044602D94FF0FF3010BD03689B68984725
:10AE80000028F7D0207C00F02FFEF5E738B5044607
:10AE9000007C07280AD800F043FD04F0FDFF0546BA
:10AEA000207C00F0D9FC10B90823237438BDFBF7CF
:10AEB000FFFB012005F024F804F0EEFF638A401B3D
:10AEC0009842EDD3207C00F0E5FCEDE77FB5044629
:10AED000007C07280D46164607D800F0BDFC10B1CF
:10AEE000207C00F01DFD082323740021684604F037
:10AEF0009BF96A68019B9A4202D1002004B070BDA0
:10AF00004FF0FF3102A804F08FF96A68039B9A4260
:10AF1000F3D00021212000F003FB07282074ECD897
:10AF2000291D324600F0D4FC04F0B6FF0546207C13
:10AF300000F092FC172815D01C2813D00028DCD074
:10AF400004F0AAFF638A401B984205D8FBF7B0FBC8
:10AF5000012004F0D5FFEAE7207C00F09BFC0823E9
:10AF60002374CAE70120C9E710B41446064A1278D0
:10AF700001EB022101EB00201A46214680B25DF868
:10AF8000044B01F00FB800BF540700207FB5037CCD
:10AF9000072B05464FF000041BD84FF00043022654
:10AFA0000394019301AC8DF8086094E80E000A4800
:10AFB00005F014FA334622460421287CFFF7D4FF1B
:10AFC0009DF804309DF80540034844EA032405F049
:10AFD00011FA204604B070BD640800207FB50B7CD8
:10AFE000072B05460E4605D9002104F01DF9284619
:10AFF00004B070BD4FF0004301930023039302237C
:10B0000001AC8DF8083094E80E00084805F0E6F928
:10B01000042322460C21307CFFF7A6FF034805F0ED
:10B02000E9F92146284604F005F9E0E76408002024
:10B030007FB5037C072B05464FF000041BD84FF06B
:10B04000004302260394019301AC8DF8086094E854
:10B050000E000A4805F0C2F9334622461021287C2A
:10B06000FFF782FF9DF804309DF80540034844EA4D
:10B07000032405F0BFF9204604B070BD6408002029
:10B0800007B5002300931A461946034804F0C0F898
:10B0900003B05DF804FB00BFF406002003681B6BDF
:10B0A00018470000024A02608A694260704700BF88
:10B0B000C4890100808B7047008A7047408C7047BC
:10B0C00013B502AB026803F8011D5468194601224A
:10B0D000A04702B010BD704710B5044690F820009C
:10B0E000072804D800F0D6FB082384F8203010BDD0
:10B0F00038B5044690F8200007280D4601D800F026
:10B10000C9FB2946022000F00BFA072884F820002A
:10B110004FF000009EBF60842582012038BD0000F2
:10B12000F0B591B0044604A80F46164604F068F83E
:10B1300000224FF47A73CDE908230CA8134B079330
:10B1400004F05EF8082368468DF83C3004F058F8A7
:10B150000F4B104D5B68039302A904A8029501F000
:10B16000FCFB41F288336A46394604A801F07EFDB3
:10B17000012808D12368019A1B6A0392029532467E
:10B1800002A92046984711B0F0BD00BFB487010066
:10B190007C060020C489010008B50023C383043164
:10B1A00090F8200000F09CFD08BD08B590F8200044
:10B1B00000F0C4FD08BD10B593B204460A46C18B29
:10B1C00090F8200000F060FDE38B0344E38310BDA2
:10B1D00013B5438C04461BB94FF0FF3002B010BDCD
:10B1E00001220DF1070190F8200000F0B7FB0028C4
:10B1F000F2DD638C9DF80700013B6384EEE710B538
:10B20000438C044613B94FF0FF3010BD934294BFF6
:10B210001AB212B290F8200000F0A0FB0028F2DD74
:10B22000638C1B1A6384F0E708B590F82030072B75
:10B2300005D8428C1AB1184600F056FC08BD4FF0F4
:10B24000FF30FBE773B5044690F8200007280E4650
:10B25000154601D800F01EFB094B00932A4673687F
:10B2600001936946822000F017FA072884F820002D
:10B270004FF000009EBF60840120258202B070BDA7
:10B28000C489010013B50446628C2AB123680021E9
:10B290001B6B20469847F7E794F8200000F0F8FB76
:10B2A000D8B10822694694F8200000F057FB002826
:10B2B00013DD694604F1140003F0C4FF9DF8042077
:10B2C0009DF805309DF8070003EB0223A3839DF84A
:10B2D000063000EB032080B2608402B010BD000095
:10B2E00007B5002300931A461946034803F090FF60
:10B2F00003B05DF804FB00BFFC06002007B5084B57
:10B300001B7801EB032101EB002001220DF1070165
:10B3100080B200F047FE9DF8070003B05DF804FB23
:10B320005407002007B5084B1B7801EB032101EB04
:10B33000002002A980B201F8012D012200F07AFD5F
:10B34000C0B203B05DF804FB5407002010B41446EB
:10B35000064A127801EB022101EB00201A46214631
:10B3600080B25DF8044B00F065BD00BF54070020BB
:10B370002DE9F7430C4617461E4601AA0223242155
:10B380000546FFF7F1FD9DF804209DF8053043EADE
:10B390000223224A1C441378332B0CBF05F108000A
:10B3A00005F11000A4B2C002C4F30A0980B24844F7
:10B3B000372B904680B22DD009EB0603B3F5006F12
:10B3C00028DDC9F500691FFA89F94A46394600F0B7
:10B3D00031FD98F80030332B0CBF05F1080005F162
:10B3E0001000C002A6EB090280B292B207EB09017D
:10B3F0003444A4B200F01EFD23128DF8043001AADB
:10B400000223242128468DF80540FFF79FFF03B053
:10B41000BDE8F08332463946EAE700BF5507002011
:10B4200008B50321FFF76AFF08BD07B50B128DF8B9
:10B4300004308DF80510022301AA0421FFF786FFCE
:10B4400003B05DF804FB08B50A4604230C21FFF79E
:10B450007DFF08BD07B50B128DF804308DF805107F
:10B46000022301AA1021FFF771FF03B05DF804FB6E
:10B4700007B5022301AA2021FFF776FD9DF80400FD
:10B480009DF8053043EA002003B05DF804FB00009E
:10B4900038B50546FFF7ECFF04462846FFF7E8FFFE
:10B4A0008442034604D1034B03EBC5039C8038BDA3
:10B4B0001C46F2E70C07002007B5022301AA26214B
:10B4C000FFF752FD9DF804009DF8053043EA002087
:10B4D00003B05DF804FB07B5022301AA2821FFF79A
:10B4E00043FD9DF804009DF8053043EA002003B0B9
:10B4F0005DF804FB044B1B78332B0CBF0C30183069
:10B50000C00280B2704700BF55070020034B1A8865
:10B51000C0F30D0050401880704700BF08000020A5
:10B520002DE9F043574B1B7885B081460F468BB30E
:10B53000332B4FF0004301934FF000054FF002030F
:10B5400003958DF8083001AE96E80E004E4814BF02
:10B550004FF008084FF0040804F040FFECB220461A
:10B56000FFF75EFF7055D8B10135EBB29845F5D8BD
:10B5700000234FF03451F25C1D2ADCB203D821FACB
:10B5800002F2D20708D40133DAB24245F3D33E487F
:10B5900004F030FF082465E01021204600F0C6FECC
:10B5A0003A4B002123F81410FA20013800BF00BFE5
:10B5B00000BF00BF00BF00BF00BF00BF00BF00BF93
:10B5C00000BF00BF00BF00BF00BF00BF00BF00BF83
:10B5D00000BF00BF00BF00BF00BF00BF00BF00BF73
:10B5E00000BF00BF00BF00BF00BF00BF00BF00BF63
:10B5F00000BF00BF00BF00BF00BF00BF00BF00BF53
:10B6000000BF00BF00BF00BF00BF00BF00BF00BF42
:10B6100000BF00BF00BF00BF00BF00BF00BF00BF32
:10B62000C3D14A462046FFF77DFEFF220221204675
:10B63000FFF778FED7B139462046154DFFF7F5FEE6
:10B6400000260121204600F071FE25F834602046D6
:10B65000FFF741FF05EBC40358809E719E800A48A6
:10B6600004F0C8FE204605B0BDE8F083094B1A88F7
:10B67000013292B2B2F5404F38BF4FF440421A80C7
:10B680001988D9E7550700206408002070070020BA
:10B690000C070020080000202DE9F047694B1B78BB
:10B6A00086B082460E461746A3B3332B4FF00043B5
:10B6B00003934FF000054FF0020305958DF810300D
:10B6C0000DF10C0898E80E005F4814BF4FF0080910
:10B6D0004FF0040904F082FEECB22046FFF7A0FE12
:10B6E00008F80500E0B10135EBB29945F4D8002324
:10B6F0004FF0345118F803201D2ADCB203D821FA88
:10B7000002F2D20708D40133DAB24A45F2D34E48E6
:10B7100004F070FE082485E01021204600F006FEAB
:10B720004A4B002123F81410FA20013800BF00BF53
:10B7300000BF00BF00BF00BF00BF00BF00BF00BF11
:10B7400000BF00BF00BF00BF00BF00BF00BF00BF01
:10B7500000BF00BF00BF00BF00BF00BF00BF00BFF1
:10B7600000BF00BF00BF00BF00BF00BF00BF00BFE1
:10B7700000BF00BF00BF00BF00BF00BF00BF00BFD1
:10B7800000BF00BF00BF00BF00BF00BF00BF00BFC1
:10B7900000BF00BF00BF00BF00BF00BF00BF00BFB1
:10B7A000C3D152462046FFF7BDFDFF2202212046AD
:10B7B000FFF7B8FD002F39D039462046FFF735FE98
:10B7C0005E238DF80630737903F07F038DF8073020
:10B7D000B3798DF808300125F3798DF80930311DE2
:10B7E0002046ADF80450FFF72EFE39462046FFF7FD
:10B7F00031FE0623194601AA2046FFF7A7FD294678
:10B80000134D0026204600F091FD25F834602046B7
:10B81000FFF761FE05EBC40358809E719E800A48C5
:10B8200004F0E8FD204606B0BDE8F087094B1A8811
:10B83000013292B2B2F5404F38BF4FF440421A8005
:10B840001988BAE755070020640800207007002017
:10B850000C0700200800002030B585B04FF00043F1
:10B860000193002303930A4C02238DF8083004ABA4
:10B8700013E90E000546204604F0B0FD2846FFF708
:10B88000CFFD0546204604F0B5FD284605B030BD85
:10B890006408002030B585B04FF0004301930023C9
:10B8A00003930A4C02238DF8083004AB13E90E0011
:10B8B0000546204604F092FD2846102100F036FD92
:10B8C000204605B0BDE8304004F094BD6408002077
:10B8D000F0B585B04FF000430193002303930F4D63
:10B8E00002238DF8083004AB04460F46164628465E
:10B8F00013E90E0004F072FD39462046FFF7A3FD60
:10B9000031462046FFF7A6FD2046042100F00EFD3B
:10B91000284605B0BDE8F04004F06CBD6408002086
:10B9200030B585B04FF000430193002303930A4CD8
:10B9300002238DF8083004AB13E90E0005462046BB
:10B9400004F04CFD2846082100F0F0FC204605B02C
:10B95000BDE8304004F04EBD640800202DE9F04FF2
:10B9600085B04FF000430193464E0023039302231A
:10B9700036F830408DF8083001AB17460546894649
:10B9800041480ECB04F02AFDA7420EDD2846FFF702
:10B9900093FD04462846FFF78FFDA042F9D106EB40
:10B9A000C5039B79E41A26F835408CB92846FFF781
:10B9B00037FD142805D020B1B0F11C0418BF4FF09A
:10B9C000FF34314804F016FD204605B0BDE8F08F85
:10B9D0004FEAC50BBC4206EB0B03A8BF3C46B3F8CD
:10B9E0000280A7B2B9F1000F21D02846FFF782FDEF
:10B9F000264A1278C8F30A0A5044372A80B23DD04A
:10BA00001AFA84F2B2F5006F38DDCAF500631FFA46
:10BA100083FA5246494600F0C5FA2846FFF76AFD08
:10BA2000A7EB0A02D14492B2494600F0BBFA06EBFA
:10BA30000B0236F835309179B844DB1B0F44BFB2A6
:10BA40001FFA88F89BB2F92FA2F8028026F8353049
:10BA500000D8ABB95E440023B3714FEA28238DF8B8
:10BA6000043001AA0223282128468DF80580FFF71B
:10BA70006DFC4021284600F059FCA2E73A46D3E786
:10BA800097719EE70C0700206408002055070020EE
:10BA90007FB5134D064635F83000F8B94FF0004336
:10BAA0000193022303908DF8083004AB0D4813E98D
:10BAB0000E0004F093FC3046FFF7FEFC04463046CF
:10BAC000FFF7FAFCA042F9D1064804F093FC05EB1D
:10BAD000C6039879201A80B225F8360004B070BDEC
:10BAE0000C070020640800207FB54FF0004301934D
:10BAF00000230393104D02238DF8083001AC94E825
:10BB00000E000646284604F069FC3046FFF7F2FCBA
:10BB10000A4B03EBC60301225B88C3F30A031844F4
:10BB2000214680B200F03EFA284604F063FC9DF8FE
:10BB3000040004B070BD00BF640800200C070020A2
:10BB40002DE9F04FB2F5006F87B028BF4FF40062C7
:10BB5000DFF8E49005468A46164603AC02234FF010
:10BB600000474FF000080397CDF814808DF810308F
:10BB700094E80E00484604F031FC2846FFF788FCA4
:10BB800083462846FFF74CFC0190484604F032FCFF
:10BB9000019B172B01D01C2B32D104F0D3F9B345F4
:10BBA000DCD303974FF000080227CDF814808DF8FE
:10BBB000107094E80E00204804F010FC4146334613
:10BBC00052462846FFF7D4FB2021284600F0AEFB62
:10BBD000DFF864804FF0004B02212846FFF78EFB10
:10BBE00010F0100A1FD12846FFF71AFC814648B909
:10BBF000114804F0FFFB4E46304607B0BDE8F08F19
:10BC00004646CEE7404604F0F5FB04F09BF9CDF83C
:10BC10000CB0CDF814A08DF8107094E80E004046DA
:10BC200004F0DCFBD8E7102202212846FFF77AFB5C
:10BC3000014804F0DFFBDFE76408002030B585B081
:10BC40004FF0004301930023039302238DF8083043
:10BC500004AB054613E90E000A4804F0BFFB284672
:10BC6000FFF716FC04462846FFF7DAFB05460548B1
:10BC700004F0C0FB172D02D01C2D18BF0024204655
:10BC800005B030BD640800202DE9FF411C464FF08F
:10BC90000043019300230393104D02238DF80830D5
:10BCA00004AB06460F469046284613E90E0004F002
:10BCB00095FB3046FFF7ECFB844228BF0446A4B254
:10BCC0002346424639463046FFF752FB284604F0E9
:10BCD00091FB204604B0BDE8F08100BF640800205D
:10BCE0007FB50B7806460D4614462BB94B781BB929
:10BCF0008B780BB9C878D0B1DCB14FF00043019319
:10BD00000023039302238DF8083004AB13E90E00DF
:10BD1000094804F063FB29463046FFF794FB2146AF
:10BD20003046FFF797FB044804F064FB012004B0A1
:10BD300070BD2046FBE700BF640800202DE9FF47E7
:10BD400000234FF000480227CDF8048003938DF8BC
:10BD5000087001AC94E80E0005461F48DFF87890A3
:10BD600004F03CFB2021284600F0E0FA022128469E
:10BD7000FFF7C4FA10F0100623D102212846FFF77E
:10BD8000BDFA10F0080A0BD0182202212846FFF74E
:10BD9000C9FA114804F02EFB304604B0BDE8F08724
:10BDA000484604F027FB04F0CDF8CDF80480CDF828
:10BDB0000CA08DF8087094E80E00484604F00EFBC5
:10BDC000D4E7102202212846FFF7ACFA024804F01B
:10BDD00011FB0120E1E700BF6408002007B5002344
:10BDE00000931A461946034803F012FA03B05DF8AF
:10BDF00004FB00BF0407002070B505460C468E18F2
:10BE0000B44206D02178284604F0F5FA04F8010B74
:10BE1000F6E770BD024B0021187804F055BA00BF58
:10BE20000A000020024B0121187804F04DBA00BF2F
:10BE30000A0000202DE9F3414F4B1B78332B0446B9
:10BE40000D4616461FD100EB02084C4F4D1E1FFA3F
:10BE500088F8A0457AD0FFF7DDFFF021384604F0DE
:10BE6000CAFA210A384604F0C6FAE1B2384604F0AC
:10BE7000C2FA013415F8011F3846A4B204F0BBFA27
:10BE8000FFF7D0FFE5E7342BC7B21DD1FFF7C2FFA4
:10BE9000330A241263F07F030422694637488DF881
:10BEA00000408DF801708DF802308DF80360FFF7C7
:10BEB000A3FF013D314CAF19AF4245D015F8011F2A
:10BEC000204604F098FAF7E7FFF7A4FFFF2C08D804
:10BED00000238DF800308DF8017004238DF80230B6
:10BEE0000DE0230419D4E41024F01F04002344F0CF
:10BEF0000C048DF800308DF801708DF80240052E8D
:10BF000028D82A46531BDBB2B34218DA02A80344EE
:10BF100012F8011B03F8051CF4E744F3871323F020
:10BF20001F03B4F5404F4FEA14228DF800208DF81E
:10BF3000017034BF43F0140343F01C03CEE7F21C3E
:10BF400069460E48FFF758FFFFF76CFF304602B016
:10BF5000BDE8F081032269460848084FFFF74CFF0F
:10BF6000731E6C1E15FA83F514F8011F384604F091
:10BF700042FAA542F8D1E7E75507002064080020FF
:10BF800007B502AB012203F8011D1946FFF752FF66
:10BF9000C0B203B05DF804FB08B501460020FFF70E
:10BFA000EFFF08BD2DE9F3413E4B1B78332B0446D0
:10BFB0000E46154620D100EB02083B4F4E1E1FFADD
:10BFC00088F8A0453AD0FFF725FF0F21384604F046
:10BFD00012FA210A384604F00EFAE1B2384604F0AB
:10BFE0000AFA0021384604F006FA013406F8010F77
:10BFF000A4B2FFF717FFE4E7342BC7B222D1FFF753
:10C0000009FF2412C5F3062304228DF804408DF89D
:10C0100005708DF806308DF807500DEB02012248AF
:10C02000FFF7EAFE2A460021304606F0AAFA2A4621
:10C0300031461D48FFF7E0FEFFF7F4FE284602B048
:10C04000BDE8F081FFF7E6FEFF2C07D800238DF84E
:10C0500004308DF805708DF806300DE023040ED401
:10C06000E41024F01F04002344F008048DF8043089
:10C070008DF805708DF80640032201A9CFE744F33F
:10C08000871323F01F03B4F5404F4FEA14228DF8B5
:10C0900004208DF8057034BF43F0100343F01803FB
:10C0A000D9E700BF550700206408002007B501222A
:10C0B0000DF10701FFF776FF9DF8070003B05DF86B
:10C0C00004FB08B50020FFF7F1FF08BD10B5802084
:10C0D000FFF762FF1424FFF7F4FF40B1013C012099
:10C0E000A4B203F00DFF002CF5D1204610BD0120B5
:10C0F000FCE7000008B50F4B33221A70FFF7E6FF8C
:10C1000008B9002008BD1020FFF746FFFFF7D9FF50
:10C110001028F6D11220FFF73FFFFFF7D2FF1228B9
:10C12000EFD10020FFF738FFFFF7CBFFB0FA80F028
:10C130004009E7E75507002008B5124B34221A7072
:10C14000FFF7C4FF08B9002008BD0820FFF724FF4F
:10C15000FFF7B7FF0828F6D11020FFF71DFFFFF704
:10C16000B0FF1028EFD10020FFF716FFFFF7A9FF5F
:10C170000028E8D11F20FFF799FFC31E58425841FD
:10C18000E2E700BF5507002008B5124B37221A70AE
:10C19000FFF79CFF08B9002008BD0820FFF7FCFE50
:10C1A000FFF78FFF0828F6D11020FFF7F5FEFFF705
:10C1B00088FF1028EFD10020FFF7EEFEFFF781FF88
:10C1C0000028E8D13920FFF771FF031F584258417A
:10C1D000E2E700BF550700207FB52D4E3478002CD4
:10C1E00053D14FF40C7003F08BFE2A4804F0E0F8B2
:10C1F000294B0121187804F03FF8FFF713FE4FF0A8
:10C200000043019302238DF80830039404AB13E933
:10C210000E00204804F0E2F8FFF78EFFB0B11F4B8C
:10C2200040221A70E5B202221E212846FFF77AF852
:10C23000013402221F212846FFF774F8082CF1D19F
:10C240001448012404F0D6F834701BE0FFF79CFF7B
:10C2500018B1124B10221A70F2E7FFF74BFF044699
:10C2600058B10E4B042255211B201A70FFF788FE8F
:10C2700055211A20FFF784FEE2E7094B18700548A4
:10C2800004F0B8F8204604B070BD0124FAE700BFFE
:10C2900056070020640800200A00002054070020F0
:10C2A000550700201FB5FFF797FF38B11D4B1B78CE
:10C2B000342B4FF0000003D0372B1BD004B010BD3F
:10C2C0004FF000430193022303908DF8083004AB34
:10C2D00013E90E00144804F081F83520FFF7E6FE5C
:10C2E0000446114804F086F814F0200F14BF012012
:10C2F0000220E3E74FF000430193022303908DF8FF
:10C30000083004AB13E90E00074804F067F82E204C
:10C31000FFF7CCFE0446044804F06CF814F0010F5B
:10C32000E4E700BF550700206408002038B50A463E
:10C3300001210446FEF7F6FF054D2402287804EBA0
:10C340000020013080B2FFF7B1FE0028F6D138BDE1
:10C350005407002007B5002300931A4619460348E6
:10C3600002F056FF03B05DF804FB00BF4C0700204D
:10C3700014220021103006F004B910B51031044623
:10C3800002F058FF204610BD10B51431044602F0EB
:10C3900051FF204610BD10B51831044602F04AFF87
:10C3A000204610BD10B52031044602F043FF204660
:10C3B00010BD30204B1C0870110902F00F02092A31
:10C3C00094BF3032373203F801290A460029F3D1ED
:10C3D0007047000007B5002300931A46194603482A
:10C3E00002F016FF03B05DF804FB00BF5807002001
:10C3F0002DE9F0418EB004468846164600212022E1
:10C4000006A806F0BEF8FF231A461946009302A8B4
:10C4100002F0FEFE04F14805554B04934322039BB2
:10C42000059304A92846FEF7B7FE013000F09D8071
:10C43000504B069363688DF821601BBA0793330A4B
:10C440008DF820301C22802306A926462846ADF808
:10C450002230FEF7B0FE1A2200210DF11E0006F078
:10C4600090F856F8080F0690B388ADF81C301022EB
:10C4700006A92846FEF79FFE2022002106A806F006
:10C4800080F80627202206A92846FEF794FE013FE1
:10C49000F8D1394B069340F23513ADF81C303D23EB
:10C4A0008DF81F3007238DF8203001238DF82130BF
:10C4B0003368CDF82230B388ADF826302F498DF897
:10C4C0001E8040F60C430DF12A00ADF8283006F02E
:10C4D000DAFFE27A0CA92046FFF76BFF227B0DF111
:10C4E00032012046FFF765FF627B0DA92046FFF76A
:10C4F00060FF1E2206A92846FEF75DFEB8F1030F75
:10C5000024D140F23243ADF81830237C8DF81A3034
:10C51000637C8DF81B30A37C8DF81C30E37C8DF898
:10C520001D3040F23643ADF81E30237F8DF82030A9
:10C53000637F8DF82130A37F8DF822300C22E37FBA
:10C540008DF8233006A92846FEF735FE0C4A0D4B20
:10C5500006A9CDE906232846FF2309228DF82030BD
:10C56000FEF729FE2846FEF720FE0EB0BDE8F0815A
:10C57000C48901000101060063825363FC87010046
:10C5800037060103060F3A3B2DE9F04391B005460B
:10C590008846164603F080FC05F14804074620460D
:10C5A000FEF770FE00280BDC03F076FCC01B404554
:10C5B00000F2D280FAF77CF8012003F0A1FCEEE74C
:10C5C000242207A92046FEF71AFE9DF81C30022BF4
:10C5D00040F0BD80B5F86430432B40F0B880089F30
:10C5E0003FBA3760062205F108010EA805F096FF54
:10C5F000064628B92B689F4202D36B689F4207D931
:10C600002046FEF768FD0026304611B0BDE8F083F5
:10C610000B9B2B610146CC222046FEF7F0FD05F175
:10C6200024072046FEF74AFD002840F3918020466B
:10C63000FEF7CEFD33287DD015DC012844D006DC82
:10C640000028EED02046FEF7C3FDC2B253E0032817
:10C6500044D00628F6D12046FEF7BAFD04228046D3
:10C6600005F1200141E03A284AD020DC352823D0CA
:10C670003628E7D12046FEF7ABFD05F11C08414600
:10C68000814601A802F0D6FD002103A802F0CCFDEE
:10C69000029A049B9A4230D0414605A802F0CAFD96
:10C6A0002A6E069B9A4228D05FFA89F223E03B2843
:10C6B00033D0FF28B5D0C5E72046FEF789FD2046D8
:10C6C000FEF786FDC6B2ACE72046FEF781FD0422E8
:10C6D00005F114012046FEF792FDA2E72046FEF781
:10C6E00077FD0422804605F118012046FEF787FDFC
:10C6F0005FFA88F2043A0021ECE704224146E9E7B8
:10C700002046FEF765FD042205F128012046FEF7CC
:10C7100076FDAB6A1BBAAB6283E72046FEF758FD95
:10C72000042205F12C012046FEF769FDEB6A1BBAD5
:10C73000EB6276E72046FEF74BFD042239462046A1
:10C74000FEF75DFD6B6A1BBA6B622B6369E700261F
:10C750002046FEF7C0FC57E7FF2655E72DE9F347D3
:10C7600004464FF4FA61012003F017FA274660608F
:10C7700047F8480B3846FEF7AFFC44213846FEF731
:10C78000B7FC002800F0908003F086FB4FF0000912
:10C79000804600254FF0030A94F84430032B1CD048
:10C7A00043BB63680133636003F076FB4FF47A7236
:10C7B000A0EB08000121B0FBF2F2204692B2FFF795
:10C7C00017FE012384F84430002DE5D103F064FB0B
:10C7D000A36BA0EB08009842DBD93846FEF77CFC3F
:10C7E00063680133636003F057FB2064284602B09E
:10C7F000BDE8F087042B11D163680133636003F057
:10C800004BFB4FF47A72A0EB08000321B0FBF2F26D
:10C81000204692B2FFF7ECFD0223D3E7012B19D19A
:10C8200001AAE16B2046FFF7AFFE0228064638D189
:10C83000019B636003F030FB4FF47A72A0EB0800B9
:10C840000321B0FBF2F2204692B2FFF7D1FD84F84B
:10C850004460B9E7022BB7D101AAE16B2046FFF78C
:10C8600093FE0528064617D1636A84F844A013B9DD
:10C870004FF461736362A36A13B9636A5B08A362CE
:10C88000E36A1BB9636AA3EBD303E362A36A23637E
:10C89000E36A636301257FE7062802D184F84490A8
:10C8A00092E7FF2EFAD08FE705469FE7F8B50025FF
:10C8B0000F460446C0E90955C562C0E90E238560EC
:10C8C0008581FFF755FD3B68A360BB88A38184F891
:10C8D00044502046BDE8F840FFF740BF10B504467D
:10C8E00003F0DAFA236CC31AB3F57A7F14D34FF44A
:10C8F0007A71B3FBF1F201FB1233C01A236B20648F
:10C9000051008B4234BF00239B1A2363636B99420F
:10C910008CBF00239B1A6363206BE0B994F844300A
:10C92000032B06D1042384F844302046FFF716FF7A
:10C930000130636B73B994F84430032B00D04BB9CA
:10C94000002384F844302046FFF712FD2046FFF70D
:10C9500005FF033010BD0020EBE74B684360002368
:10C960000381704770B500240139234611F8010F87
:10C97000B8B1A0F13005EEB2092E08D803EB83035D
:10C9800005EB43039BB2FF2BF0D900200DE02E28CE
:10C99000FBD1032CF9D0601C14442371C4B20023D2
:10C9A000E4E7032C01D1D371012070BD07B500234A
:10C9B00000931A461946034802F02AFC03B05DF8BA
:10C9C00004FB00BF600700202DE9F74305460E4633
:10C9D00003F062FA05F10C04288105F10801022236
:10C9E00002AD2046FEF7E7FB012325F8023D0222B7
:10C9F00029462046FEF7DFFB4FF4807302222946CA
:10CA00002046ADF80630FEF7D6FB00230222294669
:10CA10002046ADF80630FEF7CEFB0222294620461E
:10CA2000FEF7C9FB022229462046FEF7C4FB374623
:10CA30003378E3B13E46B04618F8013B0BB12E2BDC
:10CA400013D1A6EB0709B9F1000F0CDD01220DF19E
:10CA5000050120468DF80590FEF7ADFB4A463946A4
:10CA60002046FEF7A8FB4746E2E74646E3E702A971
:10CA7000012201F8033D2046FEF79DFB4FF480762E
:10CA8000294602222046ADF80660FEF794FB0222FA
:10CA900029462046ADF80660FEF78DFB012003B065
:10CAA000BDE8F0832DE9F04387B006460F46904677
:10CAB00003F0F2F906F10C0405462046FEF7E2FB0E
:10CAC000002808DC03F0E8F9401BB84200F2C480FB
:10CAD000F9F7EEFDF1E7726A73689A4240F0BF80A1
:10CAE000338D352B40F0BB802046FEF7E7FA0B284C
:10CAF00040F3B8800C220DEB02012046FEF77FFBCD
:10CB0000BDF80E203189130A43EA0223BDF80C2038
:10CB10001BB29DB29142ADF8065001D1002B07DB4C
:10CB20002046FEF7D8FA4FF6FC7007B0BDE8F08358
:10CB300040F20F231D4005D02046FEF7CCFA4FF6F9
:10CB4000FB70F2E7BDF812301F0A47EA0327BFB2B5
:10CB50002FB92046FEF7BFFA4FF6FA70E5E7BDF8A9
:10CB600010305BBAAAB29BB29A4216DA01220DF1DA
:10CB70000A012046FEF743FB9DF80A201AB1002166
:10CB80002046FEF73CFB9DF80A100029EED1042256
:10CB90002046FEF734FB0135E1E70026B1460122CD
:10CBA0000DF105012046FEF72AFB9DF8052012F045
:10CBB000C00134D112B12046FEF721FB9DF805508B
:10CBC000002DECD1022202A92046FEF718FB02221A
:10CBD0000DF10A012046FEF712FB042229462046E9
:10CBE000FEF70DFB02220DF106012046FEF707FBC2
:10CBF000BDF80830BDF80620B3F5807F52BA92B276
:10CC00001CD1BDF80A0040BA85B2012D16D1042A04
:10CC10000DD02046FEF75FFA4FF6F77085E7012248
:10CC200000212046FEF7EBFA8DF80590C6E708F1E3
:10CC300004012046FEF7E3FA284676E70136002194
:10CC40002046B6B2FEF7DBFAB742A8D12046FEF77F
:10CC500042FA4FF6F67068E74FF6FF7065E74FF659
:10CC6000FE7062E74FF6FD705FE700002DE9F347C5
:10CC700005468A4691469846FFF774FE0446B8BBBF
:10CC80001E4B6A685B689A4234D003F005F905F1DF
:10CC90000C0600F00F0101F580613046FEF728FA1E
:10CCA0000128074620D1164B009335226B6801936B
:10CCB00069463046FEF770FA98B151462846FFF7AC
:10CCC00083FE70B13046FEF770FA50B14A464146D5
:10CCD0002846FFF7E7FE0446F9F7EAFC384603F07A
:10CCE0000FF93046FEF7F8F9204602B0BDE8F087AC
:10CCF0000124F9E76FF00104F6E700BF60070020A8
:10CD0000C489010007B5002300931A461946034859
:10CD100002F07EFA03B05DF804FB00BF6807002054
:10CD2000006903681B691847006903685B69184755
:10CD300013B5006949680368034C01919B6900942D
:10CD40006946984702B010BDC489010000690368B4
:10CD5000DB691847006903689B6A1847006900305F
:10CD600018BF01207047006C70470164704710B510
:10CD700090F83830044633B920690368DB68984777
:10CD8000002808DA10BD03689B6898470028F3D193
:10CD90004FF0FF30F6E794F82220A2F10803022BAF
:10CDA000F0D8A36A002BC2BFE36A0133E3620A2A08
:10CDB000E8D1E36B013BE363002BE3D1092384F863
:10CDC0002230DFE710B50446006903681B6A984704
:10CDD00094F82230083B022B07D8A36A002B04DD0D
:10CDE0000028A2BFE36A1B18E36210BD73B590F878
:10CDF0002230092B04460ED10026206903689B6867
:10CE0000984740B120690368DB689847C5B20A2D8E
:10CE10001CD184F8225094F822300A2B04D1E36B01
:10CE200013B9092384F8223094F82230092B22D038
:10CE3000206903689B68984794F822300A2B03D135
:10CE4000E36B9842A8BF184602B070BD0D2DD4D038
:10CE5000284605F00CFB0028CFD0E06BADF804604D
:10CE600010228DF804500021050101A807F09AFA5C
:10CE70002844E063C1E70020E6E7000000234FF00C
:10CE8000FF32C0E90A23084A80F8223012680263A0
:10CE9000064A4362126880F83830C36347F2305361
:10CEA00042630364704700BF10000020140000209C
:10CEB00038B504461D4600204FF47A73C4E90103D7
:10CEC0000B4B2360C4E9041204F1180002F098F936
:10CED0000123258484F8443084F84530054904F161
:10CEE000480002F0B3FE2046FFF7C8FF38BD00BF80
:10CEF000648801001A89010010B5044600690368BE
:10CF00005B6A98472046BDE81040FFF7B7BF012392
:10CF100080F822307047000038B504460069154695
:10CF200002F0C7F90449206902F0C3F929462069D3
:10CF3000BDE8384002F0D4B94170010038B504466C
:10CF40000D460069114602F0B4F91D49206902F04E
:10CF5000B0F92946206902F0ACF91A49206902F0BB
:10CF6000BFF994F84530F3B16369B3B1164920694C
:10CF700002F09FF9D4E9040102F09BF9238C502BB5
:10CF800008D01249206902F094F90A22218C206904
:10CF900002F0EFF9206902F093F90D4B0D491A6880
:10CFA0002046FFF7B9FF94F8443023B10A4A0B49F1
:10CFB0002046FFF7B1FF012384F82230002038BD5E
:10CFC000687101002988010033880100587201004E
:10CFD0000C0000203A880100458801004B880100C0
:10CFE00038B504460069154602F063F90549206921
:10CFF00002F05FF9294620690A22BDE8384002F0B4
:10D00000BAB900BF4170010010B50446006902F0D2
:10D0100057F9022384F8223010BD70B590F8223001
:10D02000012B04460D46164601D8FFF7EDFF206997
:10D030000368324629465B68BDE87040184770B502
:10D0400090F82230012B04460D4601D8FFF7DCFF93
:10D050002069036829461B68BDE87040184710B571
:10D060000446206903689B68984720B120690368DB
:10D07000DB689847F5E710BD2DE9F347994690F82E
:10D080002230083B022B04460E469246DDE90A7820
:10D0900004D8FFF7E4FF2046FFF7F0FE94F8225093
:10D0A000012D44D894F8443063B1D4E90401228CB2
:10D0B0000368002934D121490091E16901919B69FC
:10D0C00069462EE0206903689B6A98470028ECD0E7
:10D0D000314652462046FFF731FF0646E0B9B9F126
:10D0E000000F04D04A4616492046FFF715FF002FCF
:10D0F00020DD3A4613492046FFF772FFB8F1000FD2
:10D1000018D001252046FFF77FFF2DB123683A464E
:10D110005B68414620469847304602B0BDE8F0873C
:10D12000DB6998470028D3D14FF0FF36F4E76FF062
:10D130000106F1E7002DEFD1E4E700BFC48901004B
:10D14000038801001088010090F82230012B01D8DB
:10D15000FFF75ABF7047FFF7F7BF000007B500237E
:10D160004FF0FF32CDE90023024AFFF785FF03B0FD
:10D170005DF804FB568801002DE9F04790F8223055
:10D18000012B044651D9DFF8D8800025032700235E
:10D190006362022384F8223002F07EFE4646824615
:10D1A0004FF00A090A2D46D002F076FE236CA0EB60
:10D1B0000A00984245D2236820469B68984748B3A6
:10D1C00023682046DB689847431C0546ECD094F85A
:10D1D0002230022B05D0032B0FD002F05DFE8246D9
:10D1E000E0E733782A2B01D083421AD17278731C7E
:10D1F0000AB984F822701E46EFE7A0F13002092A2E
:10D2000095BF636A042309FB032384F8223098BF87
:10D210006362E2E74FF47A7002F072FEC2E70A2D11
:10D2200006D16FF00300BDE8F0876FF00100FAE768
:10D230006FF00200F7E7636AC72B02DC652B18BFAB
:10D24000002594F82230042BE9D1606AC72801DC5C
:10D2500065289CD10A2D18BF6FF00200E3E700BFDC
:10D260001F88010038B501F1480504463A212846D7
:10D2700002F0CCFD421C034605D10649204602F0CF
:10D28000E5FC204638BD00222946204602F0DCFDA0
:10D29000F7E700BF1A890100F8B501F14806054615
:10D2A0000F4630463A2102F0B1FD441C013005D151
:10D2B0000C49284602F0CAFC2846F8BD3B6DA34243
:10D2C00009DD2146304602F085FD007805F0C6F8FC
:10D2D00008B10134F2E73B6D22463146284602F0A0
:10D2E000B3FDE9E71A89010010B503680446DB685D
:10D2F000984794F82230A3F10802022AC0B232D92A
:10D30000052B31D0072B39D0042B54D1226B137845
:10D3100083420BD1531C2363537823B9C4E90A33E6
:10D32000052284F822200A281DD136E0636B197883
:10D3300081420BD15A1C62635B78002BF3D101232D
:10D3400084F83830062384F82230ECE71B4909685A
:10D350008A42F7D11A4A12689342F3D10D28F1D1CB
:10D36000072384F8223010BDA0F13002092AE9D841
:10D37000A36A0A2101FB0323A362D4E70A28F2D19E
:10D3800094F838309BB1092384F822300023E363FA
:10D3900094F82230083B022BE5D9042384F822308C
:10D3A000064B1B682363064B1B686363DBE708239C
:10D3B00084F82230ECE70A28D5D1E9E710000020F4
:10D3C0001400002038B5044602F066FD054694F8C6
:10D3D0002230083B022B13D902F05EFD236C401B68
:10D3E00098420DD2236820469B68984718B1204682
:10D3F000FFF77AFFE8E74FF47A7002F081FDE6E785
:10D4000094F82230083B022B94BF00206FF00200FA
:10D4100038BD10B590F82230083B022B044601D9E4
:10D42000FFF7D0FFA06A10BD38B590F82230083B56
:10D43000022B054601D9002038BDFFF7EAFF013075
:10D44000F9D02846EC6AFFF7E4FF8442B4BF00201D
:10D450000120F1E7FFF7E8BFFFF7E6BF38B500F1BD
:10D46000480504460E49284602F04DFC94F8223047
:10D47000083B022B09D92046FFF736FF0D2801D0C3
:10D480000A2807D1236D002BF0D0206D003018BF83
:10D49000012038BDC1B2284602F056FCE6E700BFC5
:10D4A0001A89010007B5002300931A46194603485C
:10D4B00001F0AEFE03B05DF804FB00BF8007002062
:10D4C00000B55DF804FB0020704700B501205DF851
:10D4D00004FB80687047C1607047036810B59B69A2
:10D4E0000C469847036821461B68BDE81040184762
:10D4F0002DE9F84380460D46174601EB02090C461C
:10D50000A145A4EB050609D0D8F800304046DB68F9
:10D510009847431C03D004F8010BF1E73E46304620
:10D52000BDE8F883C368013310B5044612D12368FF
:10D5300020469B69984703689B68984758B12368C1
:10D540002046DB6898472028F1DD2368C1B25B697B
:10D5500020469847012010BD70B50446C068431CA2
:10D5600018D102F099FC00F5FA75236820469B69F2
:10D57000984703689B68984718B902F08DFC85426C
:10D58000F3D8236820469B6998470368BDE870403C
:10D59000DB6818474FF0FF33E36070BD10B518200B
:10D5A00004F09AFF044618B11822002104F0E9FFA4
:10D5B000204610BD70B506460C46D4B1237C656884
:10D5C0001B0704D4E16811B13046FFF7F3FF237C59
:10D5D00003F00F03042B03D1606908B104F084FF4A
:10D5E000206808B104F080FF204604F07DFF2C463F
:10D5F000E3E770BD2DE9F04F036885B0DB680546B1
:10D600000E469847421C044604D14FF0FF3005B047
:10D61000BDE8F08F2D2832D12B682846DB6898476B
:10D62000431C0446F1D04FF0FF330093A4F13003C4
:10D63000092B4FF000070DD84FF00A082B68284639
:10D64000DB689847A0F13003303C092B08FB074703
:10D650000446F3D92E2C14D024F02003452B10D0EF
:10D66000009B7B437361337C022262F303033374B8
:10D670002B6828465B69E1B298470020C7E7012381
:10D68000D3E7384604F024F92E2C8046894639D158
:10D690002B68DFF818B1DB68284698470027044656
:10D6A0004FF0000A52465B464046494604F07AF97C
:10D6B00080468946A4F1300004F00AF942464B4600
:10D6C00003F0BAFF2B688046DB68284689469847F6
:10D6D000A0F13003092B07F1FF370446E2D924F00B
:10D6E0002003452B2AD12B682846DB6898472B2836
:10D6F000044609D12B682846DB68984704464FF05A
:10D70000010A0AE00027EAE72D28F8D12B6828460D
:10D71000DB6898474FF0FF0A04464FF0000B0A22DF
:10D72000A4F13003092B0DD802FB0B3B2B680392AD
:10D73000DB6828469847039A0446F1E74FF0010A50
:10D740004FF0000B009804F0C3F842464B4604F03B
:10D7500029F9CDE90001584604F0BAF88046504650
:10D76000894604F0A5F802460B464046494604F0B7
:10D7700019F980463846894604F0AAF802460B4655
:10D780004046494603F058FF02460B460020074931
:10D7900002F072FE02460B46DDE9000104F002F9D8
:10D7A00004F0F8FB337C706103225EE70000244044
:10D7B00019B10A22496901F0BABD08467047000054
:10D7C000F8B506462DED028BD1B391ED058A18EE22
:10D7D000100A04F08FF8B5EEC08AF1EE10FA044694
:10D7E0000D4606D51A49304601F063FD05F10043A8
:10D7F0001D462946204604F0ADFB0A220146074695
:10D80000304601F0C2FD1349304601F052FD384662
:10D8100004F04EF802460B462046294603F00AFF64
:10D8200009A3D3E9002303F007FF00220A4B04F009
:10D83000B9F804F08FFB0A220146304601F0B4FD2E
:10D84000BDEC028B0020F8BD9A9999999999A93F4E
:10D850005B8E01000D81010000002440F8B50368D3
:10D86000DB6806460F469847222803D04FF0FF3466
:10D870002046F8BD3B7C042262F303033B7400F0B6
:10D88000EFFA05460028F1D033683046DB68984748
:10D89000431C044611D0222C36D01F2C34DD5C2CC6
:10D8A00004D02946E0B200F0F1FAEDE733683046E3
:10D8B000DB689847421C044603D1284600F00EFB63
:10D8C000D6E7622817D007DC2F2803D05C2801D0C8
:10D8D0002228D9D12946E6E76E280FD004DC662835
:10D8E000D2D129460C20DEE772280AD07428CBD189
:10D8F00029460920D7E729460820D4E729460A20E7
:10D90000D1E729460D20CEE7284600F0CBFA0024C7
:10D910007861ADE738B50D461D49044601F0C9FCF4
:10D920007DB3013D15F8011F59B31F2907D92229DD
:10D9300005D05C2903D0204601F0BFFCF2E75C2152
:10D94000204601F0BAFC29780C2914D007D80929FF
:10D9500015D00A2911D00829E4D16221EBE7222948
:10D96000E9D003D80D29DDD17221E4E72F29E2D0D7
:10D970005C29E0D0D6E76621DDE76E21DBE7742184
:10D98000D9E72221204601F098FC002038BD00BFD5
:10D99000447001004969FFF7BDBF0368DB6810B53B
:10D9A00004469847431C0AD02028236802DCDB6821
:10D9B0002046F6E7C1B25B6920469847002010BDBB
:10D9C00003682DE9F047DB6804460E469146984708
:10D9D0007B2803D04FF0FF30BDE8F087337C062270
:10D9E00062F3030333742046FFF7D7FF2368204612
:10D9F000DB6898477D2844D02368C1B25B69204624
:10DA00009847FF274FF0000AFFF7C8FD054600289A
:10DA1000E0D08FB3F0602046FFF7BFFF29462046D5
:10DA2000FFF71CFF0130D5D02046FFF7B6FF6B692A
:10DA30002B602368C5F814A0DB68204698473A2875
:10DA4000C8D12046FFF7A9FF4A462946204600F0E4
:10DA50001BF80130BED02046FFF79FFF2368204609
:10DA6000DB6898472C28A8464FF00007CCD07D38BB
:10DA700018BF4FF0FF30AFE7C8F80400C0F80880C7
:10DA8000C9E70020A8E70000F7B504460D46174691
:10DA9000FFF783FF013002D14FF0FF3011E0236820
:10DAA0002046DB689847431C0646F5D02368C1B280
:10DAB0005B6920469847222E05D129462046FFF76C
:10DAC000CDFE03B0F0BD2D2E03D0A6F13003092BFF
:10DAD00004D829462046FFF78DFDF2E75B2E05D1DD
:10DAE0003A462946204600F080F8EAE77B2E05D129
:10DAF0003A4629462046FFF763FFE2E76E2E17D12C
:10DB000002AE002346F8083D236804221B69314613
:10DB10002046984704280246BED12149304605F0E8
:10DB2000F2FC0028B8D12B7C6FF303032B74C8E7F9
:10DB3000662E19D1002300938DF804302368052246
:10DB40001B696946204698470528A5D10522154935
:10DB5000684605F0D8FC00289ED12B7C2875012250
:10DB600062F303032B74ACE7742E95D102AE00234D
:10DB700046F8083D236804221B6931462046984731
:10DB80000428024688D10849304605F0BCFC00282C
:10DB900082D12A7C012363F303022A742B7590E758
:10DBA000DE880100E3880100E9880100F8B5064637
:10DBB00017460D4611B900242046F8BDFFF7EEFCCC
:10DBC00004460028F7D02846FFF7E7FE3A462146EC
:10DBD0002846FFF759FF0130EED121463046FFF7C6
:10DBE000E9FCE8E70022FFF7E1BF2DE9F84303680D
:10DBF000DB6804460F46914698475B2803D04FF0F8
:10DC0000FF30BDE8F8833B7C052262F303033B74DD
:10DC10002046FFF7C2FE23682046DB6898475D2850
:10DC20002BD02368C1B25B6920469847FF26FFF7D7
:10DC3000B5FC05460028E2D0D6B1F8602046FFF7D3
:10DC4000ACFE4A4629462046FFF71EFF064600283E
:10DC5000D5D12046FFF7A1FE23682046DB68984710
:10DC60002C28A846E3D05D3818BF4FF0FF30C8E736
:10DC7000C8F80400C0F80880E0E70020C1E738B524
:10DC8000054651B3CC687B2101F017FB013002D16E
:10DC90004FF0FF3038BDB4B121682846FFF73AFE97
:10DCA0000130F5D03A21284601F007FB0130EFD0D2
:10DCB0002146284600F014F80130E9D0646814B118
:10DCC0002C212846E0E77D21284601F0F6FA0130B4
:10DCD0004FF0FF3018BF0020DCE70846DAE700000D
:10DCE000E9B10B7C03F00F03062B18D8DFE803F033
:10DCF00004070D0F111315000A4901F0DABA0B7D64
:10DD00000BB10949F9E70949F7E7FFF751BDFFF7FB
:10DD100057BDFFF73FBE00F00EB8FFF7B0BF0020C1
:10DD2000704700BFDE880100E9880100E388010038
:10DD30001046FFF7D5BF38B50546F1B1CC685B2179
:10DD400001F0BBFA013002D14FF0FF3038BD54B1C1
:10DD500021462846FFF7C4FF0130F5D0646814B1AE
:10DD60002C212846ECE75D21284601F0A6FA013077
:10DD70004FF0FF3018BF0020E8E70846E6E7CB6821
:10DD80000022D0B201320BB15B68FAE77047C86875
:10DD900020B11AB1013AD2B24068F9E7704738B5FC
:10DDA000CC68154634B12946206805F028FB08B137
:10DDB0006468F7E7204638BD4AB1CB6813B9CA603A
:10DDC00070470B4659680029FBD15A609360704731
:10DDD000F8B505460E4617461C4673B1186808B1DB
:10DDE00004F082FB384605F057FB2246206031469E
:10DDF0002846BDE8F840FFF7DFBFF8BD08B5FFF7DC
:10DE0000CDFB18B1037C6FF30303037408BD10B599
:10DE10000C46FFF7C3FB28B1037C4461022262F386
:10DE20000303037410BD70B50D461946044616462B
:10DE3000FFF7EDFF3246034629462046BDE8704015
:10DE4000FFF7C6BF07B5002300931A4619460348DB
:10DE500001F0DEF903B05DF804FB00BF8807002085
:10DE600038B50C2004F038FB044650B10648206059
:10DE70004FF480752A46002104F083FB002365607F
:10DE8000A360204638BD00BF90080020D1E90123DF
:10DE9000934204D20A68D0548B6801338B6000200F
:10DEA00070470000826838B5044622B10368134405
:10DEB00013F8013C1BB121460020FFF7E7FFA068E3
:10DEC00004F00AFB054628B1034905F0DCFA2046B8
:10DED00004F00AFB284638BD9008002008B104F081
:10DEE00003BB704710B5054C204601F0E9F9204608
:10DEF0000349BDE8104001F0D3B900BFEC07002092
:10DF000014890100F0B504789FB005464CB31A4B54
:10DF10001A4F1B68986804F08FF92846174906F0D5
:10DF20005FF91EAD012445F8780D3946002006F052
:10DF300057F91E2C264645F8240002D0013400284B
:10DF4000F3D10F4B009F1C6884B12168384605F05F
:10DF500090FA48B963682946304698470446FFF767
:10DF6000C1FF20461FB0F0BDA468EDE70549064893
:10DF700001F0ACF9F3E700BF380000206871010040
:10DF8000D40700201B890100EC070020F8B50546E6
:10DF90000C200F4604F0A0FA0C4B044618602846EB
:10DFA00005F095FA013004F097FA2946064605F087
:10DFB0006AFA284605F08BFA00233354044B1A689A
:10DFC000A260C4E900671C60F8BD00BFD407002050
:10DFD0009407002070B51648164D01F0BFFCC4B27E
:10DFE0000A2C0CD00D2C0AD0082C15D12146104833
:10DFF00001F063F92B7873B1013B2B700BE02B78A8
:10E000000D4E0E490A480024F45401F052F93046EE
:10E01000FFF778FF2C7070BD2146054801F04DF9DF
:10E020002B783A2B9FBF5A1C2A70034AD454F2E72C
:10E03000EC070020D807002098070020188901006D
:10E0400010B5044C204601F083FC10B1FFF7C2FF6D
:10E05000F8E710BDEC070020054A00231370054ABD
:10E060000146136010B1044801F032BC704700BF94
:10E07000D807002094070020EC07002070B5044664
:10E080000D4601F009FFA061A068036829461B68DE
:10E09000BDE87040184770B504460D46164601F0BD
:10E0A000FBFEA061A0680368324629465B68BDE8B4
:10E0B0007040184710B50446C06804F015FA2046B1
:10E0C00010BD2DE9F04105460E4601F0E5FE4FF486
:10E0D0007A778046A86803689B689847044658B9D1
:10E0E00001F030FF01F0D8FEAB8AA0EB08007B43C3
:10E0F0009842EFD3204605E0A8680368DB6898479C
:10E1000030700120BDE8F08138B5148821441546EF
:10E11000FFF7D7FF08B101342C8038BD2DE9F74F48
:10E1200002AD002625F8026D8A462A46C1680446DB
:10E13000FFF7EAFF18B9002003B0BDE8F08FE368ED
:10E140000DF1080993F8008009F8036D0127BDF867
:10E150000630052B07D14FF0FF33A068E363036857
:10E160005B6A9847E7E749462046FFF7AAFF002881
:10E17000E1D0BDF80630E268591CADF806109DF8F4
:10E180000510D1549DF8053003F07F0207FB0266AD
:10E190001A064FEAC717DAD49DF8063008F0F008DF
:10E1A000013BB8F1300F8AF800301DD12A46E168F2
:10E1B0002046FFF7A9FF0028BDD02A46E168204687
:10E1C000FFF7A2FF0028B6D0E2689AF800301344A7
:10E1D00059789D78137805EB01259B07ADB201D5E1
:10E1E0000235ADB2022701E000273D46BDF806B07A
:10E1F000A7EB0B0707EB0B0296422AD949462046AC
:10E20000FFF75FFF002896D0A06B88B1B8F1300F00
:10E210000ED19AF80020C2F1FF2202F57F02FE32F1
:10E220005A44AA4204D902689DF805101268904722
:10E23000BDF80620218A914208D9E1689DF80500C1
:10E240008854BDF806200132ADF806200BF1010B11
:10E25000D0E7A26B22B9218A594538BFADF8062014
:10E26000BDF8060068E70120704773B50025DC1192
:10E2700003F07F06A3B20CB146F080060DF1080C46
:10E28000681C6544C0B205F8046C0546002CEED14C
:10E29000C0F10405515501ADA04205DD231A134418
:10E2A000615D59710134F7E7013002B070BDF8B516
:10E2B000064617461C46FFF7D8FFB368C0B21A6877
:10E2C0000444C0F105015568394422461846A84760
:10E2D000054601F0E1FDB061A8B2031B5842584168
:10E2E000F8BD10B5C368E0221A70C36800225A70E6
:10E2F00004468068E168036802225B689847A0686A
:10E300004FF0FF33E36303685B699847A0680368D5
:10E310005B6A984701F0C0FDC4E9060010BD0233F6
:10E3200030B598B20C46631A14F8015B9BB21DB16C
:10E33000431C155498B2F6E7C11A0A44191202F8A0
:10E34000021C02F8013C30BD38B50546806808B9AA
:10E35000002038BD03689B6A9847EC6B68B9002CB5
:10E36000F6D1A8686FF00203EB6303685B69984716
:10E37000A86803685B6A9847EAE7B4FA84F0400942
:10E38000E7E700002DE9FF470C9D9DF840A00446FB
:10E39000894617461E46FFF7D7FF8046002840F003
:10E3A000DF80A06803689B6A9847002840D001235B
:10E3B000E3826E4B029345F25443ADF80C300423D4
:10E3C0008DF80E30052302A91944E26811F8051CE6
:10E3D000D15401330C2BF6D1002D3DD09DF83830AF
:10E3E0009DF834205B0143F0040343EAC203DBB22F
:10E3F000BAF1000F01D043F002031FB1002E2DD15E
:10E4000043F08003E2681373638AE2681B1253735C
:10E41000E368628A9A73218A484605F09BF8238A4A
:10E42000113098421DD9A06803685B6A984797E04D
:10E43000A068216B0368A28E39B1DB699847012877
:10E44000B5D06FF00103E3638AE049499B6902910B
:10E45000E16A039102A9F1E72B46C9E743F0C00343
:10E46000D0E749460F23E2682046FFF758FF814670
:10E4700005B3218A284605F06DF809F10203184416
:10E48000238A9842CFD84B462946E2682046FFF7B8
:10E4900046FF218A05460F9805F05CF8238A023072
:10E4A00028449842BFD82B46E2680F992046FFF7D0
:10E4B00036FF814617B3218A384605F04BF809F13B
:10E4C00002031844238A9842ADD84B46E268394685
:10E4D0002046FFF724FF814686B1218A304605F0A9
:10E4E00039F809F102031844238A98429BD84B4615
:10E4F000E26831462046FFF712FF8146A9F1050385
:10E500009BB2E26810212046FFF7D1FE01F0C4FC67
:10E51000C4E906004FF47A75A06803689B689847C1
:10E5200058B901F0B9FCE369C01AA38A6B43984259
:10E53000F2D36FF00303E36375E70DF107012046A3
:10E54000FFF7ECFD04287FF46EAFE368DD785DB97A
:10E5500001F0A2FC4FF00108E06184F82050E5636F
:10E56000404604B0BDE8F087E5635CE700044D5128
:10E57000C489010010B586B0012404940B9C039457
:10E580009DF8284002949DF824400194089C009432
:10E59000FFF7F8FE06B010BD2DE9F3470446FFF77C
:10E5A000D3FE8046D0B101F077FC628A4FF47A73D3
:10E5B0005343E269821A9A42074603D8A269821A33
:10E5C00093421FD294F8203063B16FF00303A06828
:10E5D000E36303685B6A98474FF00008404602B067
:10E5E000BDE8F087E268C0211170E2685370A0684E
:10E5F000E168036802225B689847C4E90677012353
:10E6000084F82030A06803689B6898470028E5D00C
:10E610000DF107012046FFF781FD83B20646002B6E
:10E6200073D0E368E7611A7802F0F002302A57D11C
:10E63000626A002AD2D09DF807209918901C497868
:10E640001D5C05EB0125ADB2D11C19442A461844C6
:10E6500003F07EFFE3689DF807202B44134400225B
:10E660009A70E1689DF807C091F8009009F00609DA
:10E67000B2B20CF10200B9F1020F0844666A0CF163
:10E680000303A2EB0C0225D12B440CF1050C11F86D
:10E6900003E00B44521B93F801A06544053A29445A
:10E6A0000AEB0E2AB047E36840221A70E36883F849
:10E6B0000190E3681FFA8AFA4FEA2A229A70E36807
:10E6C00083F803A0A068E168036804225B689847A8
:10E6D000A76183E72B44033A521B1944B0477DE7F7
:10E6E000C02A0BD1D0221A70E36800225A70A068A9
:10E6F000E168036802225B6898476FE7D02A7FF4DD
:10E700006DAF002384F8203068E72046FFF71CFE39
:10E71000002808BF4FF0000860E770B590B00546CC
:10E720000E46FFF711FEE0B1304604F0D0FE312373
:10E73000C4B28DF80030A31C8DF801303B220023B9
:10E74000314601A88DF802308DF8034004F0EDFE4B
:10E750002B68221D5B68694628469847003018BF21
:10E76000012010B070BD2DE9F047044688461746D9
:10E770001D469DF82060FFF7E7FD50B3B4F81090F8
:10E780004046494604F0E6FEEB1D1844814520D37F
:10E7900041460523E2682046FFF7C1FD00211FFA2C
:10E7A00081FC4318AC459BB2E26801F1010104D23F
:10E7B00017F80CC002F803C0F1E7002EA3F105031F
:10E7C00020469BB214BF31213021BDE8F047FFF74E
:10E7D0006EBD0020BDE8F08773B505460E461446B1
:10E7E0006AB1018A104604F0B5FE03460022009289
:10E7F000314622462846FFF7B6FF02B070BD1346E9
:10E80000F4E7F7B505460E461F46144662B1018A85
:10E81000104604F09FFE03460097224631462846E4
:10E82000FFF7A1FF03B0F0BD1046F4E72DE9F04774
:10E830000446884692461E46FFF786FD002843D0D0
:10E84000218A404604F086FE9DF82030002BE368C4
:10E850000CBF3022312287B21A70B21C3A44012018
:10E8600002F07F01E568D20918BF41F08001431C26
:10E8700029545FFA80F9D2B941469BB2E26820463A
:10E88000FFF74DFDA368E1681A68D2F804800246DC
:10E890001846C04755468046B244AA4509D0A068EC
:10E8A00015F8011B03681B6898478044F5E7184674
:10E8B000D6E701F0F1FAA06109F1030038443044D1
:10E8C000A0EB080358425841BDE8F087F7B505466C
:10E8D0000E461F46144662B1018A104604F03AFE05
:10E8E00003460097224631462846FFF79FFF03B0B4
:10E8F000F0BD1046F4E7F8B505460E4614461F462F
:10E90000FFF722FD28B331460523EA682846FFF7C2
:10E9100006FD631F002F03440CBF30213121064642
:10E920009BB2EA682846FFF7A0FC0146A868EC689D
:10E930000368053E0E44C1F105015B68214432467F
:10E940009847044601F0A8FAA861A0B2831B584278
:10E950005841F8BD70B50D460446018A2846164652
:10E9600004F0F8FD45B3012E26D8238A09308342EE
:10E9700022D32046FFF7E8FCF0B1E38A01339BB2D3
:10E98000C3B1E382E38AE2681B125371E368E28A4F
:10E990009A71E268294607232046FFF7C0FCE36826
:10E9A0001E54031FE26820469BB28221BDE87040DE
:10E9B000FFF77DBC0123E4E7002070BD0022FFF7D4
:10E9C000C9BF70B50D460446018A284604F0C2FD51
:10E9D00025B3238A0930834220D32046FFF7B4FCB5
:10E9E000E0B1E38A01339BB2B3B1E382E38AE26828
:10E9F0001B125371E368E28A9A71E2682946072381
:10EA00002046FFF78CFC431FE26820469BB2A22100
:10EA1000BDE87040FFF74BBC0123E6E7002070BD66
:10EA200001638286704741627047C06B704738B59A
:10EA300004460D4609B9002038BD038A4BB9084683
:10EA400003F04AFDE060E0682582003018BF012035
:10EA5000F2E7C06804F018FC0028F3D1EBE70000EF
:10EA600070B50C4B00250446456040F8283B0E4627
:10EA700000F0C6FB4FF0FF33E363A660A563258279
:10EA80004FF480712046FFF7D2FF0F236382A382E9
:10EA9000204670BD3489010007B5002300931A4653
:10EAA0001946034800F0B4FB03B05DF804FB00BF57
:10EAB000DC0700208271054A417112680449B2FBEB
:10EAC000F1F14FF47A724A43C26070471800002097
:10EAD00040420F0038B504460D464079022101F04E
:10EAE000CBFB01F0D9F9A0F5FA60A060657438BDE0
:10EAF00070B505460E460024687901F0F7FBB04278
:10EB0000A3B206D1EA689A4204F10104F4D84FF0A6
:10EB1000FF33184670BD30B50D46D1B0044601F044
:10EB2000BBF93DB9A368C31AB3F5FA6F02D2207CD2
:10EB300051B030BD00250221A060256060792571AB
:10EB400001F09AFB012001F0DBF90121607901F06D
:10EB500093FB2946607901F0B7FBA379153B012BA4
:10EB600000F28C8040F24C40013800BF00BF00BF73
:10EB700000BF00BF00BF00BF00BF00BF00BF00BF9D
:10EB800000BF00BF00BF00BF00BF00BF00BF00BF8D
:10EB900000BF00BF00BF00BF00BF00BF00BF00BF7D
:10EBA00000BF00BF00BF00BF00BF00BF00BF00BF6D
:10EBB00000BF00BF00BF00BF00BF00BF00BF00BF5D
:10EBC00000BF00BF00BF00BF00BF00BF00BF00BF4D
:10EBD00000BF00BF00BF00BF00BF00BF00BFC3D168
:10EBE0006079022101F048FB607C00283BD00138AD
:10EBF00000BF00BF00BF00BF00BF00BF00BF00BF1D
:10EC000000BF00BF00BF00BF00BF00BF00BF00BF0C
:10EC100000BF00BF00BF00BF00BF00BF00BF00BFFC
:10EC200000BF00BF00BF00BF00BF00BF00BF00BFEC
:10EC300000BF00BF00BF00BF00BF00BF00BF00BFDC
:10EC400000BF00BF00BF00BF00BF00BF00BF00BFCC
:10EC500000BF00BF00BF00BF00BF00BF00BF00BFBC
:10EC600000BF00BFC3D172B600212046FFF740FFAE
:10EC7000013007D10020207462B659E7142001F05A
:10EC80003FF9ADE701212046FFF732FF0130F1D017
:10EC9000002500212046FFF72BFF01214DF805003C
:10ECA0002046FFF725FF0DEB05030835B5F5A07FDE
:10ECB0005860EED162B600225DF832500DEBC2030F
:10ECC000691C586801D0431C02D1002020742FE732
:10ECD000D1108542635C4FEA4303DBB202F10102CB
:10ECE00038BF43F00103282A6354E5D161782378C3
:10ECF00022790B44A1780B44E1780B44DBB29A42B1
:10ED0000E3D10120E2E700002DE9F8430D462DEDA7
:10ED1000028B11460446FFF7FEFE00287ED0A37941
:10ED20000B3B0B2B7AD8DFE803F0063F7979797932
:10ED3000797979796565A378E07808EE103A01066B
:10ED4000B8EE488A48BFFFEE007A00F00F0048BFD7
:10ED500037EEC88A02F0BCFD31A3D3E9002302F0EC
:10ED600021FE064618EE100A0F4602F0C3FD0B46C0
:10ED700002463946304602F05FFC03F00BF90346C9
:10ED80006DB102F0B7FD2AA3D3E9002302F00AFE19
:10ED9000254B002202F050FC03F0FCF80346BDECCA
:10EDA000028B1846BDE8F883E078A67800F00F00E3
:10EDB00002F08EFD1AA3D3E9002302F0F3FD07EE63
:10EDC000906AF8EE677A804617EE900A894602F05C
:10EDD00091FD02460B464046494602F02DFC03F0E9
:10EDE000D9F83206034648BF80F00043002DD6D044
:10EDF0001846C6E7A678E378300200F4FE401843D0
:10EE000007EE900AF8EEE77A17EE900A02F072FD2C
:10EE100003A3D3E9002302F0C5FDE0E7034BBEE7FF
:10EE20009A9999999999B93F000040400000C07F94
:10EE3000CDCCCCCCCCCCFC3FD0B50446FFF76BFEA0
:10EE400090B3A3790B3B0B2B2ED8DFE803F006061B
:10EE50002D2D2D2D2D2D2D2D1C1C607802F038FD13
:10EE600014A3D3E9002302F09DFD064620780F4647
:10EE700002F02EFD02460B463046394602F0DCFB1E
:10EE800003F088F8D0BD208840BA80B207EE900A1F
:10EE9000F8EEE77A17EE900A02F02CFD05A3D3E90D
:10EEA000002302F07FFDEBE70148EBE7AFF30080C2
:10EEB0000000C07F9A9999999999B93F10B5044675
:10EEC000C06803F011FBB4F90600002802DB002142
:10EED00001F0D2F9204610BD70B50546C0680E4657
:10EEE00003F002FBEC7C2A7C94420CBF0324042434
:10EEF00014FB06F4A4B2AC80204603F0EDFAE860FF
:10EF000028B12246002103F03CFB6E8070BDA88032
:10EF10006880FBE7F0B4FF29C1F38107C1F38112D8
:10EF2000C1F30115477401F003078CBF00210121D3
:10EF30000170C168C47C067CC2740574877461B1B9
:10EF4000A41B6142A2EB050561416A426A419142FC
:10EF500003D04188F0BCFFF7BFBFF0BC704738B5A5
:10EF6000437804460D4633B1B0F90600002802DBB1
:10EF7000002101F081F96378E5804BB12846012139
:10EF800001F07AF928460021BDE8384001F09CB92B
:10EF900038BD70B50E460021044641700172C16053
:10EFA000416119461546FFF7B5FF31462046FFF788
:10EFB00093FF20462946FFF7D2FF204670BD70B56B
:10EFC00040F2FA5404FB00F303F500431B14B3F5BD
:10EFD000FF7F98B222DAFE2BD8B242DDC0F1FE00EC
:10EFE000C5B20023FF204E1CC943C9B27043013291
:10EFF00001EB2020504300F47F4406FB03F006FBA6
:10F0000005F301EB202001EB232150434A43120278
:10F0100044EA102002F47F02104370BDB3F57F7FF5
:10F020000DDAB0F53F7FDBB28BBFC3F1FC030233D7
:10F03000D8B2DBB294BFFF20FF230025D3E7A04264
:10F0400011D040F2FA44A042DBB204D80433DDB25E
:10F050000020FF23C7E7C3F1FA03DBB20020FF253E
:10F06000C1E70023FBE700231846F8E770B5044624
:10F07000083015460E4600F0C3F8FF23064A84F810
:10F0800022300023266025712361A382C4E9062271
:10F090002384204670BD00BF5B8E01000161828227
:10F0A00070470000024B002908BF19468161704774
:10F0B0005B8E0100024B002908BF1946C1617047F1
:10F0C0005B8E01000184704773B50D4601690446EB
:10F0D000164639B92B4BC2685B689A4202D10020B0
:10F0E00002B070BDA28A002AF9D094F8223005F04F
:10F0F00007000341DB0738D515F47E7F08BF238C5A
:10F10000206804BF03F47E731D43036800292ED0DA
:10F110005B6A98470128E2D13C21206800F0CDF8D5
:10F120000A222946206800F024F9237933BB1649C6
:10F13000206800F0B5F8A169206800F0BAF8202135
:10F14000206800F0BAF8E169206800F0B2F823798D
:10F15000B3B90E49206800F0A3F83146206800F0EA
:10F16000A8F8206803689B6A98470120B8E7084917
:10F170000091E16801911B6A6946CAE70549D7E732
:10F180000549E7E7E40700203C89010042890100C6
:10F19000C4890100C77001004D89010008B5FFF75F
:10F1A00093FF08BD07B5002300931A46194603488C
:10F1B00000F02EF803B05DF804FB00BFE407002068
:10F1C0002DE9F84306460D46071D00F10709002406
:10F1D00017F8011B0A22284600F0E4F82E21804689
:10F1E000284600F06AF84F4540440444F0D10A2212
:10F1F000F179284600F0D6F82044BDE8F8830000F5
:10F20000024A026000224260704700BFC4890100C8
:10F2100030B58371034D9DF80C300560017142716A
:10F22000C37130BDC4890100014AC0E900217047A3
:10F23000C4890100024A02600A684260704700BF48
:10F24000C48901000B6843607047416070472DE935
:10F25000F04106460D4601EB02080C464445A4EB7E
:10F26000050707D0336814F8011B1B683046984720
:10F270000028F3D13846BDE8F08170B50446084651
:10F280000D4604F024F923680246294620465B68AF
:10F29000BDE87040184709B1FFF7EFBF0846704757
:10F2A00008B5FFF7F8FF08BD03688A685B6809685E
:10F2B000184708B5FFF7EFFF08BD03681B6818473C
:10F2C0000149FFF7DABF00BF1889010038B50546CC
:10F2D000FFF7E1FF04462846FFF7F2FF204438BD60
:10F2E00038B50546FFF7D7FF04462846FFF7E8FF85
:10F2F000204438BD70B58AB00D460AA9002301F834
:10F30000043D012A98BF0A22B5FBF2F402FB145611
:10F31000F3B2092E94BF30333733DBB2254601F800
:10F32000013D002CF0D1FFF7B6FF0AB070BD2DE90A
:10F33000F04107460E4615462AB90368C9B21B6854
:10F34000BDE8F04118470A2A05D1002905DBBDE8D0
:10F35000F041FFF7CFBFD2B2F9E72D21FFF7ADFFA4
:10F360002A46044671423846FFF7C4FF2044BDE8F0
:10F37000F081FFF7DCBF38B50546FFF7D8FF04463C
:10F380002846FFF79DFF204438BD10B42AB9036812
:10F390005DF8044B1B68C9B21847D2B25DF8044B44
:10F3A000FFF7A8BFFFF7F1BFFFF7EFBF2DE9F84F59
:10F3B00019460646104614461D469DF8287002F070
:10F3C0008BFD28B14C493046BDE8F84FFFF755BFDB
:10F3D00025F000494FF0FF32484B2046494602F0E5
:10F3E0007BFD48B94FF0FF32444B2046494602F0BE
:10F3F00055FD08B94249E6E74FF06042414B2046CF
:10F40000294602F05FFD08B13F49DCE74FF060425A
:10F410003E4B2046294602F037FD0028F4D1002259
:10F4200000232046294602F02FFDD0B12D21304681
:10F43000FFF743FF05F1004382461D463449DFF8DC
:10F44000D8904FF0000B00204FF000085FFA8BF3CC
:10F450009F4208D942464B4602F0CEFB0BF1010B0E
:10F46000F4E78246EAE722462B4602F0E5F80D462D
:10F47000044602F06FFD0A22014680463046FFF73F
:10F4800039FF8244A7B3404602F012FA02460B4607
:10F490002046294602F0CEF804460D4630461D4966
:10F4A000DFF87490FFF7E9FE4FF000088244013F57
:10F4B000FFB2FF2F1CD04B4642462046294602F0A1
:10F4C00071FA0D46044602F01DFD0A2201468346EC
:10F4D0003046FFF72CFF8244584602F0F9F9024605
:10F4E0000B462046294602F0A5F804460D46DEE705
:10F4F0005046BDE8F88F00BFC8890100FFFFEF7FCD
:10F50000CC890100FFFFEF41D0890100FFFFEFC16F
:10F510000000E03F0D810100000024409DF8001034
:10F520000091FFF743BF08B54022002103F029F8FE
:10F530000022C0E9102208BD026C10B5531C446CB7
:10F5400003F03F039C421CBF8154036410BD0023A1
:10F55000C0E910337047D0E9102393421FBFC25C4B
:10F56000013303F03F03436414BF10464FF0FF30F4
:10F570007047D0E91030181A48BF40307047D0E9C2
:10F580001023934214BFC05C4FF0FF307047036CF0
:10F59000406C013303F03F031B1A58425841704737
:10F5A0000649074A074B9B1A03DD043BC858D05055
:10F5B000FBDC00F037F8F0F743FE00006C8E010032
:10F5C00000000020A4020020FEE7FEE7FEE7FEE7C1
:10F5D000FEE7FEE7FEE7FEE7FEE7FEE7044B1868FE
:10F5E000421C04BF034B1878831F58425841704790
:10F5F00030010010E00F00F0074B1B78062B09D1FB
:10F60000064B1B68C3F30313033B032B02D8044AC6
:10F61000D05C704700207047E00F00F0E80F00F06A
:10F62000D889010008B5FFF7D9FF28B1654B664AB4
:10F630001B68C3F304231360FFF7DEFF10B1634BB5
:10F64000634A1A60FFF7CAFF28B1624B624A1B681F
:10F65000C3F342331360FFF7CFFF20B15F4AD36893
:10F6600023F08073D360FFF7B9FF40B14FF08043C0
:10F670000022C3F80C21C3F81021C3F83825FFF786
:10F68000BBFF10B1564B03221A60FFF7B5FF40B124
:10F69000544B05221A6001229A6700229A603F2289
:10F6A0005A60514B1A68511C0BBF504B504B1A7883
:10F6B0001B6802BF08331B68C3F30313062A4DD12E
:10F6C000033B032B03D84B4AD35C002B46D04FF0AF
:10F6D0008052494BD2F80414C3F82015D2F808140C
:10F6E000C3F82415D2F80C14C3F82815D2F8101456
:10F6F000C3F82C15D2F81414C3F83015D2F8181426
:10F70000C3F83415D2F81C14C3F84015D2F82014ED
:10F71000C3F84415D2F82414C3F84815D2F82814B5
:10F72000C3F84C15D2F82C14C3F85015D2F8301485
:10F73000C3F85415D2F83414C3F86015D2F838144D
:10F74000C3F86415D2F83C14C3F86815D2F8401415
:10F75000C3F86C15D2F84424C3F87025FFF73EFFB8
:10F7600028B1264B264A1B6803F04F031360FFF7AE
:10F7700035FF48B14FF08043D3F80024D20744BF8F
:10F780006FF00102C3F80024174B1B68062B09D148
:10F79000174B1B68033B022B81BF1A4A136843F4C3
:10F7A00080631360184AD2F8883043F47003C2F8BB
:10F7B0008830BFF34F8FBFF36F8F144B144A1A601A
:10F7C00008BD00BF240300104035014074C007404D
:10F7D0000DF0ADBA440200103C050040F0ED00E031
:10F7E000A00500401056004030010010E00F00F06E
:10F7F00034010010D489010000C0004058020010FC
:10F80000E40E00403C17004000ED00E0180000202E
:10F810000090D00310B5044600F03EFBE060236882
:10F820002046DB689847002808DA00F035FBE368DB
:10F83000C01AA3689842F2D34FF0FF3010BD2DE9F3
:10F84000F04180460D468F180C46BC42A4EB0506DD
:10F8500007D04046FFF7DEFF002802DB04F8010B6B
:10F86000F3E73046BDE8F0812DE9F843804689464C
:10F8700016461C467BB1D7181546BD42A5EB0604BB
:10F8800009D04046FFF7C6FF002804DB814502D0BF
:10F8900005F8010BF1E72046BDE8F88370B50D4689
:10F8A00009490446164600F0D1F92846FFF7B2FF91
:10F8B000002806DB864204D0C1B2204600F044FA9C
:10F8C000F3E7204670BD00BF1A8901000120704790
:10F8D00003681322DB69184770470369C3F81C15D6
:10F8E0000369D3F81C21002AFBD00022C3F81C2195
:10F8F0000120704710B490F95C30144C5909012272
:10F90000203103F01F0302FA03F344F821300369A6
:10F910005DF8044B0421C3F8081303695A600369B6
:10F92000DA6003690022C3F8002502694FF0FF3353
:10F93000C2F80C350269C2F814350269C2F80835FC
:10F9400002691430C2F81035FFF701BE00E100E093
:10F950001430FFF70EBE1430FFF711BE1430FFF75E
:10F96000FABD0000036990F85E2010B5C3F80C25BD
:10F97000036990F85D20C3F8142590F861200369AD
:10F98000012A01BF90F85F40C3F81045036990F861
:10F99000604006BFC3F8084503690022B1F5966FC1
:10F9A000C3F86C2569D9B1F5166F69D9B1F5965FC1
:10F9B00069D9B1F5165F68D9B1F5615F67D9B1F55D
:10F9C000964F66D9B1F5E14F65D9B1F5164F64D9B7
:10F9D000B1F5614F64D9B1F5963F64D9B1F5E13F16
:10F9E00063D9B1F5613F63D9364B994263D9B1F51B
:10F9F000E12F63D9B1F5612F94BF4FF070634FF0E1
:10FA000080530269C2F8243503690422C3F8002533
:10FA100001690023C1F808310169C1F81C3101698D
:10FA200001230B6001698B600169C1F8042390F91F
:10FA30005C20510902F01F0293406031224A42F8D3
:10FA4000213090F95C30002BBDBF03F00F0302F6AC
:10FA5000FC32D2189B18B5BF60236022137683F85E
:10FA6000002390F95C300122590903F01F0302FAC8
:10FA700003F3154A42F8213010BD4FF49E23C0E72E
:10FA80004FF41D23BDE7114BBBE7114BB9E7114BF9
:10FA9000B7E7114BB5E7114BB3E74FF41D03B0E7E0
:10FAA0004FF46B03ADE70E4BABE74FF0EB73A8E7FA
:10FAB0004FF06C73A5E74FF08063A2E74FF0E86367
:10FAC0009FE700BF90D0030000E100E000B013000A
:10FAD0000050270000F03A0000A04E0000C0750062
:10FAE00000903A012DE9F0411E4600254FF47A734B
:10FAF000C0E901530D4B044640F8143B17468846B5
:10FB0000FFF711FD0A4AC4F8108084F85C7052F8BF
:10FB1000263084F85D309DF8183052F8233084F890
:10FB20005E3084F861502046BDE8F081E489010030
:10FB30005489010010B50369D3F8082104464AB17D
:10FB4000D3F818151430C9B2FFF7F6FC2369002268
:10FB5000C3F8082110BD00000148FFF7EBBF00BF4C
:10FB6000EC07002007B5192300930222182303494C
:10FB70000348FFF7B7FF03B05DF804FB0020004027
:10FB8000EC07002010B5044628B103F049FB90FBB8
:10FB9000F4F303FB1404204610BD884210B504465C
:10FBA00003DA081AFFF7EEFF0444204610BD10B533
:10FBB000029C401AE41A6043521A90FBF2F0184477
:10FBC00010BD10B50446006802F08EFC204610BD42
:10FBD00010B50446006808B102F086FC00232360DB
:10FBE000C4E9013310BD38B504460D460068013143
:10FBF00003F04AFB10B1C4E90005012038BD0368D9
:10FC000010B5044623B143688B4201D3012010BDD7
:10FC10002046FFF7E8FF0028F9D0A368002BF5D1B4
:10FC200022681370F2E770B50E4611460446154679
:10FC3000FFF7E5FF20B92046FFF7CAFF204670BD59
:10FC4000A5603146206803F01EFCF7E738B50023B5
:10FC50000446C0E9003383600D4639B1084603F01D
:10FC600036FC294602462046FFF7DDFF204638BD18
:10FC700038B5054608460C4603F029FC21460246E5
:10FC80002846BDE83840FFF7CEBF38B505460068C6
:10FC90000C4668B16A688B689A4207D3096803F01A
:10FCA000F2FBA368AB600023A36038BD02F01CFC2C
:10FCB00023682B6063686B60A368AB600023C4E9B2
:10FCC0000033F1E7884210B50B46044604D00968BA
:10FCD00021B19A68FFF7A7FF204610BDFFF778FF14
:10FCE000FAE710B500230446C0E900338360FFF74C
:10FCF000E9FF204610BD884210B5044601D0FFF749
:10FD0000C4FF204610BD10B5044619B1FFF7B0FF7F
:10FD1000204610BDFFF75CFFFAE770B505460E46BA
:10FD200009B9002070BD6AB1846814442146FFF708
:10FD300066FF0028F5D02868AB683146184403F008
:10FD4000A2FBAC600120EDE707B500238DF804109D
:10FD5000012201A98DF80530FFF7DFFF03B05DF840
:10FD600004FB10B58A6809680446FFF7D6FF10B98E
:10FD70002046FFF72DFF204610BD826808B53AB92E
:10FD800021B10878B0FA80F0400900E0012008BDF8
:10FD9000006809B90078F5E703F06BFBF2E78842E9
:10FDA00070B515D083688A6893420FD183B1046817
:10FDB0000D68013C14F8010F50B104F09DFB06469C
:10FDC00015F8010B04F098FB8642F3D0002070BDBB
:10FDD0000120FCE783688B4201D9006818B9034809
:10FDE0000023037070470844704700BF500800208C
:10FDF0008368934210B506D90468A01803F02CFB61
:10FE000008B1001B10BD4FF0FF30FBE70022FFF7E9
:10FE1000EFBFF8B583689342054602D84FF0FF3034
:10FE2000F8BD0368541C00221F5D1A550668304651
:10FE300003F09CFB37550028F0D02B68C01AEFE781
:10FE40008268013AFFF7E5BF2DE9F0419A420E467C
:10FE50001F460F4988BF13461546804684BF3D465E
:10FE60001F46FFF7F3FEB468AC420DD9BC4228BF71
:10FE70003C46336800221F5D1A55316840462944CC
:10FE8000FFF741FF33681F554046BDE8F08100BFD2
:10FE90001A890100FEE700000A4B19680A4B30B5C9
:10FEA000D3F804050C060D0A44EA00024FF47A71F7
:10FEB0002B46A2FB014501FB0355E00B40EA454000
:10FEC00030BD00BF5408002000100140094B1968E4
:10FED000094B30B5D3F804050D0A0C06074944EA6E
:10FEE00000022B46A2FB014501FB0355E00B40EA53
:10FEF000454030BD540800200010014040420F0032
:10FF000038B5044648B1FFF7C7FF054600F01AF8B8
:10FF1000FFF7C2FF401BA042F8D338BD074B0022B9
:10FF2000C3F8042182B0D3F80431054A0193019B40
:10FF300013680133DBB2136002B070470010014058
:10FF400054080020704770B58AB061B1931E222B0F
:10FF500020D801AB1D4648B9AB4207D00A46AB4298
:10FF600013D80023137008460AB070BDB0FBF2F43A
:10FF700002FB1406092E204603F10103F4B294BFDC
:10FF80003034573403F8014CE5E713F8010D02F85B
:10FF9000010BE4E70021E6E77047000008B500F038
:10FFA00017F8FFF7F9FF0120FFF7AAFFF5F798F917
:10FFB000034CF5F797F9002CFBD0AFF30080F8E77E
:10FFC0000000000002F088BA02F086BA02F08CBA93
:10FFD0002A4BE02283F811234FF40032C3F880212A
:10FFE0001A604FF080430122C3F818259A6003F588
:10FFF00088330021C3F808150221C3F80413C3F89D
:020000021000EC
:1000000044131A604FF01023D3F80022002A03DBB8
:10001000D3F80432002B2FDA194B0122C3F8042540
:10002000D3F80024002AFBD04FF010221521C2F88B
:100030000012D3F80024002AFBD04FF01023152221
:10004000C3F804220E4B1A46D3F800140029FBD043
:100050000021C3F80415D2F80034002BFBD0BFF305
:100060004F8F0849084BCA6802F4E0621343CB6023
:10007000BFF34F8F00BFFDE7704700BF00E100E016
:1000800000E0014000ED00E00400FA05192837B552
:100090000CD84B4B53F82030052B00F0828007D84A
:1000A000032B12D07BD8022B00F08180002074E05B
:1000B0001D2B78D003D81C2BF8D1052206E01E2B6F
:1000C00073D01F2BF2D1082200E002223D4B1968A9
:1000D00008296EDD0A296FDD0D29B5BF0C240E2419
:1000E000022303233848C0F8F0350123C0F8003557
:1000F00000200546030103F1804303F5E04301308E
:100100000828C3F81455C3F81055F3D12F4B1868BD
:100110002F4B1B6800021B0303F4805300F4E060C4
:100120001843294BC3F81805C3F81425C3F8102544
:100130000DF10602C3F82C260122C3F830261A60FE
:10014000D3F80021002AFBD00022C3F800210122AD
:100150005A601D4B1A46D3F804010028FBD000203A
:10016000C3F8040101209860D2F81431002BFBD0B1
:100170000023C2F81431BDF906209A42124AB8BFD2
:10018000ADF80630A142C2F80035BDF9060004D032
:1001900035BF611A091BC840884003B030BD032237
:1001A00094E7042292E7062290E707228EE70122D5
:1001B0008CE70824002395E70A24012392E700BF77
:1001C0005489010028000020007000402C0000200D
:1001D00060080020192830B53CD8224B53F8200085
:1001E000214B00221D4653F82240B4F1FF3F32D18B
:1001F0001E4C45F822006FEA41411D4D1D4B2468FD
:1002000053F822306FEA514125F81210012101FA0A
:1002100004F4C3F86005013CC3F8640505EB420231
:10022000C3F86805C3F86C050020C3F80015C3F8CF
:100230000C05C3F80405C3F80845C3F81405C3F852
:100240001005C3F82025C3F82415C3F82815C3F8F2
:100250002C05996030BD8442CAD00132032AC2D134
:10026000F8E700BF548901001C0000203000002086
:10027000580800200C8A010019280FD8114B53F898
:10028000203003290AD8DFE801F002160A1003F52E
:10029000E0734FF0A042002142F82310704703F5AD
:1002A000E0734FF0A0420C21F6E703F5E0734FF046
:1002B000A0420421F0E703F5E0734FF0A0420321D0
:1002C000EAE700BF5489010019280CD8064B53F8FF
:1002D0002020012393404FF0A04211B9C2F80C3501
:1002E0007047C2F8083570475489010019289FBF2C
:1002F0004FF0A043054AD3F8103552F820009ABFBA
:1003000023FA00F000F0010000207047548901003A
:1003100038B50025057329B90B4B0C4A0C4825212B
:1003200001F088FE01600B4951F82220027151F85A
:10033000233083719DF8103051F82330437102232C
:10034000C371856038BD00BF188A01007B8A010037
:10035000268A010054890100037B23B94373837308
:10036000036101230373704784B00DF1100C0CE995
:100370000E009DF80810026800230129C2F800351C
:10038000039B12D00BD303290CD0C2F85435019B28
:10039000C2F824350123C2F8003504B0704743F099
:1003A0000203F2E743F00403EFE743F00603ECE750
:1003B00010B5FFF7D1FF03688279C3F808254279A9
:1003C000C3F80C250279C3F81025034BBDE8104093
:1003D0000ECBFFF7C9BF00BF7808002010B485B06E
:1003E00001AC84E80E0094E80E0005B05DF8044B03
:1003F000FFF7BABF70470368C3F81C15D3F808218C
:10040000002AFBD0D3F818050022C3F80821C0B297
:100410007047000007B5094B09490A484FF0804270
:100420001A6000229A6002221A710B2300930C2298
:100430000D23FFF76DFF03B05DF804FB7808002083
:1004400000300240640800200B460146184601F0C7
:100450001BBE0000C0F3C7537F3B162B024605DCD2
:10046000002B04DB0348184122EA0000704700F02B
:1004700000407047FFFF7F002DE9F04FDFF82C931D
:100480008DB006460F4614461D4600F095F999F9C1
:100490000080B8F1FF3FCDE9000136D022462B465F
:1004A0002046294601F018FD834670BB32463B4684
:1004B0003046394601F010FD8246002840F0A28007
:1004C000304639460022002301F0D4FC10B300224C
:1004D00000232046294601F0CDFC8346002867D042
:1004E0009FEDA77B0122AC4BCDF828A00292CDE96D
:1004F0000467CDE906458DED087B0393B8F1000F45
:1005000041D09FEDA17B8DED007BDDE900010DB0B9
:10051000BDE8F08FDDE9000100F066FF80460028AD
:1005200000F08D804FF0000A4FF0000BDDE9000174
:1005300052465B4601F09EFC0028E6D03046394624
:1005400000F052FF0028E0D02046294600F04CFF82
:100550000028DAD099F900308F4A03920421002252
:10056000022BCDE90467CDE90645CDE908AB029140
:100570000A9203D002A800F03DFF50B901F092FDAD
:100580002223036005E002A800F034FF002800F0F9
:100590009B800A9B1BB101F085FD0A9B03609DEDCA
:1005A000087B8DED007BDDE900010DB0BDE8F08F2B
:1005B0002046294600F018FF0028A6D0002200237C
:1005C0002046294601F060FC00289ED0724A99F925
:1005D0000030CDF828B00121CDE90467CDE906450A
:1005E000CDE90212002B74D06C490020022BCDE91A
:1005F000080172D101F056FD212303600A9B002BF4
:10060000CDD0C8E7002200232046294601F032FC65
:1006100000283FF47AAF624B5F49CDF828B0002242
:100620000120B8F1020FCDE904670290CDE906453B
:10063000CDE908230391A6D1CDE9002365E7304633
:10064000394600F0D1FE00283FF46CAF2046294621
:1006500000F0CAFE00283FF465AFDDE90023104634
:10066000194601F039FC99F900A000286BD1032349
:10067000DFF824C10A902946204602930022494B04
:10068000CDF80CC0CDE90645CDE9046701F08AF943
:1006900004460D46BAF1000F25D1DFF814B14FF032
:1006A000604A0022002330463946CDE908AB01F00C
:1006B000EBFB38BB02A800F09DFE00289ED101F0A4
:1006C000F1FC2223036099E701F0ECFC2123036095
:1006D0005FE79FED2B7B8DED087B02A800F08AFE83
:1006E00000288BD186E79FED2A7B0022002330462D
:1006F00039468DED087B01F0C7FBA0B9BAF1020FB6
:10070000DDD0D7E72046294600F07CFE22462B4666
:1007100001F0B0FBA0B9244B99F900A04FF0604262
:10072000CDE90823EAE72046294600F06BFE224681
:100730002B4601F09FFB18B9184B0022CDE9082386
:1007400099F900A0DAE70122134BCDF82880029234
:10075000CDE90467CDE906450393BAF1000FB8D09F
:10076000002200231046194601F046FABAF1020FA2
:10077000CDE908013FF43EAFAFE700BFAFF3008023
:100780000000000000000000000000000000F03F3A
:10079000000000000000F07FB88A01000000F0FFB8
:1007A0000000F03F0000E03FFFFFEFC734000020F3
:1007B000FFFFEF47000000002DE9F04F23F0004558
:1007C00055EA020493B00DD06B4E21F00044B442C0
:1007D0000F4682460BDD04F1404404F5801454EAD0
:1007E0000A0350D16549002013B0BDE8F08F9B4645
:1007F000944647D0B542EEDC5F4EB5425DD0002F47
:1008000080468946CDE900235BDB0026BCF1000F62
:100810000ED1594B9D423FD0584B9D4200F08880ED
:10082000BBF1804F00F09C80554B9B4500F0B88396
:100830004046494600F0D4FDBAF1000F06D1002C25
:1008400059D04E4B27F040429A4254D0FF0F013FFF
:1008500056EA070373D04B4B9D4240F39B8003F154
:1008600004739D4240F33E84474B9C4272DDBBF1D2
:10087000000F72DD3EA3D3E900231046194601F0B4
:1008800091F8B1E728B1414813B0BDE8F04F00F04E
:10089000B3BDA542F7DCAFE704F1404303F5801395
:1008A00053EA0A039ED0384B9C4240F38383BBF14A
:1008B000000F52DBDDE9000196E7BCF1000F9ED08E
:1008C00089E7334B9D4231DCA3F154739D429CDD9B
:1008D0002B15A3F2FF33142B40F3A583C3F134038C
:1008E0002CFA03F202FA03F363458ED102F00102FF
:1008F000C2F102068AE7BBF1000F05DA02460B4699
:1009000000201E4901F078F9002FBFF66DAF04F109
:10091000404404F5801454EA060300F03F84012E9D
:100920007FF462AF01F1004319465DE702266DE7EF
:10093000BBF1000FC0F248834046494654E74246A7
:100940004B461046194600F075FE02460B4601F074
:1009500053F949E7BBF1000F8CDB0020002143E78E
:1009600042464B464046494601F01CF83CE700BF72
:100970009C7500883CE4377E0000F07F0000F03F6B
:100980000000E03F0000E041FFFFEF3FBC8A0100B4
:10099000FFFF3F43B4F5801F80F261830022D24BFA
:1009A00001F000F86FF0340C0C462315CF4DC4F362
:1009B0001302A3F2FF3342F07F546344AA420B9325
:1009C00044F4401440F33F83C94B9A4240F30484FB
:1009D0009FEDAF7B8DED087B8DED107B9FEDAE7BAA
:1009E0000B9B8DED067B01330B93A4F58014002542
:1009F000DDE906232146824600F01CFEA346DDE920
:100A000006238046894650462146CDE90CAB00F0CE
:100A100013FE02460B460020B64901F0EDF80A46E7
:100A20000146CDE90E12134649460246404600F003
:100A3000B9FF631043F0005382468B4603F5002351
:100A40008C46CDE904AB5919D3460023CDE902BC4D
:100A50000293DDE902AB002004460D4602460B4638
:100A60005046594600F09EFF02460B464046494616
:100A700000F0E0FDDDE90623804689462046294650
:100A800000F0D8FD02460B46DDE90C0100F0D2FD76
:100A900052465B4600F086FF02460B4640464946FA
:100AA00000F0C8FDDDE90E2300F07CFFDDE9044520
:100AB000CDE9060122462B462046294600F072FF6A
:100AC00077A3D3E9002304460D4600F06BFF76A31D
:100AD000D3E9002300F0B0FD22462B4600F062FF70
:100AE00073A3D3E9002300F0A7FD22462B4600F0B4
:100AF00059FF71A3D3E9002300F09EFD22462B4647
:100B000000F050FF6EA3D3E9002300F095FD2246CC
:100B10002B4600F047FF6CA3D3E9002300F08CFDC7
:100B20002246804689462B462046294600F03AFF59
:100B300002460B464046494600F034FF5246044602
:100B40000D465B46DDE9040100F076FDDDE9062394
:100B500000F028FF22462B4600F06EFD52468046EC
:100B600089465B465046594600F01CFF0022624B06
:100B7000CDE90C0100F060FD42464B4600F05CFD03
:100B800002980D46044622462B465046594600F030
:100B900009FF002282468B46574B2046294600F02B
:100BA00049FDDDE90C2300F045FD02460B464046B9
:100BB000494600F03FFDDDE9042300F0F3FE224644
:100BC000804689462B46DDE9060100F0EBFE024631
:100BD0000B464046494600F02FFD804689460246B6
:100BE0000B465046594600F027FD029838A3D3E93A
:100BF000002304460D4600F0D5FE5246CDE904011F
:100C00005B462046294600F015FD02460B4640464D
:100C1000494600F00FFD30A3D3E9002300F0C2FEE7
:100C20002FA3D3E90023804689462046294600F0B9
:100C3000B9FE02460B464046494600F0FDFCDDE9A0
:100C4000102300F0F9FC80460B98894600F040FE26
:100C5000424682468B464B46DDE9040100F0ECFC3F
:100C6000DDE9082300F0E8FC52465B4600F0E4FCB6
:100C7000029852465B4604460D4600F0DBFCDDE977
:100C8000082300F0D7FCDDE9042337E0AFF3008050
:100C90000000000000000000000000000000F03F25
:100CA000EF4E454A287ECA3F65DBC9934A86CD3F51
:100CB00001411DA96074D13F4D268F515555D53F37
:100CC000FFAB6FDBB66DDB3F033333333333E33FCF
:100CD000000000E009C7EE3FFD033ADC09C7EE3F24
:100CE000F5015B14E02F3EBE000040438E980300E8
:100CF00079B60B000000F03F0000084000F09AFCBD
:100D00000B4602464946404600F094FC013E56EA36
:100D1000070382468B4600F05E819FEDD37B8DED0D
:100D2000047BDDE9001200230E461746CDE9026779
:100D30000293DDE9026708463B461146324600F061
:100D400079FC22462B4600F02DFEDDE9002380468B
:100D500089465046594600F025FE02460B4640465D
:100D6000494600F069FC3246804689463B462046AB
:100D70002946CDE9008900F015FE0B4602460646DD
:100D80000F464046494600F057FCD14B9942044675
:100D90000D468A4640F3248101F13F4303F5E00309
:100DA000034340F0FF81B2A3D3E90023DDE9000152
:100DB00000F042FC3246804689463B4620462946A2
:100DC00000F038FC02460B464046494601F07AF8EE
:100DD000002840F0E781A8464FEA2853A3F2FE32EC
:100DE0004FF4801313415344C3F30A52B94DA2F296
:100DF000FF321541C3F3130423EA05010020C2F1B9
:100E0000140B44F48014BAF1000F02460B4644FA66
:100E10000BFB30463946B8BFCBF1000B00F00AFCA3
:100E200006460F463246DDE900013B4600F004FC71
:100E30004FEA0B5A0D4600248FA3D3E90023204626
:100E4000294600F0AFFD3246804689463B462046A3
:100E5000294600F0EFFB02460B46DDE9000100F0F9
:100E6000E9FB87A3D3E9002300F09CFD86A3D3E927
:100E7000002306460F462046294600F093FD024611
:100E80000B463046394600F0D7FB06460F46024671
:100E90000B464046494600F0CFFB42464B460446CF
:100EA0000D4600F0C7FB02460B463046394600F0BF
:100EB000C1FB2246804689462B462046294600F043
:100EC00071FD73A3D3E9002306460F4600F06AFDC7
:100ED00071A3D3E9002300F0ADFB32463B4600F09E
:100EE00061FD6FA3D3E9002300F0A6FB32463B4629
:100EF00000F058FD6CA3D3E9002300F09BFB3246C1
:100F00003B4600F04FFD6AA3D3E9002300F094FBB9
:100F100032463B4600F046FD02460B462046294637
:100F200000F088FB06460F4602460B46204629463F
:100F300000F038FD0022CDE900014FF0804330463B
:100F4000394600F077FB02460B46DDE9000100F070
:100F500053FE424606460F464B462046294600F0C1
:100F600021FD42464B4600F067FB02460B463046E9
:100F7000394600F05FFB22462B4600F05BFB024641
:100F80000B460020544900F055FB8A44BAF5801FF7
:100F9000C0F232815146DDE9042300F003FD23E471
:100FA000002FFFF645AC4046494613B0BDE8F04F70
:100FB00000F056B9BBF1000FBFF6CFACDDE900344D
:100FC000184604F100410FE442464B4600204249D6
:100FD00000F012FE08E49FED387B8DED047BA0E667
:100FE0003E4B21F00048984540F3EA803C4B0B44CF
:100FF00003430AD132463B4600F01CFBDDE90023E7
:1010000000F056FF00283FF4E7AEDDE904012CA311
:10101000D3E9002300F0C6FC29A3D3E9002300F0A4
:10102000C1FCFFF7E1BBBCF1000F40F0D280C3F17F
:10103000140345FA03F202FA03F3AB4200F0E08036
:101040006646FFF7E9BB9FED207B8DED087B8DEDBC
:10105000107B9FED057B00258DED067BC8E44FF0EE
:10106000000CA2E4AFF30080000000000000F03F9D
:10107000FE822B654715973C00000000432EE63F9B
:10108000EF39FAFE422EE63F396CA80C615C20BEB7
:10109000D0A4BE726937663EF16BD2C541BDBB3E7E
:1010A0002CDE25AF6A56113F93BDBE166CC1663F5C
:1010B0003E5555555555C53F000000000000F0BF96
:1010C00059F3F8C21F6EA5010000000000000000E7
:1010D000FFFF8F40FFFF0F000000F03FFFCB90406D
:1010E00000346F3F5A4B9C427FF734AC594B9C42C3
:1010F0003FF7BDAB0022574B00F09CFA44A3D3E965
:10110000002304460D4600F04DFC43A3D3E9002321
:1011100082468B462046294600F044FC0022CDE959
:1011200002014D4B2046294600F03CFC02460B468E
:101130003BA1D1E9000100F07DFA22462B4600F0E8
:1011400031FC02460B460020444900F073FA224667
:10115000804689462B462046294600F023FC02465D
:101160000B464046494600F01DFC2FA3D3E900235F
:1011700000F018FC02460B46DDE9020100F05AFAC5
:1011800002460B46804689465046594600F054FABE
:10119000002004460D4652465B46AFE502460B462C
:1011A000FFF7CFBBDDE9040121A3D3E9002300F061
:1011B000F9FB1FA3D3E9002300F0F4FBFFF714BBF6
:1011C000264B98453FF708AEDDE902239246934649
:1011D00031E60026FFF72CBB9FED177B8DED087BDA
:1011E0009FED177B8DED107B9FED177B4FF48025D6
:1011F0008DED067BFFF7FCBB5A4600F091F9CAE67D
:1012000002F00102C2F10206FFF706BBAFF3008055
:10121000000000604715F73F44DF5DF80BAE543E19
:10122000555555555555D53FFE822B654715F73F0A
:101230009C7500883CE4377E0000004003B8E23F24
:1012400006D0CF43EBFD4C3E000000000000F83F0D
:10125000FEFFEF3F0000F03F0000D03F0000E03F06
:101260005E4A8A432DE9F04104460D4600F0958020
:1012700000290B460646844656DD0F1500F0A58072
:10128000C3F31303A7F2FF3743F480134FEADC7272
:10129000F80702EB43034FEA4C0504D5ED0F05EBCD
:1012A00043034FEA8C0500267F10B44616224FF404
:1012B00000110CEB010098424FEAD5744FEA450546
:1012C00003DC1B1A00EB010C0E44013A04EB430350
:1012D0004FEA5101EDD11046964620244FF00042CE
:1012E00009E051D05B00013C03EBD5734FEA520299
:1012F0004FEA450537D0634502EB0E01F1DD0029C9
:1013000001EB020E0ADBE046A3EB0C03A94288BF07
:1013100003F1FF336D1A1044C446E3E7BEF1000F3A
:10132000F1DB0CF10108EFE721F00042024329D084
:10133000002942D10146CA0A153B4905002AFAD0C4
:1013400012F4801001D044E060465200D40200F153
:10135000010CF9D5CCF1200401FA0CFCE1401F1A74
:1013600041EA02038CE72B4321D14408731003F1B7
:101370007F53F20703F5001348BF44F0004403EB2A
:1013800007512046BDE8F081A942ABD8002901EB06
:10139000020EC3DB98460023BCE702460B4600F072
:1013A00001FB22462B4600F047F9BDE8F081411CC5
:1013B00016BF421C01365408D8E7024600F03AF93D
:1013C00002460B4600F018FCDCE71A4631463B4665
:1013D000B6E78C4620244FF0FF30BFE70000F07FD7
:1013E00021F000431946704741F0004101F580109B
:1013F000C00F70470020704700200149704700BFB0
:101400000000F87F2DE9F041C1F30A57A7F2FF353C
:10141000132D82B002460B460C464FEAD1780646A1
:1014200033DC002D4EDB3C49294103EA0100104327
:1014300026D049080B4052EA03060CD04FF4802313
:10144000132D24EA010143FA05F444EA01040CBF18
:101450004FF000460026314901EBC8082346D8E981
:10146000004532462046294600F0E6F8CDE9000165
:1014700022462B46DDE9000100F0DCF802460B466F
:101480001046194602B0BDE8F081332D07DDB5F5F1
:10149000806FF5D100F0D0F802460B46F0E7A7F2D6
:1014A00013474FF0FF31F9400842E9D0490808429C
:1014B000D1D04FF0804320EA010143FA07F741EA17
:1014C0000706C8E721F000410143D9D0C3F3130157
:1014D00001434E420E43114D5C0C360B640406F47E
:1014E000002305EBC80243EA0401D2E900450B469C
:1014F00002462946204600F09FF8CDE90001224629
:101500002B46DDE9000100F095F821F0004102468C
:1015100041EAC873B4E700BFFFFF0F00C08A0100B3
:10152000F8B5C1F30A5304460D460E4617460BBBE9
:1015300021F00046034633431BD0354B002200F018
:1015400031FA344B9F4204460D4635DBC1F30A5352
:101550000E46363B3B4440F2FE72934232DC002B97
:1015600011DD26F0FF4626F4E00646EA0355204644
:101570002946F8BD40F2FF729342EBD102460B467A
:1015800000F05AF8F8BD13F1350F28DA4CF2503359
:101590009F4222462B460ADD19A1D1E9000100F045
:1015A0003DF817A3D3E9002300F0FCF9F8BD16A11C
:1015B000D1E9000100F032F813A3D3E9002300F0D1
:1015C000F1F9F8BD22462B460DA1D1E9000100F04A
:1015D00025F80BA3D3E9002300F0E4F9F8BD26F0C9
:1015E000FF4626F4E006363346EA035520462946F0
:1015F0000022094B00F0D6F9F8BD00BFAFF3008020
:101600009C7500883CE4377E59F3F8C21F6EA50133
:1016100000005043B03CFFFF0000903C03F000434B
:1016200021F0004242EA0301704700BF81F000410F
:1016300002E000BF83F0004330B54FEA41044FEAB7
:10164000430594EA050F08BF90EA020F1FBF54EA52
:10165000000C55EA020C7FEA645C7FEA655C00F0EE
:10166000E2804FEA5454D4EB5555B8BF6D420CDDBF
:101670002C4480EA020281EA030382EA000083EA42
:10168000010180EA020281EA0303362D88BF30BDE2
:1016900011F0004F4FEA01314FF4801C4CEA113138
:1016A00002D0404261EB410113F0004F4FEA033397
:1016B0004CEA133302D0524263EB430394EA050F22
:1016C00000F0A780A4F10104D5F1200E0DDB02FA91
:1016D0000EFC22FA05F2801841F1000103FA0EF225
:1016E000801843FA05F359410EE0A5F120050EF1EB
:1016F000200E012A03FA0EFC28BF4CF0020C43FA1C
:1017000005F3C01851EBE37101F0004507D54FF028
:10171000000EDCF1000C7EEB00006EEB0101B1F578
:10172000801F1BD3B1F5001F0CD349085FEA3000BE
:101730004FEA3C0C04F101044FEA445212F5800FC9
:1017400080F09A80BCF1004F08BF5FEA500C50F166
:10175000000041EB045141EA050130BD5FEA4C0C49
:10176000404141EB010111F4801FA4F10104E9D1D2
:1017700091F0000F04BF01460020B1FA81F308BFC9
:101780002033A3F10B03B3F120020CDA0C3208DD95
:1017900002F1140CC2F10C0201FA0CF021FA02F170
:1017A0000CE002F11402D8BFC2F1200C01FA02F1E0
:1017B00020FA0CFCDCBF41EA0C019040E41AA2BF05
:1017C00001EB0451294330BD6FEA04041F3C1CDACD
:1017D0000C340EDC04F11404C4F1200220FA04F0ED
:1017E00001FA02F340EA030021FA04F345EA030197
:1017F00030BDC4F10C04C4F1200220FA02F001FA59
:1018000004F340EA0300294630BD21FA04F02946DA
:1018100030BD94F0000F83F4801306BF81F4801173
:101820000134013D4EE77FEA645C18BF7FEA655CE6
:1018300029D094EA050F08BF90EA020F05D054EAB8
:10184000000C04BF1946104630BD91EA030F1EBFBD
:101850000021002030BD5FEA545C05D140004941C1
:1018600028BF41F0004130BD14F580043CBF01F5B4
:10187000801130BD01F0004545F0FE4141F470019A
:101880004FF0000030BD7FEA645C1ABF1946104675
:101890007FEA655C1CBF0B46024650EA013406BF76
:1018A00052EA033591EA030F41F4002130BD00BF35
:1018B00090F0000F04BF0021704730B54FF48064F2
:1018C00004F132044FF000054FF0000150E700BF73
:1018D00090F0000F04BF0021704730B54FF48064D2
:1018E00004F1320410F0004548BF40424FF00001BF
:1018F0003EE700BF42004FEAE2014FEA31014FEA02
:1019000002701FBF12F07F4393F07F4F81F0605150
:10191000704732F07F4208BF704793F07F4F04BF9B
:1019200041F40021704730B54FF4607401F0004578
:1019300021F000411CE700BF50EA010208BF7047D8
:1019400030B54FF000050AE050EA010208BF7047C9
:1019500030B511F0004502D5404261EB41014FF432
:10196000806404F132045FEA915C3FF4D8AE4FF03A
:1019700003025FEADC0C18BF03325FEADC0C18BF1D
:10198000033202EBDC02C2F1200300FA03FC20FA6E
:1019900002F001FA03FE40EA0E0021FA02F11444BB
:1019A000BDE600BF70B54FF0FF0C4CF4E06C1CEAD4
:1019B00011541DBF1CEA135594EA0C0F95EA0C0F45
:1019C00000F0DEF82C4481EA030621EA4C5123EAB8
:1019D0004C5350EA013518BF52EA033541F48011E7
:1019E00043F4801338D0A0FB02CE4FF00005E1FB9A
:1019F00002E506F00042E0FB03E54FF00006E1FBE4
:101A000003569CF0000F18BF4EF0010EA4F1FF0426
:101A1000B6F5007F64F5407404D25FEA4E0E6D4166
:101A200046EB060642EAC62141EA55514FEAC52077
:101A300040EA5E504FEACE2EB4F1FD0C88BFBCF5F3
:101A4000E06F1ED8BEF1004F08BF5FEA500E50F1A4
:101A5000000041EB045170BD06F0004646EA01016A
:101A600040EA020081EA0301B4EB5C04C2BFD4EB9C
:101A70000C0541EA045170BD41F480114FF0000E95
:101A8000013C00F3AB8014F1360FDEBF002001F003
:101A9000004170BDC4F10004203C35DA0C341BDC7D
:101AA00004F11404C4F1200500FA05F320FA04F04F
:101AB00001FA05F240EA020001F0004221F0004183
:101AC00010EBD37021FA04F642EB06015EEA430EF6
:101AD00008BF20EAD37070BDC4F10C04C4F1200526
:101AE00000FA04F320FA05F001FA04F240EA0200D9
:101AF00001F0004110EBD37041F100015EEA430EAA
:101B000008BF20EAD37070BDC4F1200500FA05F2C9
:101B10004EEA020E20FA04F301FA05F243EA020348
:101B200021FA04F001F0004121FA04F220EA020057
:101B300000EBD3705EEA430E08BF20EAD37070BD9D
:101B400094F0000F0FD101F00046400041EB01017D
:101B500011F4801F08BF013CF7D041EA060195F05F
:101B6000000F18BF704703F00046520043EB030319
:101B700013F4801F08BF013DF7D043EA0603704706
:101B800094EA0C0F0CEA135518BF95EA0C0F0CD011
:101B900050EA410618BF52EA4306D1D181EA030157
:101BA00001F000414FF0000070BD50EA410606BF51
:101BB0001046194652EA430619D094EA0C0F02D196
:101BC00050EA013613D195EA0C0F05D152EA0336DB
:101BD0001CBF104619460AD181EA030101F00041F9
:101BE00041F0FE4141F470014FF0000070BD41F042
:101BF000FE4141F4780170BD70B54FF0FF0C4CF41C
:101C0000E06C1CEA11541DBF1CEA135594EA0C0F3A
